Archive member included to satisfy reference by file (symbol)

C:\Users\tomas\AppData\Local\Temp\arduino-sketch-3D6AC107FF947055EEB72537F7027E49/..\arduino-core-cache\core_47e1560ce04abac12f346abb2f6d40c8.a(SerialUSB.cpp.o)
                              C:\Users\tomas\AppData\Local\Temp\arduino-sketch-3D6AC107FF947055EEB72537F7027E49\sketch\skinImpedance.ino.cpp.o (Serial)
C:\Users\tomas\AppData\Local\Temp\arduino-sketch-3D6AC107FF947055EEB72537F7027E49/..\arduino-core-cache\core_47e1560ce04abac12f346abb2f6d40c8.a(Print.cpp.o)
                              C:\Users\tomas\AppData\Local\Temp\arduino-sketch-3D6AC107FF947055EEB72537F7027E49\libraries\SdFat\ExFatLib\ExFatDbg.cpp.o (_ZN7arduino5Print5printEPKNS_19__FlashStringHelperE)
C:\Users\tomas\AppData\Local\Temp\arduino-sketch-3D6AC107FF947055EEB72537F7027E49/..\arduino-core-cache\core_47e1560ce04abac12f346abb2f6d40c8.a(String.cpp.o)
                              C:\Users\tomas\AppData\Local\Temp\arduino-sketch-3D6AC107FF947055EEB72537F7027E49\sketch\skinImpedance.ino.cpp.o (_ZN7arduino6StringD2Ev)
C:\Users\tomas\AppData\Local\Temp\arduino-sketch-3D6AC107FF947055EEB72537F7027E49/..\arduino-core-cache\core_47e1560ce04abac12f346abb2f6d40c8.a(delay.cpp.o)
                              C:\Users\tomas\AppData\Local\Temp\arduino-sketch-3D6AC107FF947055EEB72537F7027E49\sketch\skinImpedance.ino.cpp.o (delay)
C:\Users\tomas\AppData\Local\Temp\arduino-sketch-3D6AC107FF947055EEB72537F7027E49/..\arduino-core-cache\core_47e1560ce04abac12f346abb2f6d40c8.a(main.cpp.o)
                              c:/users/tomas/appdata/local/arduino15/packages/rp2040/tools/pqt-gcc/1.4.0-c-0196c06/bin/../lib/gcc/arm-none-eabi/10.3.0/../../../../arm-none-eabi/lib/thumb/crt0.o (main)
C:\Users\tomas\AppData\Local\Temp\arduino-sketch-3D6AC107FF947055EEB72537F7027E49/..\arduino-core-cache\core_47e1560ce04abac12f346abb2f6d40c8.a(stdlib_noniso.cpp.o)
                              C:\Users\tomas\AppData\Local\Temp\arduino-sketch-3D6AC107FF947055EEB72537F7027E49/..\arduino-core-cache\core_47e1560ce04abac12f346abb2f6d40c8.a(String.cpp.o) (ltoa)
C:\Users\tomas\AppData\Local\Temp\arduino-sketch-3D6AC107FF947055EEB72537F7027E49/..\arduino-core-cache\core_47e1560ce04abac12f346abb2f6d40c8.a(wiring_analog.cpp.o)
                              C:\Users\tomas\AppData\Local\Temp\arduino-sketch-3D6AC107FF947055EEB72537F7027E49\sketch\skinImpedance.ino.cpp.o (analogRead)
C:\Users\tomas\AppData\Local\Temp\arduino-sketch-3D6AC107FF947055EEB72537F7027E49/..\arduino-core-cache\core_47e1560ce04abac12f346abb2f6d40c8.a(wiring_digital.cpp.o)
                              C:\Users\tomas\AppData\Local\Temp\arduino-sketch-3D6AC107FF947055EEB72537F7027E49\libraries\SdFat\SpiDriver\SdSpiChipSelect.cpp.o (pinMode)
C:\Users\tomas\AppData\Local\Temp\arduino-sketch-3D6AC107FF947055EEB72537F7027E49/..\arduino-core-cache\core_47e1560ce04abac12f346abb2f6d40c8.a(wiring_private.cpp.o)
                              C:\Users\tomas\AppData\Local\Temp\arduino-sketch-3D6AC107FF947055EEB72537F7027E49/..\arduino-core-cache\core_47e1560ce04abac12f346abb2f6d40c8.a(main.cpp.o) (interrupts)
C:\Users\tomas\AppData\Local\Temp\arduino-sketch-3D6AC107FF947055EEB72537F7027E49/..\arduino-core-cache\core_47e1560ce04abac12f346abb2f6d40c8.a(CoreMutex.cpp.o)
                              C:\Users\tomas\AppData\Local\Temp\arduino-sketch-3D6AC107FF947055EEB72537F7027E49/..\arduino-core-cache\core_47e1560ce04abac12f346abb2f6d40c8.a(SerialUSB.cpp.o) (_ZN9CoreMutexC1EP5mutexb)
C:\Users\tomas\AppData\Local\Temp\arduino-sketch-3D6AC107FF947055EEB72537F7027E49/..\arduino-core-cache\core_47e1560ce04abac12f346abb2f6d40c8.a(RP2040USB.cpp.o)
                              C:\Users\tomas\AppData\Local\Temp\arduino-sketch-3D6AC107FF947055EEB72537F7027E49/..\arduino-core-cache\core_47e1560ce04abac12f346abb2f6d40c8.a(main.cpp.o) (_Z10__USBStartv)
C:\Users\tomas\AppData\Local\Temp\arduino-sketch-3D6AC107FF947055EEB72537F7027E49/..\arduino-core-cache\core_47e1560ce04abac12f346abb2f6d40c8.a(_freertos.cpp.o)
                              C:\Users\tomas\AppData\Local\Temp\arduino-sketch-3D6AC107FF947055EEB72537F7027E49/..\arduino-core-cache\core_47e1560ce04abac12f346abb2f6d40c8.a(CoreMutex.cpp.o) (__get_freertos_mutex_for_ptr)
C:\Users\tomas\AppData\Local\Arduino15\packages\rp2040\hardware\rp2040\2.6.0/lib/libpico.a(adc.c.obj)
                              C:\Users\tomas\AppData\Local\Temp\arduino-sketch-3D6AC107FF947055EEB72537F7027E49/..\arduino-core-cache\core_47e1560ce04abac12f346abb2f6d40c8.a(wiring_analog.cpp.o) (adc_init)
C:\Users\tomas\AppData\Local\Arduino15\packages\rp2040\hardware\rp2040\2.6.0/lib/libpico.a(sync.c.obj)
                              C:\Users\tomas\AppData\Local\Temp\arduino-sketch-3D6AC107FF947055EEB72537F7027E49/..\arduino-core-cache\core_47e1560ce04abac12f346abb2f6d40c8.a(main.cpp.o) (next_striped_spin_lock_num)
C:\Users\tomas\AppData\Local\Arduino15\packages\rp2040\hardware\rp2040\2.6.0/lib/libpico.a(clocks.c.obj)
                              C:\Users\tomas\AppData\Local\Temp\arduino-sketch-3D6AC107FF947055EEB72537F7027E49/..\arduino-core-cache\core_47e1560ce04abac12f346abb2f6d40c8.a(wiring_analog.cpp.o) (clock_get_hz)
C:\Users\tomas\AppData\Local\Arduino15\packages\rp2040\hardware\rp2040\2.6.0/lib/libpico.a(gpio.c.obj)
                              C:\Users\tomas\AppData\Local\Temp\arduino-sketch-3D6AC107FF947055EEB72537F7027E49\sketch\skinImpedance.ino.cpp.o (gpio_set_function)
C:\Users\tomas\AppData\Local\Arduino15\packages\rp2040\hardware\rp2040\2.6.0/lib/libpico.a(irq.c.obj)
                              C:\Users\tomas\AppData\Local\Temp\arduino-sketch-3D6AC107FF947055EEB72537F7027E49/..\arduino-core-cache\core_47e1560ce04abac12f346abb2f6d40c8.a(main.cpp.o) (irq_set_enabled)
C:\Users\tomas\AppData\Local\Arduino15\packages\rp2040\hardware\rp2040\2.6.0/lib/libpico.a(irq_handler_chain.S.obj)
                              C:\Users\tomas\AppData\Local\Arduino15\packages\rp2040\hardware\rp2040\2.6.0/lib/libpico.a(irq.c.obj) (irq_handler_chain_slots)
C:\Users\tomas\AppData\Local\Arduino15\packages\rp2040\hardware\rp2040\2.6.0/lib/libpico.a(time.c.obj)
                              C:\Users\tomas\AppData\Local\Temp\arduino-sketch-3D6AC107FF947055EEB72537F7027E49/..\arduino-core-cache\core_47e1560ce04abac12f346abb2f6d40c8.a(RP2040USB.cpp.o) (alarm_pool_get_default)
C:\Users\tomas\AppData\Local\Arduino15\packages\rp2040\hardware\rp2040\2.6.0/lib/libpico.a(timer.c.obj)
                              C:\Users\tomas\AppData\Local\Arduino15\packages\rp2040\hardware\rp2040\2.6.0/lib/libpico.a(time.c.obj) (hardware_alarm_claim)
C:\Users\tomas\AppData\Local\Arduino15\packages\rp2040\hardware\rp2040\2.6.0/lib/libpico.a(pheap.c.obj)
                              C:\Users\tomas\AppData\Local\Arduino15\packages\rp2040\hardware\rp2040\2.6.0/lib/libpico.a(time.c.obj) (ph_post_alloc_init)
C:\Users\tomas\AppData\Local\Arduino15\packages\rp2040\hardware\rp2040\2.6.0/lib/libpico.a(queue.c.obj)
                              C:\Users\tomas\AppData\Local\Temp\arduino-sketch-3D6AC107FF947055EEB72537F7027E49/..\arduino-core-cache\core_47e1560ce04abac12f346abb2f6d40c8.a(main.cpp.o) (queue_init_with_spinlock)
C:\Users\tomas\AppData\Local\Arduino15\packages\rp2040\hardware\rp2040\2.6.0/lib/libpico.a(mutex.c.obj)
                              C:\Users\tomas\AppData\Local\Temp\arduino-sketch-3D6AC107FF947055EEB72537F7027E49/..\arduino-core-cache\core_47e1560ce04abac12f346abb2f6d40c8.a(main.cpp.o) (mutex_init)
C:\Users\tomas\AppData\Local\Arduino15\packages\rp2040\hardware\rp2040\2.6.0/lib/libpico.a(pll.c.obj)
                              C:\Users\tomas\AppData\Local\Arduino15\packages\rp2040\hardware\rp2040\2.6.0/lib/libpico.a(clocks.c.obj) (pll_init)
C:\Users\tomas\AppData\Local\Arduino15\packages\rp2040\hardware\rp2040\2.6.0/lib/libpico.a(watchdog.c.obj)
                              C:\Users\tomas\AppData\Local\Arduino15\packages\rp2040\hardware\rp2040\2.6.0/lib/libpico.a(clocks.c.obj) (watchdog_start_tick)
C:\Users\tomas\AppData\Local\Arduino15\packages\rp2040\hardware\rp2040\2.6.0/lib/libpico.a(xosc.c.obj)
                              C:\Users\tomas\AppData\Local\Arduino15\packages\rp2040\hardware\rp2040\2.6.0/lib/libpico.a(clocks.c.obj) (xosc_init)
C:\Users\tomas\AppData\Local\Arduino15\packages\rp2040\hardware\rp2040\2.6.0/lib/libpico.a(exception.c.obj)
                              C:\Users\tomas\AppData\Local\Temp\arduino-sketch-3D6AC107FF947055EEB72537F7027E49/..\arduino-core-cache\core_47e1560ce04abac12f346abb2f6d40c8.a(main.cpp.o) (exception_set_exclusive_handler)
C:\Users\tomas\AppData\Local\Arduino15\packages\rp2040\hardware\rp2040\2.6.0/lib/libpico.a(bootrom.c.obj)
                              C:\Users\tomas\AppData\Local\Temp\arduino-sketch-3D6AC107FF947055EEB72537F7027E49/..\arduino-core-cache\core_47e1560ce04abac12f346abb2f6d40c8.a(SerialUSB.cpp.o) (rom_func_lookup)
C:\Users\tomas\AppData\Local\Arduino15\packages\rp2040\hardware\rp2040\2.6.0/lib/libpico.a(pio.c.obj)
                              C:\Users\tomas\AppData\Local\Temp\arduino-sketch-3D6AC107FF947055EEB72537F7027E49/..\arduino-core-cache\core_47e1560ce04abac12f346abb2f6d40c8.a(main.cpp.o) (pio_claim_unused_sm)
C:\Users\tomas\AppData\Local\Arduino15\packages\rp2040\hardware\rp2040\2.6.0/lib/libpico.a(spi.c.obj)
                              C:\Users\tomas\AppData\Local\Temp\arduino-sketch-3D6AC107FF947055EEB72537F7027E49\sketch\skinImpedance.ino.cpp.o (spi_deinit)
C:\Users\tomas\AppData\Local\Arduino15\packages\rp2040\hardware\rp2040\2.6.0/lib/libpico.a(bit_ops_aeabi.S.obj)
                              C:\Users\tomas\AppData\Local\Arduino15\packages\rp2040\hardware\rp2040\2.6.0/lib/libpico.a(pio.c.obj) (__wrap___ctzsi2)
C:\Users\tomas\AppData\Local\Arduino15\packages\rp2040\hardware\rp2040\2.6.0/lib/libpico.a(unique_id.c.obj)
                              C:\Users\tomas\AppData\Local\Temp\arduino-sketch-3D6AC107FF947055EEB72537F7027E49/..\arduino-core-cache\core_47e1560ce04abac12f346abb2f6d40c8.a(RP2040USB.cpp.o) (pico_get_unique_board_id_string)
C:\Users\tomas\AppData\Local\Arduino15\packages\rp2040\hardware\rp2040\2.6.0/lib/libpico.a(stdlib.c.obj)
                              C:\Users\tomas\AppData\Local\Temp\arduino-sketch-3D6AC107FF947055EEB72537F7027E49/..\arduino-core-cache\core_47e1560ce04abac12f346abb2f6d40c8.a(main.cpp.o) (set_sys_clock_pll)
C:\Users\tomas\AppData\Local\Arduino15\packages\rp2040\hardware\rp2040\2.6.0/lib/libpico.a(runtime.c.obj)
                              c:/users/tomas/appdata/local/arduino15/packages/rp2040/tools/pqt-gcc/1.4.0-c-0196c06/bin/../lib/gcc/arm-none-eabi/10.3.0/../../../../arm-none-eabi/lib/thumb/crt0.o (exit)
C:\Users\tomas\AppData\Local\Arduino15\packages\rp2040\hardware\rp2040\2.6.0/lib/libpico.a(divider.S.obj)
                              C:\Users\tomas\AppData\Local\Temp\arduino-sketch-3D6AC107FF947055EEB72537F7027E49\libraries\SdFat\common\FsStructs.cpp.o (__wrap___aeabi_idiv)
C:\Users\tomas\AppData\Local\Arduino15\packages\rp2040\hardware\rp2040\2.6.0/lib/libpico.a(double_aeabi.S.obj)
                              C:\Users\tomas\AppData\Local\Temp\arduino-sketch-3D6AC107FF947055EEB72537F7027E49\libraries\SdFat\common\FmtNumber.cpp.o (__wrap___aeabi_dsub)
C:\Users\tomas\AppData\Local\Arduino15\packages\rp2040\hardware\rp2040\2.6.0/lib/libpico.a(double_init_rom.c.obj)
                              C:\Users\tomas\AppData\Local\Arduino15\packages\rp2040\hardware\rp2040\2.6.0/lib/libpico.a(double_aeabi.S.obj) (__aeabi_double_init)
C:\Users\tomas\AppData\Local\Arduino15\packages\rp2040\hardware\rp2040\2.6.0/lib/libpico.a(double_math.c.obj)
                              C:\Users\tomas\AppData\Local\Arduino15\packages\rp2040\hardware\rp2040\2.6.0/lib/libpico.a(double_aeabi.S.obj) (__wrap_remainder)
C:\Users\tomas\AppData\Local\Arduino15\packages\rp2040\hardware\rp2040\2.6.0/lib/libpico.a(double_v1_rom_shim.S.obj)
                              C:\Users\tomas\AppData\Local\Arduino15\packages\rp2040\hardware\rp2040\2.6.0/lib/libpico.a(double_init_rom.c.obj) (double_table_shim_on_use_helper)
C:\Users\tomas\AppData\Local\Arduino15\packages\rp2040\hardware\rp2040\2.6.0/lib/libpico.a(pico_int64_ops_aeabi.S.obj)
                              C:\Users\tomas\AppData\Local\Temp\arduino-sketch-3D6AC107FF947055EEB72537F7027E49\sketch\skinImpedance.ino.cpp.o (__wrap___aeabi_lmul)
C:\Users\tomas\AppData\Local\Arduino15\packages\rp2040\hardware\rp2040\2.6.0/lib/libpico.a(float_aeabi.S.obj)
                              C:\Users\tomas\AppData\Local\Temp\arduino-sketch-3D6AC107FF947055EEB72537F7027E49/..\arduino-core-cache\core_47e1560ce04abac12f346abb2f6d40c8.a(wiring_analog.cpp.o) (__wrap___aeabi_fsub)
C:\Users\tomas\AppData\Local\Arduino15\packages\rp2040\hardware\rp2040\2.6.0/lib/libpico.a(float_init_rom.c.obj)
                              C:\Users\tomas\AppData\Local\Arduino15\packages\rp2040\hardware\rp2040\2.6.0/lib/libpico.a(float_aeabi.S.obj) (__aeabi_float_init)
C:\Users\tomas\AppData\Local\Arduino15\packages\rp2040\hardware\rp2040\2.6.0/lib/libpico.a(float_math.c.obj)
                              C:\Users\tomas\AppData\Local\Arduino15\packages\rp2040\hardware\rp2040\2.6.0/lib/libpico.a(float_aeabi.S.obj) (__wrap_remainderf)
C:\Users\tomas\AppData\Local\Arduino15\packages\rp2040\hardware\rp2040\2.6.0/lib/libpico.a(float_v1_rom_shim.S.obj)
                              C:\Users\tomas\AppData\Local\Arduino15\packages\rp2040\hardware\rp2040\2.6.0/lib/libpico.a(float_init_rom.c.obj) (float_table_shim_on_use_helper)
C:\Users\tomas\AppData\Local\Arduino15\packages\rp2040\hardware\rp2040\2.6.0/lib/libpico.a(mem_ops_aeabi.S.obj)
                              c:/users/tomas/appdata/local/arduino15/packages/rp2040/tools/pqt-gcc/1.4.0-c-0196c06/bin/../lib/gcc/arm-none-eabi/10.3.0/../../../../arm-none-eabi/lib/thumb/crt0.o (__wrap_memset)
C:\Users\tomas\AppData\Local\Arduino15\packages\rp2040\hardware\rp2040\2.6.0/lib/libpico.a(crt0.S.obj)
                              C:\Users\tomas\AppData\Local\Arduino15\packages\rp2040\hardware\rp2040\2.6.0/lib/libpico.a(exception.c.obj) (__default_isrs_start)
C:\Users\tomas\AppData\Local\Arduino15\packages\rp2040\hardware\rp2040\2.6.0/lib/libpico.a(new_delete.cpp.obj)
                              C:\Users\tomas\AppData\Local\Temp\arduino-sketch-3D6AC107FF947055EEB72537F7027E49/..\arduino-core-cache\core_47e1560ce04abac12f346abb2f6d40c8.a(main.cpp.o) (_Znwj)
C:\Users\tomas\AppData\Local\Arduino15\packages\rp2040\hardware\rp2040\2.6.0/lib/libpico.a(stdio_uart.c.obj)
                              C:\Users\tomas\AppData\Local\Arduino15\packages\rp2040\hardware\rp2040\2.6.0/lib/libpico.a(stdlib.c.obj) (stdio_uart_init)
C:\Users\tomas\AppData\Local\Arduino15\packages\rp2040\hardware\rp2040\2.6.0/lib/libpico.a(multicore.c.obj)
                              C:\Users\tomas\AppData\Local\Temp\arduino-sketch-3D6AC107FF947055EEB72537F7027E49/..\arduino-core-cache\core_47e1560ce04abac12f346abb2f6d40c8.a(main.cpp.o) (multicore_fifo_pop_blocking)
C:\Users\tomas\AppData\Local\Arduino15\packages\rp2040\hardware\rp2040\2.6.0/lib/libpico.a(usbd.c.obj)
                              C:\Users\tomas\AppData\Local\Temp\arduino-sketch-3D6AC107FF947055EEB72537F7027E49/..\arduino-core-cache\core_47e1560ce04abac12f346abb2f6d40c8.a(SerialUSB.cpp.o) (tud_task)
C:\Users\tomas\AppData\Local\Arduino15\packages\rp2040\hardware\rp2040\2.6.0/lib/libpico.a(usbd_control.c.obj)
                              C:\Users\tomas\AppData\Local\Arduino15\packages\rp2040\hardware\rp2040\2.6.0/lib/libpico.a(usbd.c.obj) (tud_control_status)
C:\Users\tomas\AppData\Local\Arduino15\packages\rp2040\hardware\rp2040\2.6.0/lib/libpico.a(cdc_device.c.obj)
                              C:\Users\tomas\AppData\Local\Temp\arduino-sketch-3D6AC107FF947055EEB72537F7027E49/..\arduino-core-cache\core_47e1560ce04abac12f346abb2f6d40c8.a(SerialUSB.cpp.o) (tud_cdc_n_connected)
C:\Users\tomas\AppData\Local\Arduino15\packages\rp2040\hardware\rp2040\2.6.0/lib/libpico.a(hid_device.c.obj)
                              C:\Users\tomas\AppData\Local\Arduino15\packages\rp2040\hardware\rp2040\2.6.0/lib/libpico.a(usbd.c.obj) (hidd_reset)
C:\Users\tomas\AppData\Local\Arduino15\packages\rp2040\hardware\rp2040\2.6.0/lib/libpico.a(tusb.c.obj)
                              C:\Users\tomas\AppData\Local\Temp\arduino-sketch-3D6AC107FF947055EEB72537F7027E49/..\arduino-core-cache\core_47e1560ce04abac12f346abb2f6d40c8.a(RP2040USB.cpp.o) (tusb_init)
C:\Users\tomas\AppData\Local\Arduino15\packages\rp2040\hardware\rp2040\2.6.0/lib/libpico.a(tusb_fifo.c.obj)
                              C:\Users\tomas\AppData\Local\Arduino15\packages\rp2040\hardware\rp2040\2.6.0/lib/libpico.a(cdc_device.c.obj) (tu_fifo_config)
C:\Users\tomas\AppData\Local\Arduino15\packages\rp2040\hardware\rp2040\2.6.0/lib/libpico.a(claim.c.obj)
                              C:\Users\tomas\AppData\Local\Arduino15\packages\rp2040\hardware\rp2040\2.6.0/lib/libpico.a(pio.c.obj) (hw_claim_lock)
C:\Users\tomas\AppData\Local\Arduino15\packages\rp2040\hardware\rp2040\2.6.0/lib/libpico.a(platform.c.obj)
                              C:\Users\tomas\AppData\Local\Arduino15\packages\rp2040\hardware\rp2040\2.6.0/lib/libpico.a(clocks.c.obj) (running_on_fpga)
C:\Users\tomas\AppData\Local\Arduino15\packages\rp2040\hardware\rp2040\2.6.0/lib/libpico.a(lock_core.c.obj)
                              C:\Users\tomas\AppData\Local\Arduino15\packages\rp2040\hardware\rp2040\2.6.0/lib/libpico.a(time.c.obj) (lock_init)
C:\Users\tomas\AppData\Local\Arduino15\packages\rp2040\hardware\rp2040\2.6.0/lib/libpico.a(critical_section.c.obj)
                              C:\Users\tomas\AppData\Local\Arduino15\packages\rp2040\hardware\rp2040\2.6.0/lib/libpico.a(usbd.c.obj) (critical_section_init)
C:\Users\tomas\AppData\Local\Arduino15\packages\rp2040\hardware\rp2040\2.6.0/lib/libpico.a(flash.c.obj)
                              C:\Users\tomas\AppData\Local\Arduino15\packages\rp2040\hardware\rp2040\2.6.0/lib/libpico.a(unique_id.c.obj) (flash_get_unique_id)
C:\Users\tomas\AppData\Local\Arduino15\packages\rp2040\hardware\rp2040\2.6.0/lib/libpico.a(uart.c.obj)
                              C:\Users\tomas\AppData\Local\Arduino15\packages\rp2040\hardware\rp2040\2.6.0/lib/libpico.a(stdio_uart.c.obj) (uart_init)
C:\Users\tomas\AppData\Local\Arduino15\packages\rp2040\hardware\rp2040\2.6.0/lib/libpico.a(dcd_rp2040.c.obj)
                              C:\Users\tomas\AppData\Local\Arduino15\packages\rp2040\hardware\rp2040\2.6.0/lib/libpico.a(usbd.c.obj) (dcd_int_enable)
C:\Users\tomas\AppData\Local\Arduino15\packages\rp2040\hardware\rp2040\2.6.0/lib/libpico.a(rp2040_usb.c.obj)
                              C:\Users\tomas\AppData\Local\Arduino15\packages\rp2040\hardware\rp2040\2.6.0/lib/libpico.a(dcd_rp2040.c.obj) (rp2040_usb_init)
c:/users/tomas/appdata/local/arduino15/packages/rp2040/tools/pqt-gcc/1.4.0-c-0196c06/bin/../lib/gcc/arm-none-eabi/10.3.0/../../../../arm-none-eabi/lib/thumb\libstdc++.a(pure.o)
                              C:\Users\tomas\AppData\Local\Temp\arduino-sketch-3D6AC107FF947055EEB72537F7027E49/..\arduino-core-cache\core_47e1560ce04abac12f346abb2f6d40c8.a(Print.cpp.o) (__cxa_pure_virtual)
c:/users/tomas/appdata/local/arduino15/packages/rp2040/tools/pqt-gcc/1.4.0-c-0196c06/bin/../lib/gcc/arm-none-eabi/10.3.0/../../../../arm-none-eabi/lib/thumb\libstdc++.a(tree.o)
                              C:\Users\tomas\AppData\Local\Temp\arduino-sketch-3D6AC107FF947055EEB72537F7027E49/..\arduino-core-cache\core_47e1560ce04abac12f346abb2f6d40c8.a(wiring_private.cpp.o) (_ZSt18_Rb_tree_incrementPKSt18_Rb_tree_node_base)
c:/users/tomas/appdata/local/arduino15/packages/rp2040/tools/pqt-gcc/1.4.0-c-0196c06/bin/../lib/gcc/arm-none-eabi/10.3.0/../../../../arm-none-eabi/lib/thumb\libstdc++.a(functexcept.o)
                              C:\Users\tomas\AppData\Local\Temp\arduino-sketch-3D6AC107FF947055EEB72537F7027E49/..\arduino-core-cache\core_47e1560ce04abac12f346abb2f6d40c8.a(wiring_private.cpp.o) (_ZSt17__throw_bad_allocv)
c:/users/tomas/appdata/local/arduino15/packages/rp2040/tools/pqt-gcc/1.4.0-c-0196c06/bin/../lib/gcc/arm-none-eabi/10.3.0/../../../../arm-none-eabi/lib/thumb\libstdc++.a(snprintf_lite.o)
                              c:/users/tomas/appdata/local/arduino15/packages/rp2040/tools/pqt-gcc/1.4.0-c-0196c06/bin/../lib/gcc/arm-none-eabi/10.3.0/../../../../arm-none-eabi/lib/thumb\libstdc++.a(functexcept.o) (_ZN9__gnu_cxx15__snprintf_liteEPcjPKcSt9__va_list)
c:/users/tomas/appdata/local/arduino15/packages/rp2040/tools/pqt-gcc/1.4.0-c-0196c06/bin/../lib/gcc/arm-none-eabi/10.3.0/../../../../arm-none-eabi/lib/thumb\libstdc++.a(eh_terminate.o)
                              c:/users/tomas/appdata/local/arduino15/packages/rp2040/tools/pqt-gcc/1.4.0-c-0196c06/bin/../lib/gcc/arm-none-eabi/10.3.0/../../../../arm-none-eabi/lib/thumb\libstdc++.a(pure.o) (_ZSt9terminatev)
c:/users/tomas/appdata/local/arduino15/packages/rp2040/tools/pqt-gcc/1.4.0-c-0196c06/bin/../lib/gcc/arm-none-eabi/10.3.0/../../../../arm-none-eabi/lib/thumb\libstdc++.a(eh_unex_handler.o)
                              c:/users/tomas/appdata/local/arduino15/packages/rp2040/tools/pqt-gcc/1.4.0-c-0196c06/bin/../lib/gcc/arm-none-eabi/10.3.0/../../../../arm-none-eabi/lib/thumb\libstdc++.a(eh_terminate.o) (_ZN10__cxxabiv120__unexpected_handlerE)
c:/users/tomas/appdata/local/arduino15/packages/rp2040/tools/pqt-gcc/1.4.0-c-0196c06/bin/../lib/gcc/arm-none-eabi/10.3.0/../../../../arm-none-eabi/lib/thumb\libstdc++.a(eh_term_handler.o)
                              c:/users/tomas/appdata/local/arduino15/packages/rp2040/tools/pqt-gcc/1.4.0-c-0196c06/bin/../lib/gcc/arm-none-eabi/10.3.0/../../../../arm-none-eabi/lib/thumb\libstdc++.a(eh_terminate.o) (_ZN10__cxxabiv119__terminate_handlerE)
c:/users/tomas/appdata/local/arduino15/packages/rp2040/tools/pqt-gcc/1.4.0-c-0196c06/bin/../lib/gcc/arm-none-eabi/10.3.0/../../../../arm-none-eabi/lib/thumb\libc.a(lib_a-abort.o)
                              c:/users/tomas/appdata/local/arduino15/packages/rp2040/tools/pqt-gcc/1.4.0-c-0196c06/bin/../lib/gcc/arm-none-eabi/10.3.0/../../../../arm-none-eabi/lib/thumb\libstdc++.a(functexcept.o) (abort)
c:/users/tomas/appdata/local/arduino15/packages/rp2040/tools/pqt-gcc/1.4.0-c-0196c06/bin/../lib/gcc/arm-none-eabi/10.3.0/../../../../arm-none-eabi/lib/thumb\libc.a(lib_a-atexit.o)
                              c:/users/tomas/appdata/local/arduino15/packages/rp2040/tools/pqt-gcc/1.4.0-c-0196c06/bin/../lib/gcc/arm-none-eabi/10.3.0/../../../../arm-none-eabi/lib/thumb/crt0.o (atexit)
c:/users/tomas/appdata/local/arduino15/packages/rp2040/tools/pqt-gcc/1.4.0-c-0196c06/bin/../lib/gcc/arm-none-eabi/10.3.0/../../../../arm-none-eabi/lib/thumb\libc.a(lib_a-atof.o)
                              C:\Users\tomas\AppData\Local\Temp\arduino-sketch-3D6AC107FF947055EEB72537F7027E49/..\arduino-core-cache\core_47e1560ce04abac12f346abb2f6d40c8.a(String.cpp.o) (atof)
c:/users/tomas/appdata/local/arduino15/packages/rp2040/tools/pqt-gcc/1.4.0-c-0196c06/bin/../lib/gcc/arm-none-eabi/10.3.0/../../../../arm-none-eabi/lib/thumb\libc.a(lib_a-atol.o)
                              C:\Users\tomas\AppData\Local\Temp\arduino-sketch-3D6AC107FF947055EEB72537F7027E49/..\arduino-core-cache\core_47e1560ce04abac12f346abb2f6d40c8.a(String.cpp.o) (atol)
c:/users/tomas/appdata/local/arduino15/packages/rp2040/tools/pqt-gcc/1.4.0-c-0196c06/bin/../lib/gcc/arm-none-eabi/10.3.0/../../../../arm-none-eabi/lib/thumb\libc.a(lib_a-calloc.o)
                              C:\Users\tomas\AppData\Local\Temp\arduino-sketch-3D6AC107FF947055EEB72537F7027E49\sketch\skinImpedance.ino.cpp.o (calloc)
c:/users/tomas/appdata/local/arduino15/packages/rp2040/tools/pqt-gcc/1.4.0-c-0196c06/bin/../lib/gcc/arm-none-eabi/10.3.0/../../../../arm-none-eabi/lib/thumb\libc.a(lib_a-callocr.o)
                              c:/users/tomas/appdata/local/arduino15/packages/rp2040/tools/pqt-gcc/1.4.0-c-0196c06/bin/../lib/gcc/arm-none-eabi/10.3.0/../../../../arm-none-eabi/lib/thumb\libc.a(lib_a-calloc.o) (_calloc_r)
c:/users/tomas/appdata/local/arduino15/packages/rp2040/tools/pqt-gcc/1.4.0-c-0196c06/bin/../lib/gcc/arm-none-eabi/10.3.0/../../../../arm-none-eabi/lib/thumb\libc.a(lib_a-errno.o)
                              c:/users/tomas/appdata/local/arduino15/packages/rp2040/tools/pqt-gcc/1.4.0-c-0196c06/bin/../lib/gcc/arm-none-eabi/10.3.0/../../../../arm-none-eabi/lib/thumb\libc.a(lib_a-callocr.o) (__errno)
c:/users/tomas/appdata/local/arduino15/packages/rp2040/tools/pqt-gcc/1.4.0-c-0196c06/bin/../lib/gcc/arm-none-eabi/10.3.0/../../../../arm-none-eabi/lib/thumb\libc.a(lib_a-findfp.o)
                              C:\Users\tomas\AppData\Local\Temp\arduino-sketch-3D6AC107FF947055EEB72537F7027E49/..\arduino-core-cache\core_47e1560ce04abac12f346abb2f6d40c8.a(main.cpp.o) (__sf_fake_stderr)
c:/users/tomas/appdata/local/arduino15/packages/rp2040/tools/pqt-gcc/1.4.0-c-0196c06/bin/../lib/gcc/arm-none-eabi/10.3.0/../../../../arm-none-eabi/lib/thumb\libc.a(lib_a-fini.o)
                              c:/users/tomas/appdata/local/arduino15/packages/rp2040/tools/pqt-gcc/1.4.0-c-0196c06/bin/../lib/gcc/arm-none-eabi/10.3.0/../../../../arm-none-eabi/lib/thumb/crt0.o (__libc_fini_array)
c:/users/tomas/appdata/local/arduino15/packages/rp2040/tools/pqt-gcc/1.4.0-c-0196c06/bin/../lib/gcc/arm-none-eabi/10.3.0/../../../../arm-none-eabi/lib/thumb\libc.a(lib_a-fwalk.o)
                              c:/users/tomas/appdata/local/arduino15/packages/rp2040/tools/pqt-gcc/1.4.0-c-0196c06/bin/../lib/gcc/arm-none-eabi/10.3.0/../../../../arm-none-eabi/lib/thumb\libc.a(lib_a-findfp.o) (_fwalk)
c:/users/tomas/appdata/local/arduino15/packages/rp2040/tools/pqt-gcc/1.4.0-c-0196c06/bin/../lib/gcc/arm-none-eabi/10.3.0/../../../../arm-none-eabi/lib/thumb\libc.a(lib_a-impure.o)
                              c:/users/tomas/appdata/local/arduino15/packages/rp2040/tools/pqt-gcc/1.4.0-c-0196c06/bin/../lib/gcc/arm-none-eabi/10.3.0/../../../../arm-none-eabi/lib/thumb\libc.a(lib_a-findfp.o) (_global_impure_ptr)
c:/users/tomas/appdata/local/arduino15/packages/rp2040/tools/pqt-gcc/1.4.0-c-0196c06/bin/../lib/gcc/arm-none-eabi/10.3.0/../../../../arm-none-eabi/lib/thumb\libc.a(lib_a-init.o)
                              c:/users/tomas/appdata/local/arduino15/packages/rp2040/tools/pqt-gcc/1.4.0-c-0196c06/bin/../lib/gcc/arm-none-eabi/10.3.0/../../../../arm-none-eabi/lib/thumb/crt0.o (__libc_init_array)
c:/users/tomas/appdata/local/arduino15/packages/rp2040/tools/pqt-gcc/1.4.0-c-0196c06/bin/../lib/gcc/arm-none-eabi/10.3.0/../../../../arm-none-eabi/lib/thumb\libc.a(lib_a-isalpha.o)
                              C:\Users\tomas\AppData\Local\Temp\arduino-sketch-3D6AC107FF947055EEB72537F7027E49\libraries\SdFat\iostream\istream.cpp.o (isalpha)
c:/users/tomas/appdata/local/arduino15/packages/rp2040/tools/pqt-gcc/1.4.0-c-0196c06/bin/../lib/gcc/arm-none-eabi/10.3.0/../../../../arm-none-eabi/lib/thumb\libc.a(lib_a-isspace.o)
                              C:\Users\tomas\AppData\Local\Temp\arduino-sketch-3D6AC107FF947055EEB72537F7027E49\libraries\SdFat\iostream\istream.cpp.o (isspace)
c:/users/tomas/appdata/local/arduino15/packages/rp2040/tools/pqt-gcc/1.4.0-c-0196c06/bin/../lib/gcc/arm-none-eabi/10.3.0/../../../../arm-none-eabi/lib/thumb\libc.a(lib_a-isupper.o)
                              C:\Users\tomas\AppData\Local\Temp\arduino-sketch-3D6AC107FF947055EEB72537F7027E49\libraries\SdFat\iostream\istream.cpp.o (isupper)
c:/users/tomas/appdata/local/arduino15/packages/rp2040/tools/pqt-gcc/1.4.0-c-0196c06/bin/../lib/gcc/arm-none-eabi/10.3.0/../../../../arm-none-eabi/lib/thumb\libc.a(lib_a-itoa.o)
                              C:\Users\tomas\AppData\Local\Temp\arduino-sketch-3D6AC107FF947055EEB72537F7027E49/..\arduino-core-cache\core_47e1560ce04abac12f346abb2f6d40c8.a(String.cpp.o) (itoa)
c:/users/tomas/appdata/local/arduino15/packages/rp2040/tools/pqt-gcc/1.4.0-c-0196c06/bin/../lib/gcc/arm-none-eabi/10.3.0/../../../../arm-none-eabi/lib/thumb\libc.a(lib_a-malloc.o)
                              C:\Users\tomas\AppData\Local\Temp\arduino-sketch-3D6AC107FF947055EEB72537F7027E49\sketch\skinImpedance.ino.cpp.o (malloc)
c:/users/tomas/appdata/local/arduino15/packages/rp2040/tools/pqt-gcc/1.4.0-c-0196c06/bin/../lib/gcc/arm-none-eabi/10.3.0/../../../../arm-none-eabi/lib/thumb\libc.a(lib_a-mallocr.o)
                              c:/users/tomas/appdata/local/arduino15/packages/rp2040/tools/pqt-gcc/1.4.0-c-0196c06/bin/../lib/gcc/arm-none-eabi/10.3.0/../../../../arm-none-eabi/lib/thumb\libc.a(lib_a-callocr.o) (_malloc_r)
c:/users/tomas/appdata/local/arduino15/packages/rp2040/tools/pqt-gcc/1.4.0-c-0196c06/bin/../lib/gcc/arm-none-eabi/10.3.0/../../../../arm-none-eabi/lib/thumb\libc.a(lib_a-memchr-stub.o)
                              C:\Users\tomas\AppData\Local\Temp\arduino-sketch-3D6AC107FF947055EEB72537F7027E49\libraries\SdFat\iostream\StdioStream.cpp.o (memchr)
c:/users/tomas/appdata/local/arduino15/packages/rp2040/tools/pqt-gcc/1.4.0-c-0196c06/bin/../lib/gcc/arm-none-eabi/10.3.0/../../../../arm-none-eabi/lib/thumb\libc.a(lib_a-memcmp.o)
                              C:\Users\tomas\AppData\Local\Temp\arduino-sketch-3D6AC107FF947055EEB72537F7027E49\libraries\SdFat\FatLib\FatFileLFN.cpp.o (memcmp)
c:/users/tomas/appdata/local/arduino15/packages/rp2040/tools/pqt-gcc/1.4.0-c-0196c06/bin/../lib/gcc/arm-none-eabi/10.3.0/../../../../arm-none-eabi/lib/thumb\libc.a(lib_a-memmove.o)
                              C:\Users\tomas\AppData\Local\Temp\arduino-sketch-3D6AC107FF947055EEB72537F7027E49/..\arduino-core-cache\core_47e1560ce04abac12f346abb2f6d40c8.a(String.cpp.o) (memmove)
c:/users/tomas/appdata/local/arduino15/packages/rp2040/tools/pqt-gcc/1.4.0-c-0196c06/bin/../lib/gcc/arm-none-eabi/10.3.0/../../../../arm-none-eabi/lib/thumb\libc.a(lib_a-mlock.o)
                              c:/users/tomas/appdata/local/arduino15/packages/rp2040/tools/pqt-gcc/1.4.0-c-0196c06/bin/../lib/gcc/arm-none-eabi/10.3.0/../../../../arm-none-eabi/lib/thumb\libc.a(lib_a-mallocr.o) (__malloc_lock)
c:/users/tomas/appdata/local/arduino15/packages/rp2040/tools/pqt-gcc/1.4.0-c-0196c06/bin/../lib/gcc/arm-none-eabi/10.3.0/../../../../arm-none-eabi/lib/thumb\libc.a(lib_a-nano-vfprintf_float.o)
                              (_printf_float)
c:/users/tomas/appdata/local/arduino15/packages/rp2040/tools/pqt-gcc/1.4.0-c-0196c06/bin/../lib/gcc/arm-none-eabi/10.3.0/../../../../arm-none-eabi/lib/thumb\libc.a(lib_a-nano-vfprintf_i.o)
                              c:/users/tomas/appdata/local/arduino15/packages/rp2040/tools/pqt-gcc/1.4.0-c-0196c06/bin/../lib/gcc/arm-none-eabi/10.3.0/../../../../arm-none-eabi/lib/thumb\libc.a(lib_a-nano-vfprintf_float.o) (_printf_common)
c:/users/tomas/appdata/local/arduino15/packages/rp2040/tools/pqt-gcc/1.4.0-c-0196c06/bin/../lib/gcc/arm-none-eabi/10.3.0/../../../../arm-none-eabi/lib/thumb\libc.a(lib_a-nano-vfscanf_float.o)
                              (_scanf_float)
c:/users/tomas/appdata/local/arduino15/packages/rp2040/tools/pqt-gcc/1.4.0-c-0196c06/bin/../lib/gcc/arm-none-eabi/10.3.0/../../../../arm-none-eabi/lib/thumb\libc.a(lib_a-printf.o)
                              C:\Users\tomas\AppData\Local\Arduino15\packages\rp2040\hardware\rp2040\2.6.0/lib/libpico.a(time.c.obj) (printf)
c:/users/tomas/appdata/local/arduino15/packages/rp2040/tools/pqt-gcc/1.4.0-c-0196c06/bin/../lib/gcc/arm-none-eabi/10.3.0/../../../../arm-none-eabi/lib/thumb\libc.a(lib_a-putchar.o)
                              C:\Users\tomas\AppData\Local\Arduino15\packages\rp2040\hardware\rp2040\2.6.0/lib/libpico.a(pheap.c.obj) (putchar)
c:/users/tomas/appdata/local/arduino15/packages/rp2040/tools/pqt-gcc/1.4.0-c-0196c06/bin/../lib/gcc/arm-none-eabi/10.3.0/../../../../arm-none-eabi/lib/thumb\libc.a(lib_a-puts.o)
                              C:\Users\tomas\AppData\Local\Arduino15\packages\rp2040\hardware\rp2040\2.6.0/lib/libpico.a(runtime.c.obj) (puts)
c:/users/tomas/appdata/local/arduino15/packages/rp2040/tools/pqt-gcc/1.4.0-c-0196c06/bin/../lib/gcc/arm-none-eabi/10.3.0/../../../../arm-none-eabi/lib/thumb\libc.a(lib_a-realloc.o)
                              C:\Users\tomas\AppData\Local\Temp\arduino-sketch-3D6AC107FF947055EEB72537F7027E49/..\arduino-core-cache\core_47e1560ce04abac12f346abb2f6d40c8.a(String.cpp.o) (realloc)
c:/users/tomas/appdata/local/arduino15/packages/rp2040/tools/pqt-gcc/1.4.0-c-0196c06/bin/../lib/gcc/arm-none-eabi/10.3.0/../../../../arm-none-eabi/lib/thumb\libc.a(lib_a-reallocr.o)
                              c:/users/tomas/appdata/local/arduino15/packages/rp2040/tools/pqt-gcc/1.4.0-c-0196c06/bin/../lib/gcc/arm-none-eabi/10.3.0/../../../../arm-none-eabi/lib/thumb\libc.a(lib_a-realloc.o) (_realloc_r)
c:/users/tomas/appdata/local/arduino15/packages/rp2040/tools/pqt-gcc/1.4.0-c-0196c06/bin/../lib/gcc/arm-none-eabi/10.3.0/../../../../arm-none-eabi/lib/thumb\libc.a(lib_a-sbrkr.o)
                              c:/users/tomas/appdata/local/arduino15/packages/rp2040/tools/pqt-gcc/1.4.0-c-0196c06/bin/../lib/gcc/arm-none-eabi/10.3.0/../../../../arm-none-eabi/lib/thumb\libc.a(lib_a-mallocr.o) (_sbrk_r)
c:/users/tomas/appdata/local/arduino15/packages/rp2040/tools/pqt-gcc/1.4.0-c-0196c06/bin/../lib/gcc/arm-none-eabi/10.3.0/../../../../arm-none-eabi/lib/thumb\libc.a(lib_a-sf_nan.o)
                              c:/users/tomas/appdata/local/arduino15/packages/rp2040/tools/pqt-gcc/1.4.0-c-0196c06/bin/../lib/gcc/arm-none-eabi/10.3.0/../../../../arm-none-eabi/lib/thumb\libc.a(lib_a-nano-vfscanf_float.o) (nanf)
c:/users/tomas/appdata/local/arduino15/packages/rp2040/tools/pqt-gcc/1.4.0-c-0196c06/bin/../lib/gcc/arm-none-eabi/10.3.0/../../../../arm-none-eabi/lib/thumb\libc.a(lib_a-signal.o)
                              c:/users/tomas/appdata/local/arduino15/packages/rp2040/tools/pqt-gcc/1.4.0-c-0196c06/bin/../lib/gcc/arm-none-eabi/10.3.0/../../../../arm-none-eabi/lib/thumb\libc.a(lib_a-abort.o) (raise)
c:/users/tomas/appdata/local/arduino15/packages/rp2040/tools/pqt-gcc/1.4.0-c-0196c06/bin/../lib/gcc/arm-none-eabi/10.3.0/../../../../arm-none-eabi/lib/thumb\libc.a(lib_a-signalr.o)
                              c:/users/tomas/appdata/local/arduino15/packages/rp2040/tools/pqt-gcc/1.4.0-c-0196c06/bin/../lib/gcc/arm-none-eabi/10.3.0/../../../../arm-none-eabi/lib/thumb\libc.a(lib_a-signal.o) (_kill_r)
c:/users/tomas/appdata/local/arduino15/packages/rp2040/tools/pqt-gcc/1.4.0-c-0196c06/bin/../lib/gcc/arm-none-eabi/10.3.0/../../../../arm-none-eabi/lib/thumb\libc.a(lib_a-sprintf.o)
                              C:\Users\tomas\AppData\Local\Temp\arduino-sketch-3D6AC107FF947055EEB72537F7027E49\sketch\skinImpedance.ino.cpp.o (sprintf)
c:/users/tomas/appdata/local/arduino15/packages/rp2040/tools/pqt-gcc/1.4.0-c-0196c06/bin/../lib/gcc/arm-none-eabi/10.3.0/../../../../arm-none-eabi/lib/thumb\libc.a(lib_a-stdio.o)
                              c:/users/tomas/appdata/local/arduino15/packages/rp2040/tools/pqt-gcc/1.4.0-c-0196c06/bin/../lib/gcc/arm-none-eabi/10.3.0/../../../../arm-none-eabi/lib/thumb\libc.a(lib_a-findfp.o) (__sread)
c:/users/tomas/appdata/local/arduino15/packages/rp2040/tools/pqt-gcc/1.4.0-c-0196c06/bin/../lib/gcc/arm-none-eabi/10.3.0/../../../../arm-none-eabi/lib/thumb\libc.a(lib_a-strchr.o)
                              C:\Users\tomas\AppData\Local\Temp\arduino-sketch-3D6AC107FF947055EEB72537F7027E49\libraries\SdFat\ExFatLib\ExFatFile.cpp.o (strchr)
c:/users/tomas/appdata/local/arduino15/packages/rp2040/tools/pqt-gcc/1.4.0-c-0196c06/bin/../lib/gcc/arm-none-eabi/10.3.0/../../../../arm-none-eabi/lib/thumb\libc.a(lib_a-strcmp.o)
                              C:\Users\tomas\AppData\Local\Temp\arduino-sketch-3D6AC107FF947055EEB72537F7027E49/..\arduino-core-cache\core_47e1560ce04abac12f346abb2f6d40c8.a(String.cpp.o) (strcmp)
c:/users/tomas/appdata/local/arduino15/packages/rp2040/tools/pqt-gcc/1.4.0-c-0196c06/bin/../lib/gcc/arm-none-eabi/10.3.0/../../../../arm-none-eabi/lib/thumb\libc.a(lib_a-strcpy.o)
                              C:\Users\tomas\AppData\Local\Temp\arduino-sketch-3D6AC107FF947055EEB72537F7027E49\sketch\skinImpedance.ino.cpp.o (strcpy)
c:/users/tomas/appdata/local/arduino15/packages/rp2040/tools/pqt-gcc/1.4.0-c-0196c06/bin/../lib/gcc/arm-none-eabi/10.3.0/../../../../arm-none-eabi/lib/thumb\libc.a(lib_a-strlen.o)
                              C:\Users\tomas\AppData\Local\Temp\arduino-sketch-3D6AC107FF947055EEB72537F7027E49\sketch\skinImpedance.ino.cpp.o (strlen)
c:/users/tomas/appdata/local/arduino15/packages/rp2040/tools/pqt-gcc/1.4.0-c-0196c06/bin/../lib/gcc/arm-none-eabi/10.3.0/../../../../arm-none-eabi/lib/thumb\libc.a(lib_a-strncmp.o)
                              C:\Users\tomas\AppData\Local\Temp\arduino-sketch-3D6AC107FF947055EEB72537F7027E49\libraries\SdFat\ExFatLib\ExFatPartition.cpp.o (strncmp)
c:/users/tomas/appdata/local/arduino15/packages/rp2040/tools/pqt-gcc/1.4.0-c-0196c06/bin/../lib/gcc/arm-none-eabi/10.3.0/../../../../arm-none-eabi/lib/thumb\libc.a(lib_a-strncpy.o)
                              C:\Users\tomas\AppData\Local\Temp\arduino-sketch-3D6AC107FF947055EEB72537F7027E49/..\arduino-core-cache\core_47e1560ce04abac12f346abb2f6d40c8.a(String.cpp.o) (strncpy)
c:/users/tomas/appdata/local/arduino15/packages/rp2040/tools/pqt-gcc/1.4.0-c-0196c06/bin/../lib/gcc/arm-none-eabi/10.3.0/../../../../arm-none-eabi/lib/thumb\libc.a(lib_a-strrchr.o)
                              C:\Users\tomas\AppData\Local\Temp\arduino-sketch-3D6AC107FF947055EEB72537F7027E49/..\arduino-core-cache\core_47e1560ce04abac12f346abb2f6d40c8.a(String.cpp.o) (strrchr)
c:/users/tomas/appdata/local/arduino15/packages/rp2040/tools/pqt-gcc/1.4.0-c-0196c06/bin/../lib/gcc/arm-none-eabi/10.3.0/../../../../arm-none-eabi/lib/thumb\libc.a(lib_a-strstr.o)
                              C:\Users\tomas\AppData\Local\Temp\arduino-sketch-3D6AC107FF947055EEB72537F7027E49/..\arduino-core-cache\core_47e1560ce04abac12f346abb2f6d40c8.a(String.cpp.o) (strstr)
c:/users/tomas/appdata/local/arduino15/packages/rp2040/tools/pqt-gcc/1.4.0-c-0196c06/bin/../lib/gcc/arm-none-eabi/10.3.0/../../../../arm-none-eabi/lib/thumb\libc.a(lib_a-strtod.o)
                              c:/users/tomas/appdata/local/arduino15/packages/rp2040/tools/pqt-gcc/1.4.0-c-0196c06/bin/../lib/gcc/arm-none-eabi/10.3.0/../../../../arm-none-eabi/lib/thumb\libc.a(lib_a-nano-vfscanf_float.o) (_strtod_r)
c:/users/tomas/appdata/local/arduino15/packages/rp2040/tools/pqt-gcc/1.4.0-c-0196c06/bin/../lib/gcc/arm-none-eabi/10.3.0/../../../../arm-none-eabi/lib/thumb\libc.a(lib_a-strtol.o)
                              c:/users/tomas/appdata/local/arduino15/packages/rp2040/tools/pqt-gcc/1.4.0-c-0196c06/bin/../lib/gcc/arm-none-eabi/10.3.0/../../../../arm-none-eabi/lib/thumb\libc.a(lib_a-atol.o) (_strtol_r)
c:/users/tomas/appdata/local/arduino15/packages/rp2040/tools/pqt-gcc/1.4.0-c-0196c06/bin/../lib/gcc/arm-none-eabi/10.3.0/../../../../arm-none-eabi/lib/thumb\libc.a(lib_a-syssbrk.o)
                              C:\Users\tomas\AppData\Local\Temp\arduino-sketch-3D6AC107FF947055EEB72537F7027E49\libraries\SdFat\FreeStack.cpp.o (sbrk)
c:/users/tomas/appdata/local/arduino15/packages/rp2040/tools/pqt-gcc/1.4.0-c-0196c06/bin/../lib/gcc/arm-none-eabi/10.3.0/../../../../arm-none-eabi/lib/thumb\libc.a(lib_a-tolower.o)
                              C:\Users\tomas\AppData\Local\Temp\arduino-sketch-3D6AC107FF947055EEB72537F7027E49/..\arduino-core-cache\core_47e1560ce04abac12f346abb2f6d40c8.a(String.cpp.o) (tolower)
c:/users/tomas/appdata/local/arduino15/packages/rp2040/tools/pqt-gcc/1.4.0-c-0196c06/bin/../lib/gcc/arm-none-eabi/10.3.0/../../../../arm-none-eabi/lib/thumb\libc.a(lib_a-toupper.o)
                              C:\Users\tomas\AppData\Local\Temp\arduino-sketch-3D6AC107FF947055EEB72537F7027E49/..\arduino-core-cache\core_47e1560ce04abac12f346abb2f6d40c8.a(String.cpp.o) (toupper)
c:/users/tomas/appdata/local/arduino15/packages/rp2040/tools/pqt-gcc/1.4.0-c-0196c06/bin/../lib/gcc/arm-none-eabi/10.3.0/../../../../arm-none-eabi/lib/thumb\libc.a(lib_a-utoa.o)
                              c:/users/tomas/appdata/local/arduino15/packages/rp2040/tools/pqt-gcc/1.4.0-c-0196c06/bin/../lib/gcc/arm-none-eabi/10.3.0/../../../../arm-none-eabi/lib/thumb\libc.a(lib_a-itoa.o) (__utoa)
c:/users/tomas/appdata/local/arduino15/packages/rp2040/tools/pqt-gcc/1.4.0-c-0196c06/bin/../lib/gcc/arm-none-eabi/10.3.0/../../../../arm-none-eabi/lib/thumb\libc.a(lib_a-vprintf.o)
                              C:\Users\tomas\AppData\Local\Arduino15\packages\rp2040\hardware\rp2040\2.6.0/lib/libpico.a(runtime.c.obj) (vprintf)
c:/users/tomas/appdata/local/arduino15/packages/rp2040/tools/pqt-gcc/1.4.0-c-0196c06/bin/../lib/gcc/arm-none-eabi/10.3.0/../../../../arm-none-eabi/lib/thumb\libc.a(lib_a-vsnprintf.o)
                              C:\Users\tomas\AppData\Local\Temp\arduino-sketch-3D6AC107FF947055EEB72537F7027E49/..\arduino-core-cache\core_47e1560ce04abac12f346abb2f6d40c8.a(Print.cpp.o) (vsnprintf)
c:/users/tomas/appdata/local/arduino15/packages/rp2040/tools/pqt-gcc/1.4.0-c-0196c06/bin/../lib/gcc/arm-none-eabi/10.3.0/../../../../arm-none-eabi/lib/thumb\libc.a(lib_a-writer.o)
                              c:/users/tomas/appdata/local/arduino15/packages/rp2040/tools/pqt-gcc/1.4.0-c-0196c06/bin/../lib/gcc/arm-none-eabi/10.3.0/../../../../arm-none-eabi/lib/thumb\libc.a(lib_a-stdio.o) (_write_r)
c:/users/tomas/appdata/local/arduino15/packages/rp2040/tools/pqt-gcc/1.4.0-c-0196c06/bin/../lib/gcc/arm-none-eabi/10.3.0/../../../../arm-none-eabi/lib/thumb\libc.a(lib_a-__atexit.o)
                              c:/users/tomas/appdata/local/arduino15/packages/rp2040/tools/pqt-gcc/1.4.0-c-0196c06/bin/../lib/gcc/arm-none-eabi/10.3.0/../../../../arm-none-eabi/lib/thumb\libc.a(lib_a-atexit.o) (__register_exitproc)
c:/users/tomas/appdata/local/arduino15/packages/rp2040/tools/pqt-gcc/1.4.0-c-0196c06/bin/../lib/gcc/arm-none-eabi/10.3.0/../../../../arm-none-eabi/lib/thumb\libc.a(lib_a-__call_atexit.o)
                              c:/users/tomas/appdata/local/arduino15/packages/rp2040/tools/pqt-gcc/1.4.0-c-0196c06/bin/../lib/gcc/arm-none-eabi/10.3.0/../../../../arm-none-eabi/lib/thumb\libc.a(lib_a-__atexit.o) (__atexit_recursive_mutex)
c:/users/tomas/appdata/local/arduino15/packages/rp2040/tools/pqt-gcc/1.4.0-c-0196c06/bin/../lib/gcc/arm-none-eabi/10.3.0/../../../../arm-none-eabi/lib/thumb\libc.a(lib_a-closer.o)
                              c:/users/tomas/appdata/local/arduino15/packages/rp2040/tools/pqt-gcc/1.4.0-c-0196c06/bin/../lib/gcc/arm-none-eabi/10.3.0/../../../../arm-none-eabi/lib/thumb\libc.a(lib_a-stdio.o) (_close_r)
c:/users/tomas/appdata/local/arduino15/packages/rp2040/tools/pqt-gcc/1.4.0-c-0196c06/bin/../lib/gcc/arm-none-eabi/10.3.0/../../../../arm-none-eabi/lib/thumb\libc.a(lib_a-ctype_.o)
                              c:/users/tomas/appdata/local/arduino15/packages/rp2040/tools/pqt-gcc/1.4.0-c-0196c06/bin/../lib/gcc/arm-none-eabi/10.3.0/../../../../arm-none-eabi/lib/thumb\libc.a(lib_a-isalpha.o) (_ctype_)
c:/users/tomas/appdata/local/arduino15/packages/rp2040/tools/pqt-gcc/1.4.0-c-0196c06/bin/../lib/gcc/arm-none-eabi/10.3.0/../../../../arm-none-eabi/lib/thumb\libc.a(lib_a-dtoa.o)
                              c:/users/tomas/appdata/local/arduino15/packages/rp2040/tools/pqt-gcc/1.4.0-c-0196c06/bin/../lib/gcc/arm-none-eabi/10.3.0/../../../../arm-none-eabi/lib/thumb\libc.a(lib_a-nano-vfprintf_float.o) (_dtoa_r)
c:/users/tomas/appdata/local/arduino15/packages/rp2040/tools/pqt-gcc/1.4.0-c-0196c06/bin/../lib/gcc/arm-none-eabi/10.3.0/../../../../arm-none-eabi/lib/thumb\libc.a(lib_a-fclose.o)
                              c:/users/tomas/appdata/local/arduino15/packages/rp2040/tools/pqt-gcc/1.4.0-c-0196c06/bin/../lib/gcc/arm-none-eabi/10.3.0/../../../../arm-none-eabi/lib/thumb\libc.a(lib_a-findfp.o) (_fclose_r)
c:/users/tomas/appdata/local/arduino15/packages/rp2040/tools/pqt-gcc/1.4.0-c-0196c06/bin/../lib/gcc/arm-none-eabi/10.3.0/../../../../arm-none-eabi/lib/thumb\libc.a(lib_a-fflush.o)
                              c:/users/tomas/appdata/local/arduino15/packages/rp2040/tools/pqt-gcc/1.4.0-c-0196c06/bin/../lib/gcc/arm-none-eabi/10.3.0/../../../../arm-none-eabi/lib/thumb\libc.a(lib_a-fclose.o) (__sflush_r)
c:/users/tomas/appdata/local/arduino15/packages/rp2040/tools/pqt-gcc/1.4.0-c-0196c06/bin/../lib/gcc/arm-none-eabi/10.3.0/../../../../arm-none-eabi/lib/thumb\libc.a(lib_a-freer.o)
                              c:/users/tomas/appdata/local/arduino15/packages/rp2040/tools/pqt-gcc/1.4.0-c-0196c06/bin/../lib/gcc/arm-none-eabi/10.3.0/../../../../arm-none-eabi/lib/thumb\libc.a(lib_a-malloc.o) (_free_r)
c:/users/tomas/appdata/local/arduino15/packages/rp2040/tools/pqt-gcc/1.4.0-c-0196c06/bin/../lib/gcc/arm-none-eabi/10.3.0/../../../../arm-none-eabi/lib/thumb\libc.a(lib_a-fvwrite.o)
                              c:/users/tomas/appdata/local/arduino15/packages/rp2040/tools/pqt-gcc/1.4.0-c-0196c06/bin/../lib/gcc/arm-none-eabi/10.3.0/../../../../arm-none-eabi/lib/thumb\libc.a(lib_a-puts.o) (__sfvwrite_r)
c:/users/tomas/appdata/local/arduino15/packages/rp2040/tools/pqt-gcc/1.4.0-c-0196c06/bin/../lib/gcc/arm-none-eabi/10.3.0/../../../../arm-none-eabi/lib/thumb\libc.a(lib_a-gdtoa-gethex.o)
                              c:/users/tomas/appdata/local/arduino15/packages/rp2040/tools/pqt-gcc/1.4.0-c-0196c06/bin/../lib/gcc/arm-none-eabi/10.3.0/../../../../arm-none-eabi/lib/thumb\libc.a(lib_a-strtod.o) (__gethex)
c:/users/tomas/appdata/local/arduino15/packages/rp2040/tools/pqt-gcc/1.4.0-c-0196c06/bin/../lib/gcc/arm-none-eabi/10.3.0/../../../../arm-none-eabi/lib/thumb\libc.a(lib_a-gdtoa-hexnan.o)
                              c:/users/tomas/appdata/local/arduino15/packages/rp2040/tools/pqt-gcc/1.4.0-c-0196c06/bin/../lib/gcc/arm-none-eabi/10.3.0/../../../../arm-none-eabi/lib/thumb\libc.a(lib_a-strtod.o) (__match)
c:/users/tomas/appdata/local/arduino15/packages/rp2040/tools/pqt-gcc/1.4.0-c-0196c06/bin/../lib/gcc/arm-none-eabi/10.3.0/../../../../arm-none-eabi/lib/thumb\libc.a(lib_a-lnumeric.o)
                              c:/users/tomas/appdata/local/arduino15/packages/rp2040/tools/pqt-gcc/1.4.0-c-0196c06/bin/../lib/gcc/arm-none-eabi/10.3.0/../../../../arm-none-eabi/lib/thumb\libc.a(lib_a-strtod.o) (_C_numeric_locale)
c:/users/tomas/appdata/local/arduino15/packages/rp2040/tools/pqt-gcc/1.4.0-c-0196c06/bin/../lib/gcc/arm-none-eabi/10.3.0/../../../../arm-none-eabi/lib/thumb\libc.a(lib_a-locale.o)
                              c:/users/tomas/appdata/local/arduino15/packages/rp2040/tools/pqt-gcc/1.4.0-c-0196c06/bin/../lib/gcc/arm-none-eabi/10.3.0/../../../../arm-none-eabi/lib/thumb\libc.a(lib_a-strtod.o) (__global_locale)
c:/users/tomas/appdata/local/arduino15/packages/rp2040/tools/pqt-gcc/1.4.0-c-0196c06/bin/../lib/gcc/arm-none-eabi/10.3.0/../../../../arm-none-eabi/lib/thumb\libc.a(lib_a-localeconv.o)
                              c:/users/tomas/appdata/local/arduino15/packages/rp2040/tools/pqt-gcc/1.4.0-c-0196c06/bin/../lib/gcc/arm-none-eabi/10.3.0/../../../../arm-none-eabi/lib/thumb\libc.a(lib_a-nano-vfprintf_float.o) (_localeconv_r)
c:/users/tomas/appdata/local/arduino15/packages/rp2040/tools/pqt-gcc/1.4.0-c-0196c06/bin/../lib/gcc/arm-none-eabi/10.3.0/../../../../arm-none-eabi/lib/thumb\libc.a(lib_a-lseekr.o)
                              c:/users/tomas/appdata/local/arduino15/packages/rp2040/tools/pqt-gcc/1.4.0-c-0196c06/bin/../lib/gcc/arm-none-eabi/10.3.0/../../../../arm-none-eabi/lib/thumb\libc.a(lib_a-stdio.o) (_lseek_r)
c:/users/tomas/appdata/local/arduino15/packages/rp2040/tools/pqt-gcc/1.4.0-c-0196c06/bin/../lib/gcc/arm-none-eabi/10.3.0/../../../../arm-none-eabi/lib/thumb\libc.a(lib_a-mbtowc_r.o)
                              c:/users/tomas/appdata/local/arduino15/packages/rp2040/tools/pqt-gcc/1.4.0-c-0196c06/bin/../lib/gcc/arm-none-eabi/10.3.0/../../../../arm-none-eabi/lib/thumb\libc.a(lib_a-locale.o) (__ascii_mbtowc)
c:/users/tomas/appdata/local/arduino15/packages/rp2040/tools/pqt-gcc/1.4.0-c-0196c06/bin/../lib/gcc/arm-none-eabi/10.3.0/../../../../arm-none-eabi/lib/thumb\libc.a(lib_a-mprec.o)
                              c:/users/tomas/appdata/local/arduino15/packages/rp2040/tools/pqt-gcc/1.4.0-c-0196c06/bin/../lib/gcc/arm-none-eabi/10.3.0/../../../../arm-none-eabi/lib/thumb\libc.a(lib_a-strtod.o) (_Balloc)
c:/users/tomas/appdata/local/arduino15/packages/rp2040/tools/pqt-gcc/1.4.0-c-0196c06/bin/../lib/gcc/arm-none-eabi/10.3.0/../../../../arm-none-eabi/lib/thumb\libc.a(lib_a-nano-svfprintf.o)
                              c:/users/tomas/appdata/local/arduino15/packages/rp2040/tools/pqt-gcc/1.4.0-c-0196c06/bin/../lib/gcc/arm-none-eabi/10.3.0/../../../../arm-none-eabi/lib/thumb\libc.a(lib_a-sprintf.o) (_svfprintf_r)
c:/users/tomas/appdata/local/arduino15/packages/rp2040/tools/pqt-gcc/1.4.0-c-0196c06/bin/../lib/gcc/arm-none-eabi/10.3.0/../../../../arm-none-eabi/lib/thumb\libc.a(lib_a-nano-vfprintf.o)
                              c:/users/tomas/appdata/local/arduino15/packages/rp2040/tools/pqt-gcc/1.4.0-c-0196c06/bin/../lib/gcc/arm-none-eabi/10.3.0/../../../../arm-none-eabi/lib/thumb\libc.a(lib_a-printf.o) (_vfprintf_r)
c:/users/tomas/appdata/local/arduino15/packages/rp2040/tools/pqt-gcc/1.4.0-c-0196c06/bin/../lib/gcc/arm-none-eabi/10.3.0/../../../../arm-none-eabi/lib/thumb\libc.a(lib_a-putc.o)
                              c:/users/tomas/appdata/local/arduino15/packages/rp2040/tools/pqt-gcc/1.4.0-c-0196c06/bin/../lib/gcc/arm-none-eabi/10.3.0/../../../../arm-none-eabi/lib/thumb\libc.a(lib_a-putchar.o) (_putc_r)
c:/users/tomas/appdata/local/arduino15/packages/rp2040/tools/pqt-gcc/1.4.0-c-0196c06/bin/../lib/gcc/arm-none-eabi/10.3.0/../../../../arm-none-eabi/lib/thumb\libc.a(lib_a-readr.o)
                              c:/users/tomas/appdata/local/arduino15/packages/rp2040/tools/pqt-gcc/1.4.0-c-0196c06/bin/../lib/gcc/arm-none-eabi/10.3.0/../../../../arm-none-eabi/lib/thumb\libc.a(lib_a-stdio.o) (_read_r)
c:/users/tomas/appdata/local/arduino15/packages/rp2040/tools/pqt-gcc/1.4.0-c-0196c06/bin/../lib/gcc/arm-none-eabi/10.3.0/../../../../arm-none-eabi/lib/thumb\libc.a(lib_a-reent.o)
                              c:/users/tomas/appdata/local/arduino15/packages/rp2040/tools/pqt-gcc/1.4.0-c-0196c06/bin/../lib/gcc/arm-none-eabi/10.3.0/../../../../arm-none-eabi/lib/thumb\libc.a(lib_a-sbrkr.o) (errno)
c:/users/tomas/appdata/local/arduino15/packages/rp2040/tools/pqt-gcc/1.4.0-c-0196c06/bin/../lib/gcc/arm-none-eabi/10.3.0/../../../../arm-none-eabi/lib/thumb\libc.a(lib_a-s_nan.o)
                              c:/users/tomas/appdata/local/arduino15/packages/rp2040/tools/pqt-gcc/1.4.0-c-0196c06/bin/../lib/gcc/arm-none-eabi/10.3.0/../../../../arm-none-eabi/lib/thumb\libc.a(lib_a-strtod.o) (nan)
c:/users/tomas/appdata/local/arduino15/packages/rp2040/tools/pqt-gcc/1.4.0-c-0196c06/bin/../lib/gcc/arm-none-eabi/10.3.0/../../../../arm-none-eabi/lib/thumb\libc.a(lib_a-wbuf.o)
                              c:/users/tomas/appdata/local/arduino15/packages/rp2040/tools/pqt-gcc/1.4.0-c-0196c06/bin/../lib/gcc/arm-none-eabi/10.3.0/../../../../arm-none-eabi/lib/thumb\libc.a(lib_a-nano-vfprintf.o) (__swbuf_r)
c:/users/tomas/appdata/local/arduino15/packages/rp2040/tools/pqt-gcc/1.4.0-c-0196c06/bin/../lib/gcc/arm-none-eabi/10.3.0/../../../../arm-none-eabi/lib/thumb\libc.a(lib_a-wctomb_r.o)
                              c:/users/tomas/appdata/local/arduino15/packages/rp2040/tools/pqt-gcc/1.4.0-c-0196c06/bin/../lib/gcc/arm-none-eabi/10.3.0/../../../../arm-none-eabi/lib/thumb\libc.a(lib_a-locale.o) (__ascii_wctomb)
c:/users/tomas/appdata/local/arduino15/packages/rp2040/tools/pqt-gcc/1.4.0-c-0196c06/bin/../lib/gcc/arm-none-eabi/10.3.0/../../../../arm-none-eabi/lib/thumb\libc.a(lib_a-wsetup.o)
                              c:/users/tomas/appdata/local/arduino15/packages/rp2040/tools/pqt-gcc/1.4.0-c-0196c06/bin/../lib/gcc/arm-none-eabi/10.3.0/../../../../arm-none-eabi/lib/thumb\libc.a(lib_a-fvwrite.o) (__swsetup_r)
c:/users/tomas/appdata/local/arduino15/packages/rp2040/tools/pqt-gcc/1.4.0-c-0196c06/bin/../lib/gcc/arm-none-eabi/10.3.0/../../../../arm-none-eabi/lib/thumb\libc.a(lib_a-fputwc.o)
                              c:/users/tomas/appdata/local/arduino15/packages/rp2040/tools/pqt-gcc/1.4.0-c-0196c06/bin/../lib/gcc/arm-none-eabi/10.3.0/../../../../arm-none-eabi/lib/thumb\libc.a(lib_a-nano-vfprintf.o) (_fputwc_r)
c:/users/tomas/appdata/local/arduino15/packages/rp2040/tools/pqt-gcc/1.4.0-c-0196c06/bin/../lib/gcc/arm-none-eabi/10.3.0/../../../../arm-none-eabi/lib/thumb\libc.a(lib_a-makebuf.o)
                              c:/users/tomas/appdata/local/arduino15/packages/rp2040/tools/pqt-gcc/1.4.0-c-0196c06/bin/../lib/gcc/arm-none-eabi/10.3.0/../../../../arm-none-eabi/lib/thumb\libc.a(lib_a-wsetup.o) (__smakebuf_r)
c:/users/tomas/appdata/local/arduino15/packages/rp2040/tools/pqt-gcc/1.4.0-c-0196c06/bin/../lib/gcc/arm-none-eabi/10.3.0/../../../../arm-none-eabi/lib/thumb\libc.a(lib_a-wcrtomb.o)
                              c:/users/tomas/appdata/local/arduino15/packages/rp2040/tools/pqt-gcc/1.4.0-c-0196c06/bin/../lib/gcc/arm-none-eabi/10.3.0/../../../../arm-none-eabi/lib/thumb\libc.a(lib_a-fputwc.o) (_wcrtomb_r)
c:/users/tomas/appdata/local/arduino15/packages/rp2040/tools/pqt-gcc/1.4.0-c-0196c06/bin/../lib/gcc/arm-none-eabi/10.3.0/../../../../arm-none-eabi/lib/thumb\libc.a(lib_a-fstatr.o)
                              c:/users/tomas/appdata/local/arduino15/packages/rp2040/tools/pqt-gcc/1.4.0-c-0196c06/bin/../lib/gcc/arm-none-eabi/10.3.0/../../../../arm-none-eabi/lib/thumb\libc.a(lib_a-makebuf.o) (_fstat_r)
c:/users/tomas/appdata/local/arduino15/packages/rp2040/tools/pqt-gcc/1.4.0-c-0196c06/bin/../lib/gcc/arm-none-eabi/10.3.0/../../../../arm-none-eabi/lib/thumb\libc.a(lib_a-isattyr.o)
                              c:/users/tomas/appdata/local/arduino15/packages/rp2040/tools/pqt-gcc/1.4.0-c-0196c06/bin/../lib/gcc/arm-none-eabi/10.3.0/../../../../arm-none-eabi/lib/thumb\libc.a(lib_a-makebuf.o) (_isatty_r)
C:\Users\tomas\AppData\Local\Temp\arduino-sketch-3D6AC107FF947055EEB72537F7027E49/..\arduino-core-cache\core_47e1560ce04abac12f346abb2f6d40c8.a(lock.cpp.o)
                              c:/users/tomas/appdata/local/arduino15/packages/rp2040/tools/pqt-gcc/1.4.0-c-0196c06/bin/../lib/gcc/arm-none-eabi/10.3.0/../../../../arm-none-eabi/lib/thumb\libc.a(lib_a-findfp.o) (__retarget_lock_init_recursive)
C:\Users\tomas\AppData\Local\Temp\arduino-sketch-3D6AC107FF947055EEB72537F7027E49/..\arduino-core-cache\core_47e1560ce04abac12f346abb2f6d40c8.a(posix.cpp.o)
                              c:/users/tomas/appdata/local/arduino15/packages/rp2040/tools/pqt-gcc/1.4.0-c-0196c06/bin/../lib/gcc/arm-none-eabi/10.3.0/../../../../arm-none-eabi/lib/thumb\libc.a(lib_a-writer.o) (_write)
c:/users/tomas/appdata/local/arduino15/packages/rp2040/tools/pqt-gcc/1.4.0-c-0196c06/bin/../lib/gcc/arm-none-eabi/10.3.0/thumb\libgcc.a(_thumb1_case_uqi.o)
                              C:\Users\tomas\AppData\Local\Temp\arduino-sketch-3D6AC107FF947055EEB72537F7027E49\sketch\skinImpedance.ino.cpp.o (__gnu_thumb1_case_uqi)
c:/users/tomas/appdata/local/arduino15/packages/rp2040/tools/pqt-gcc/1.4.0-c-0196c06/bin/../lib/gcc/arm-none-eabi/10.3.0/thumb\libgcc.a(_thumb1_case_shi.o)
                              C:\Users\tomas\AppData\Local\Arduino15\packages\rp2040\hardware\rp2040\2.6.0/lib/libpico.a(usbd.c.obj) (__gnu_thumb1_case_shi)
c:/users/tomas/appdata/local/arduino15/packages/rp2040/tools/pqt-gcc/1.4.0-c-0196c06/bin/../lib/gcc/arm-none-eabi/10.3.0/thumb\libgcc.a(_thumb1_case_uhi.o)
                              C:\Users\tomas\AppData\Local\Arduino15\packages\rp2040\hardware\rp2040\2.6.0/lib/libpico.a(usbd.c.obj) (__gnu_thumb1_case_uhi)
c:/users/tomas/appdata/local/arduino15/packages/rp2040/tools/pqt-gcc/1.4.0-c-0196c06/bin/../lib/gcc/arm-none-eabi/10.3.0/thumb\libgcc.a(_dvmd_tls.o)
                              C:\Users\tomas\AppData\Local\Arduino15\packages\rp2040\hardware\rp2040\2.6.0/lib/libpico.a(divider.S.obj) (__aeabi_idiv0)
c:/users/tomas/appdata/local/arduino15/packages/rp2040/tools/pqt-gcc/1.4.0-c-0196c06/bin/../lib/gcc/arm-none-eabi/10.3.0/thumb\libgcc.a(_lshrdi3.o)
                              C:\Users\tomas\AppData\Local\Temp\arduino-sketch-3D6AC107FF947055EEB72537F7027E49\libraries\SdFat\ExFatLib\ExFatFile.cpp.o (__aeabi_llsr)
c:/users/tomas/appdata/local/arduino15/packages/rp2040/tools/pqt-gcc/1.4.0-c-0196c06/bin/../lib/gcc/arm-none-eabi/10.3.0/thumb\libgcc.a(_ashldi3.o)
                              C:\Users\tomas\AppData\Local\Arduino15\packages\rp2040\hardware\rp2040\2.6.0/lib/libpico.a(double_math.c.obj) (__aeabi_llsl)

Discarded input sections

 .text          0x0000000000000000        0x0 c:/users/tomas/appdata/local/arduino15/packages/rp2040/tools/pqt-gcc/1.4.0-c-0196c06/bin/../lib/gcc/arm-none-eabi/10.3.0/thumb/crti.o
 .data          0x0000000000000000        0x0 c:/users/tomas/appdata/local/arduino15/packages/rp2040/tools/pqt-gcc/1.4.0-c-0196c06/bin/../lib/gcc/arm-none-eabi/10.3.0/thumb/crti.o
 .bss           0x0000000000000000        0x0 c:/users/tomas/appdata/local/arduino15/packages/rp2040/tools/pqt-gcc/1.4.0-c-0196c06/bin/../lib/gcc/arm-none-eabi/10.3.0/thumb/crti.o
 .data          0x0000000000000000        0x0 c:/users/tomas/appdata/local/arduino15/packages/rp2040/tools/pqt-gcc/1.4.0-c-0196c06/bin/../lib/gcc/arm-none-eabi/10.3.0/thumb/crtbegin.o
 .rodata        0x0000000000000000       0x24 c:/users/tomas/appdata/local/arduino15/packages/rp2040/tools/pqt-gcc/1.4.0-c-0196c06/bin/../lib/gcc/arm-none-eabi/10.3.0/thumb/crtbegin.o
 .fini_array    0x0000000000000000        0x4 c:/users/tomas/appdata/local/arduino15/packages/rp2040/tools/pqt-gcc/1.4.0-c-0196c06/bin/../lib/gcc/arm-none-eabi/10.3.0/thumb/crtbegin.o
 .text          0x0000000000000000       0x74 c:/users/tomas/appdata/local/arduino15/packages/rp2040/tools/pqt-gcc/1.4.0-c-0196c06/bin/../lib/gcc/arm-none-eabi/10.3.0/../../../../arm-none-eabi/lib/thumb/crt0.o
 .data          0x0000000000000000        0x0 c:/users/tomas/appdata/local/arduino15/packages/rp2040/tools/pqt-gcc/1.4.0-c-0196c06/bin/../lib/gcc/arm-none-eabi/10.3.0/../../../../arm-none-eabi/lib/thumb/crt0.o
 .bss           0x0000000000000000        0x0 c:/users/tomas/appdata/local/arduino15/packages/rp2040/tools/pqt-gcc/1.4.0-c-0196c06/bin/../lib/gcc/arm-none-eabi/10.3.0/../../../../arm-none-eabi/lib/thumb/crt0.o
 .ARM.extab     0x0000000000000000        0x0 c:/users/tomas/appdata/local/arduino15/packages/rp2040/tools/pqt-gcc/1.4.0-c-0196c06/bin/../lib/gcc/arm-none-eabi/10.3.0/../../../../arm-none-eabi/lib/thumb/crt0.o
 .ARM.exidx     0x0000000000000000       0x10 c:/users/tomas/appdata/local/arduino15/packages/rp2040/tools/pqt-gcc/1.4.0-c-0196c06/bin/../lib/gcc/arm-none-eabi/10.3.0/../../../../arm-none-eabi/lib/thumb/crt0.o
 .debug_line    0x0000000000000000       0x89 c:/users/tomas/appdata/local/arduino15/packages/rp2040/tools/pqt-gcc/1.4.0-c-0196c06/bin/../lib/gcc/arm-none-eabi/10.3.0/../../../../arm-none-eabi/lib/thumb/crt0.o
 .debug_info    0x0000000000000000       0x26 c:/users/tomas/appdata/local/arduino15/packages/rp2040/tools/pqt-gcc/1.4.0-c-0196c06/bin/../lib/gcc/arm-none-eabi/10.3.0/../../../../arm-none-eabi/lib/thumb/crt0.o
 .debug_abbrev  0x0000000000000000       0x14 c:/users/tomas/appdata/local/arduino15/packages/rp2040/tools/pqt-gcc/1.4.0-c-0196c06/bin/../lib/gcc/arm-none-eabi/10.3.0/../../../../arm-none-eabi/lib/thumb/crt0.o
 .debug_aranges
                0x0000000000000000       0x20 c:/users/tomas/appdata/local/arduino15/packages/rp2040/tools/pqt-gcc/1.4.0-c-0196c06/bin/../lib/gcc/arm-none-eabi/10.3.0/../../../../arm-none-eabi/lib/thumb/crt0.o
 .debug_str     0x0000000000000000       0x7b c:/users/tomas/appdata/local/arduino15/packages/rp2040/tools/pqt-gcc/1.4.0-c-0196c06/bin/../lib/gcc/arm-none-eabi/10.3.0/../../../../arm-none-eabi/lib/thumb/crt0.o
 .ARM.attributes
Memory Configuration

Name             Origin             Length             Attributes
FLASH            0x0000000010000000 0x00000000001ff000 xr
RAM              0x0000000020000000 0x0000000000040000 xrw
SCRATCH_X        0x0000000020040000 0x0000000000001000 xrw
SCRATCH_Y        0x0000000020041000 0x0000000000001000 xrw
*default*        0x0000000000000000 0xffffffffffffffff

Linker script and memory map

LOAD c:/users/tomas/appdata/local/arduino15/packages/rp2040/tools/pqt-gcc/1.4.0-c-0196c06/bin/../lib/gcc/arm-none-eabi/10.3.0/thumb/crti.o
LOAD c:/users/tomas/appdata/local/arduino15/packages/rp2040/tools/pqt-gcc/1.4.0-c-0196c06/bin/../lib/gcc/arm-none-eabi/10.3.0/thumb/crtbegin.o
LOAD c:/users/tomas/appdata/local/arduino15/packages/rp2040/tools/pqt-gcc/1.4.0-c-0196c06/bin/../lib/gcc/arm-none-eabi/10.3.0/../../../../arm-none-eabi/lib/thumb/crt0.o
                [!provide]                        PROVIDE (_EEPROM_start = 0x101ff000)
                [!provide]                        PROVIDE (_FS_start = 0x101ff000)
                [!provide]                        PROVIDE (_FS_end = 0x101ff000)

.flash_begin    0x0000000010000000        0x0
                0x0000000010000000                __flash_binary_start = .

.boot2          0x0000000010000000      0x100
                0x0000000010000000                __boot2_start__ = .
 *(.boot2)
 .boot2         0x0000000010000000      0x100 C:\Users\tomas\AppData\Local\Temp\arduino-sketch-3D6AC107FF947055EEB72537F7027E49/boot2.o
                0x0000000010000100                __boot2_end__ = .
                0x0000000000000001                ASSERT (((__boot2_end__ - __boot2_start__) == 0x100), ERROR: Pico second stage bootloader must be 256 bytes in size)

.ota            0x0000000010000100     0x25e8
 *(.OTA)
 .OTA           0x0000000010000100     0x25e8 C:\Users\tomas\AppData\Local\Arduino15\packages\rp2040\hardware\rp2040\2.6.0/lib/ota.o
                0x0000000010000100                _binary_ota_bin_start
                0x00000000100026e8                _binary_ota_bin_end

.partition      0x00000000100026e8      0x918
                0x0000000010002ff0                . = (__flash_binary_start + 0x2ff0)
 *fill*         0x00000000100026e8      0x908 
                0x0000000010002ff0        0x4 LONG 0x101ff000
                0x0000000010002ff4        0x4 LONG 0x101ff000
                0x0000000010002ff8        0x4 LONG 0x101ff000
                0x0000000010002ffc        0x4 LONG 0x1ff000

.text           0x0000000010003000    0x116a8
                0x0000000010003000                __logical_binary_start = .
 *(.vectors)
 .vectors       0x0000000010003000       0xd4 C:\Users\tomas\AppData\Local\Arduino15\packages\rp2040\hardware\rp2040\2.6.0/lib/libpico.a(crt0.S.obj)
                0x0000000010003000                __VECTOR_TABLE
                0x0000000010003000                __vectors
                0x00000000100030c0                isr_invalid
                0x00000000100030c0                __default_isrs_start
                0x00000000100030c2                isr_nmi
                0x00000000100030c4                isr_hardfault
                0x00000000100030c6                isr_svcall
                0x00000000100030c8                isr_pendsv
                0x00000000100030ca                isr_systick
                0x00000000100030cc                isr_irq23
                0x00000000100030cc                isr_irq18
                0x00000000100030cc                isr_irq11
                0x00000000100030cc                isr_irq28
                0x00000000100030cc                isr_irq19
                0x00000000100030cc                isr_irq0
                0x00000000100030cc                isr_irq6
                0x00000000100030cc                isr_irq5
                0x00000000100030cc                isr_irq12
                0x00000000100030cc                isr_irq22
                0x00000000100030cc                isr_irq31
                0x00000000100030cc                isr_irq17
                0x00000000100030cc                isr_irq27
                0x00000000100030cc                isr_irq30
                0x00000000100030cc                isr_irq2
                0x00000000100030cc                isr_irq10
                0x00000000100030cc                isr_irq8
                0x00000000100030cc                isr_irq24
                0x00000000100030cc                isr_irq1
                0x00000000100030cc                isr_irq7
                0x00000000100030cc                isr_irq21
                0x00000000100030cc                isr_irq20
                0x00000000100030cc                isr_irq15
                0x00000000100030cc                isr_irq25
                0x00000000100030cc                isr_irq13
                0x00000000100030cc                __unhandled_user_irq
                0x00000000100030cc                isr_irq4
                0x00000000100030cc                isr_irq16
                0x00000000100030cc                isr_irq29
                0x00000000100030cc                isr_irq26
                0x00000000100030cc                __default_isrs_end
                0x00000000100030cc                isr_irq3
                0x00000000100030cc                isr_irq14
                0x00000000100030cc                isr_irq9
                0x00000000100030d2                unhandled_user_irq_num_in_r0
 *(.binary_info_header)
 .binary_info_header
                0x00000000100030d4        0x0 C:\Users\tomas\AppData\Local\Arduino15\packages\rp2040\hardware\rp2040\2.6.0/lib/libpico.a(crt0.S.obj)
                0x00000000100030d4                __binary_info_header_end = .
 *(.reset)
 .reset         0x00000000100030d4       0xa8 C:\Users\tomas\AppData\Local\Arduino15\packages\rp2040\hardware\rp2040\2.6.0/lib/libpico.a(crt0.S.obj)
                0x00000000100030d4                _entry_point
                0x0000000010003152                __get_current_exception
 *(.init)
 .init          0x000000001000317c        0x4 c:/users/tomas/appdata/local/arduino15/packages/rp2040/tools/pqt-gcc/1.4.0-c-0196c06/bin/../lib/gcc/arm-none-eabi/10.3.0/thumb/crti.o
                0x000000001000317c                _init
 *(EXCLUDE_FILE(*libm.a: *libc.a:*lib_a-mem*.o *libgcc.a:) .text*)
 .text          0x0000000010003180       0x98 c:/users/tomas/appdata/local/arduino15/packages/rp2040/tools/pqt-gcc/1.4.0-c-0196c06/bin/../lib/gcc/arm-none-eabi/10.3.0/thumb/crtbegin.o
 .text._ZN7arduino5Print17availableForWriteEv
                0x0000000010003218        0x4 C:\Users\tomas\AppData\Local\Temp\arduino-sketch-3D6AC107FF947055EEB72537F7027E49\sketch\skinImpedance.ino.cpp.o
                0x0000000010003218                _ZN7arduino5Print17availableForWriteEv
 .text.pwm_set_gpio_level
                0x000000001000321c       0x3c C:\Users\tomas\AppData\Local\Temp\arduino-sketch-3D6AC107FF947055EEB72537F7027E49\sketch\skinImpedance.ino.cpp.o
 .text._ZN14SdSpiBaseClass3endEv
                0x0000000010003258        0x2 C:\Users\tomas\AppData\Local\Temp\arduino-sketch-3D6AC107FF947055EEB72537F7027E49\sketch\skinImpedance.ino.cpp.o
                0x0000000010003258                _ZN14SdSpiBaseClass3endEv
 *fill*         0x000000001000325a        0x2 
 .text._ZN10MySpiClass11setSckSpeedEm
                0x000000001000325c       0x10 C:\Users\tomas\AppData\Local\Temp\arduino-sketch-3D6AC107FF947055EEB72537F7027E49\sketch\skinImpedance.ino.cpp.o
                0x000000001000325c                _ZN10MySpiClass11setSckSpeedEm
 .text._ZN10MySpiClass4sendEPKhj
                0x000000001000326c       0x10 C:\Users\tomas\AppData\Local\Temp\arduino-sketch-3D6AC107FF947055EEB72537F7027E49\sketch\skinImpedance.ino.cpp.o
                0x000000001000326c                _ZN10MySpiClass4sendEPKhj
 .text._ZN10MySpiClass4sendEh
                0x000000001000327c       0x18 C:\Users\tomas\AppData\Local\Temp\arduino-sketch-3D6AC107FF947055EEB72537F7027E49\sketch\skinImpedance.ino.cpp.o
                0x000000001000327c                _ZN10MySpiClass4sendEh
 .text._ZN10MySpiClass7receiveEPhj
                0x0000000010003294       0x18 C:\Users\tomas\AppData\Local\Temp\arduino-sketch-3D6AC107FF947055EEB72537F7027E49\sketch\skinImpedance.ino.cpp.o
                0x0000000010003294                _ZN10MySpiClass7receiveEPhj
 .text._ZN10MySpiClass7receiveEv
                0x00000000100032ac       0x1c C:\Users\tomas\AppData\Local\Temp\arduino-sketch-3D6AC107FF947055EEB72537F7027E49\sketch\skinImpedance.ino.cpp.o
                0x00000000100032ac                _ZN10MySpiClass7receiveEv
 .text._ZN10MySpiClass10deactivateEv
                0x00000000100032c8       0x10 C:\Users\tomas\AppData\Local\Temp\arduino-sketch-3D6AC107FF947055EEB72537F7027E49\sketch\skinImpedance.ino.cpp.o
                0x00000000100032c8                _ZN10MySpiClass10deactivateEv
 .text._ZN10MySpiClass5beginE11SdSpiConfig
                0x00000000100032d8       0x50 C:\Users\tomas\AppData\Local\Temp\arduino-sketch-3D6AC107FF947055EEB72537F7027E49\sketch\skinImpedance.ino.cpp.o
                0x00000000100032d8                _ZN10MySpiClass5beginE11SdSpiConfig
 .text._ZN10MySpiClass8activateEv
                0x0000000010003328       0x4c C:\Users\tomas\AppData\Local\Temp\arduino-sketch-3D6AC107FF947055EEB72537F7027E49\sketch\skinImpedance.ino.cpp.o
                0x0000000010003328                _ZN10MySpiClass8activateEv
 .text._ZN10StreamFileI10FsBaseFileyE5flushEv
                0x0000000010003374       0x1c C:\Users\tomas\AppData\Local\Temp\arduino-sketch-3D6AC107FF947055EEB72537F7027E49\sketch\skinImpedance.ino.cpp.o
                0x0000000010003374                _ZN10StreamFileI10FsBaseFileyE5flushEv
 .text._ZN10StreamFileI10FsBaseFileyE4peekEv
                0x0000000010003390       0x22 C:\Users\tomas\AppData\Local\Temp\arduino-sketch-3D6AC107FF947055EEB72537F7027E49\sketch\skinImpedance.ino.cpp.o
                0x0000000010003390                _ZN10StreamFileI10FsBaseFileyE4peekEv
 *fill*         0x00000000100033b2        0x2 
 .text._ZN10StreamFileI10FsBaseFileyE9availableEv
                0x00000000100033b4       0x50 C:\Users\tomas\AppData\Local\Temp\arduino-sketch-3D6AC107FF947055EEB72537F7027E49\sketch\skinImpedance.ino.cpp.o
                0x00000000100033b4                _ZN10StreamFileI10FsBaseFileyE9availableEv
 .text._ZN10FsBaseFile4readEPvj
                0x0000000010003404       0x22 C:\Users\tomas\AppData\Local\Temp\arduino-sketch-3D6AC107FF947055EEB72537F7027E49\sketch\skinImpedance.ino.cpp.o
                0x0000000010003404                _ZN10FsBaseFile4readEPvj
 .text._ZN10StreamFileI10FsBaseFileyE4readEv
                0x0000000010003426       0x1e C:\Users\tomas\AppData\Local\Temp\arduino-sketch-3D6AC107FF947055EEB72537F7027E49\sketch\skinImpedance.ino.cpp.o
                0x0000000010003426                _ZN10StreamFileI10FsBaseFileyE4readEv
 .text._ZN10FsBaseFile5writeEPKvj
                0x0000000010003444       0x1e C:\Users\tomas\AppData\Local\Temp\arduino-sketch-3D6AC107FF947055EEB72537F7027E49\sketch\skinImpedance.ino.cpp.o
                0x0000000010003444                _ZN10FsBaseFile5writeEPKvj
 .text._ZN10StreamFileI10FsBaseFileyE5writeEPKhj
                0x0000000010003462        0xa C:\Users\tomas\AppData\Local\Temp\arduino-sketch-3D6AC107FF947055EEB72537F7027E49\sketch\skinImpedance.ino.cpp.o
                0x0000000010003462                _ZN10StreamFileI10FsBaseFileyE5writeEPKhj
 .text._ZN10StreamFileI10FsBaseFileyE5writeEh
                0x000000001000346c       0x14 C:\Users\tomas\AppData\Local\Temp\arduino-sketch-3D6AC107FF947055EEB72537F7027E49\sketch\skinImpedance.ino.cpp.o
                0x000000001000346c                _ZN10StreamFileI10FsBaseFileyE5writeEh
 .text._ZN10FsBaseFile5writeEPKc.isra.0
                0x0000000010003480       0x18 C:\Users\tomas\AppData\Local\Temp\arduino-sketch-3D6AC107FF947055EEB72537F7027E49\sketch\skinImpedance.ino.cpp.o
 .text._ZN11ArduinoJson8V6213PB26detail14CollectionData7addSlotEPNS1_10MemoryPoolE
                0x0000000010003498       0x36 C:\Users\tomas\AppData\Local\Temp\arduino-sketch-3D6AC107FF947055EEB72537F7027E49\sketch\skinImpedance.ino.cpp.o
                0x0000000010003498                _ZN11ArduinoJson8V6213PB26detail14CollectionData7addSlotEPNS1_10MemoryPoolE
 *fill*         0x00000000100034ce        0x2 
 .text._ZN11ArduinoJson8V6213PB26detail11parseNumberEPKcRNS1_11VariantDataE
                0x00000000100034d0      0x25c C:\Users\tomas\AppData\Local\Temp\arduino-sketch-3D6AC107FF947055EEB72537F7027E49\sketch\skinImpedance.ino.cpp.o
                0x00000000100034d0                _ZN11ArduinoJson8V6213PB26detail11parseNumberEPKcRNS1_11VariantDataE
 .text._Z6setup1v
                0x000000001000372c       0x28 C:\Users\tomas\AppData\Local\Temp\arduino-sketch-3D6AC107FF947055EEB72537F7027E49\sketch\skinImpedance.ino.cpp.o
                0x000000001000372c                _Z6setup1v
 .text._Z5loop1v
                0x0000000010003754      0x1ec C:\Users\tomas\AppData\Local\Temp\arduino-sketch-3D6AC107FF947055EEB72537F7027E49\sketch\skinImpedance.ino.cpp.o
                0x0000000010003754                _Z5loop1v
 .text._Z13set_led_colorttt
                0x0000000010003940       0x20 C:\Users\tomas\AppData\Local\Temp\arduino-sketch-3D6AC107FF947055EEB72537F7027E49\sketch\skinImpedance.ino.cpp.o
                0x0000000010003940                _Z13set_led_colorttt
 .text._Z11set_currenth
                0x0000000010003960       0x60 C:\Users\tomas\AppData\Local\Temp\arduino-sketch-3D6AC107FF947055EEB72537F7027E49\sketch\skinImpedance.ino.cpp.o
                0x0000000010003960                _Z11set_currenth
 .text._Z9storeDatam
                0x00000000100039c0      0x10c C:\Users\tomas\AppData\Local\Temp\arduino-sketch-3D6AC107FF947055EEB72537F7027E49\sketch\skinImpedance.ino.cpp.o
                0x00000000100039c0                _Z9storeDatam
 .text._Z9storeRestv
                0x0000000010003acc        0xc C:\Users\tomas\AppData\Local\Temp\arduino-sketch-3D6AC107FF947055EEB72537F7027E49\sketch\skinImpedance.ino.cpp.o
                0x0000000010003acc                _Z9storeRestv
 .text._Z13get_led_colorPt
                0x0000000010003ad8       0x18 C:\Users\tomas\AppData\Local\Temp\arduino-sketch-3D6AC107FF947055EEB72537F7027E49\sketch\skinImpedance.ino.cpp.o
                0x0000000010003ad8                _Z13get_led_colorPt
 .text._ZN6SdBaseI8FsVolume11FsFormatterE5beginE11SdSpiConfig
                0x0000000010003af0       0x50 C:\Users\tomas\AppData\Local\Temp\arduino-sketch-3D6AC107FF947055EEB72537F7027E49\sketch\skinImpedance.ino.cpp.o
                0x0000000010003af0                _ZN6SdBaseI8FsVolume11FsFormatterE5beginE11SdSpiConfig
 .text._ZN11ArduinoJson8V6213PB29ConverterItvE8fromJsonENS0_16JsonVariantConstE
                0x0000000010003b40       0x9c C:\Users\tomas\AppData\Local\Temp\arduino-sketch-3D6AC107FF947055EEB72537F7027E49\sketch\skinImpedance.ino.cpp.o
                0x0000000010003b40                _ZN11ArduinoJson8V6213PB29ConverterItvE8fromJsonENS0_16JsonVariantConstE
 .text._ZNK11ArduinoJson8V6213PB26detail11VariantData10asIntegralIlEET_v
                0x0000000010003bdc       0xa0 C:\Users\tomas\AppData\Local\Temp\arduino-sketch-3D6AC107FF947055EEB72537F7027E49\sketch\skinImpedance.ino.cpp.o
                0x0000000010003bdc                _ZNK11ArduinoJson8V6213PB26detail11VariantData10asIntegralIlEET_v
 .text._ZNK11ArduinoJson8V6213PB26detail11VariantData7asFloatIfEET_v
                0x0000000010003c7c       0x60 C:\Users\tomas\AppData\Local\Temp\arduino-sketch-3D6AC107FF947055EEB72537F7027E49\sketch\skinImpedance.ino.cpp.o
                0x0000000010003c7c                _ZNK11ArduinoJson8V6213PB26detail11VariantData7asFloatIfEET_v
 .text._ZNK11ArduinoJson8V6213PB26detail11VariantData10asIntegralIyEET_v
                0x0000000010003cdc       0x88 C:\Users\tomas\AppData\Local\Temp\arduino-sketch-3D6AC107FF947055EEB72537F7027E49\sketch\skinImpedance.ino.cpp.o
                0x0000000010003cdc                _ZNK11ArduinoJson8V6213PB26detail11VariantData10asIntegralIyEET_v
 .text._ZN11ArduinoJson8V6213PB26detail16JsonDeserializerINS1_6ReaderIPcvEENS1_11StringMoverEE7currentEv
                0x0000000010003d64       0x18 C:\Users\tomas\AppData\Local\Temp\arduino-sketch-3D6AC107FF947055EEB72537F7027E49\sketch\skinImpedance.ino.cpp.o
                0x0000000010003d64                _ZN11ArduinoJson8V6213PB26detail16JsonDeserializerINS1_6ReaderIPcvEENS1_11StringMoverEE7currentEv
 .text._ZN11ArduinoJson8V6213PB26detail16JsonDeserializerINS1_6ReaderIPcvEENS1_11StringMoverEE21skipSpacesAndCommentsEv
                0x0000000010003d7c       0x40 C:\Users\tomas\AppData\Local\Temp\arduino-sketch-3D6AC107FF947055EEB72537F7027E49\sketch\skinImpedance.ino.cpp.o
                0x0000000010003d7c                _ZN11ArduinoJson8V6213PB26detail16JsonDeserializerINS1_6ReaderIPcvEENS1_11StringMoverEE21skipSpacesAndCommentsEv
 .text._ZN11ArduinoJson8V6213PB26detail16JsonDeserializerINS1_6ReaderIPcvEENS1_11StringMoverEE11skipKeywordEPKc
                0x0000000010003dbc       0x2c C:\Users\tomas\AppData\Local\Temp\arduino-sketch-3D6AC107FF947055EEB72537F7027E49\sketch\skinImpedance.ino.cpp.o
                0x0000000010003dbc                _ZN11ArduinoJson8V6213PB26detail16JsonDeserializerINS1_6ReaderIPcvEENS1_11StringMoverEE11skipKeywordEPKc
 .text._ZN11ArduinoJson8V6213PB26detail16JsonDeserializerINS1_6ReaderIPcvEENS1_11StringMoverEE3eatEc
                0x0000000010003de8       0x18 C:\Users\tomas\AppData\Local\Temp\arduino-sketch-3D6AC107FF947055EEB72537F7027E49\sketch\skinImpedance.ino.cpp.o
                0x0000000010003de8                _ZN11ArduinoJson8V6213PB26detail16JsonDeserializerINS1_6ReaderIPcvEENS1_11StringMoverEE3eatEc
 .text._ZNK11ArduinoJson8V6213PB26detail14CollectionData9getMemberINS1_19StaticStringAdapterEEEPNS1_11VariantDataET_
                0x0000000010003e00       0x4a C:\Users\tomas\AppData\Local\Temp\arduino-sketch-3D6AC107FF947055EEB72537F7027E49\sketch\skinImpedance.ino.cpp.o
                0x0000000010003e00                _ZNK11ArduinoJson8V6213PB26detail14CollectionData9getMemberINS1_19StaticStringAdapterEEEPNS1_11VariantDataET_
 *fill*         0x0000000010003e4a        0x2 
 .text._ZN11ArduinoJson8V6213PB26detail16JsonDeserializerINS1_6ReaderIPcvEENS1_11StringMoverEE17parseQuotedStringEv
                0x0000000010003e4c      0x150 C:\Users\tomas\AppData\Local\Temp\arduino-sketch-3D6AC107FF947055EEB72537F7027E49\sketch\skinImpedance.ino.cpp.o
                0x0000000010003e4c                _ZN11ArduinoJson8V6213PB26detail16JsonDeserializerINS1_6ReaderIPcvEENS1_11StringMoverEE17parseQuotedStringEv
 .text._ZN11ArduinoJson8V6213PB26detail16JsonDeserializerINS1_6ReaderIPcvEENS1_11StringMoverEE22canBeInNonQuotedStringEc
                0x0000000010003f9c       0x2a C:\Users\tomas\AppData\Local\Temp\arduino-sketch-3D6AC107FF947055EEB72537F7027E49\sketch\skinImpedance.ino.cpp.o
                0x0000000010003f9c                _ZN11ArduinoJson8V6213PB26detail16JsonDeserializerINS1_6ReaderIPcvEENS1_11StringMoverEE22canBeInNonQuotedStringEc
 *fill*         0x0000000010003fc6        0x2 
 .text._ZN11ArduinoJson8V6213PB26detail16JsonDeserializerINS1_6ReaderIPcvEENS1_11StringMoverEE12parseVariantINS1_14AllowAllFilterEEENS0_20DeserializationError4CodeERNS1_11VariantDataET_NS0_21DeserializationOption12NestingLimitE.isra.0
                0x0000000010003fc8      0x2a0 C:\Users\tomas\AppData\Local\Temp\arduino-sketch-3D6AC107FF947055EEB72537F7027E49\sketch\skinImpedance.ino.cpp.o
 .text._ZNK11ArduinoJson8V6213PB26detail11VariantData9getMemberINS1_19StaticStringAdapterEEEPS2_T_
                0x0000000010004268       0x18 C:\Users\tomas\AppData\Local\Temp\arduino-sketch-3D6AC107FF947055EEB72537F7027E49\sketch\skinImpedance.ino.cpp.o
                0x0000000010004268                _ZNK11ArduinoJson8V6213PB26detail11VariantData9getMemberINS1_19StaticStringAdapterEEEPS2_T_
 .text._Z10readConfigb
                0x0000000010004280      0x2f0 C:\Users\tomas\AppData\Local\Temp\arduino-sketch-3D6AC107FF947055EEB72537F7027E49\sketch\skinImpedance.ino.cpp.o
                0x0000000010004280                _Z10readConfigb
 .text.setup    0x0000000010004570      0x1f8 C:\Users\tomas\AppData\Local\Temp\arduino-sketch-3D6AC107FF947055EEB72537F7027E49\sketch\skinImpedance.ino.cpp.o
                0x0000000010004570                setup
 .text._Z12startStopLogv
                0x0000000010004768      0x320 C:\Users\tomas\AppData\Local\Temp\arduino-sketch-3D6AC107FF947055EEB72537F7027E49\sketch\skinImpedance.ino.cpp.o
                0x0000000010004768                _Z12startStopLogv
 .text.loop     0x0000000010004a88      0x3a8 C:\Users\tomas\AppData\Local\Temp\arduino-sketch-3D6AC107FF947055EEB72537F7027E49\sketch\skinImpedance.ino.cpp.o
                0x0000000010004a88                loop
 .text.startup._GLOBAL__sub_I_mySpi
                0x0000000010004e30       0x98 C:\Users\tomas\AppData\Local\Temp\arduino-sketch-3D6AC107FF947055EEB72537F7027E49\sketch\skinImpedance.ino.cpp.o
 .text._Z7getLe32PKh
                0x0000000010004ec8       0x16 C:\Users\tomas\AppData\Local\Temp\arduino-sketch-3D6AC107FF947055EEB72537F7027E49\libraries\SdFat\ExFatLib\ExFatDbg.cpp.o
                0x0000000010004ec8                _Z7getLe32PKh
 .text._Z7getLe64PKh
                0x0000000010004ede       0x2e C:\Users\tomas\AppData\Local\Temp\arduino-sketch-3D6AC107FF947055EEB72537F7027E49\libraries\SdFat\ExFatLib\ExFatDbg.cpp.o
                0x0000000010004ede                _Z7getLe64PKh
 .text._ZN9ExFatFile8dirCacheEhh
                0x0000000010004f0c       0x38 C:\Users\tomas\AppData\Local\Temp\arduino-sketch-3D6AC107FF947055EEB72537F7027E49\libraries\SdFat\ExFatLib\ExFatFile.cpp.o
                0x0000000010004f0c                _ZN9ExFatFile8dirCacheEhh
 .text._ZN9ExFatFile5closeEv
                0x0000000010004f44       0x16 C:\Users\tomas\AppData\Local\Temp\arduino-sketch-3D6AC107FF947055EEB72537F7027E49\libraries\SdFat\ExFatLib\ExFatFile.cpp.o
                0x0000000010004f44                _ZN9ExFatFile5closeEv
 .text._ZN9ExFatFile8openRootEP11ExFatVolume
                0x0000000010004f5a       0x2a C:\Users\tomas\AppData\Local\Temp\arduino-sketch-3D6AC107FF947055EEB72537F7027E49\libraries\SdFat\ExFatLib\ExFatFile.cpp.o
                0x0000000010004f5a                _ZN9ExFatFile8openRootEP11ExFatVolume
 .text._ZN9ExFatFile13parsePathNameEPKcP8ExName_tPS1_
                0x0000000010004f84       0x80 C:\Users\tomas\AppData\Local\Temp\arduino-sketch-3D6AC107FF947055EEB72537F7027E49\libraries\SdFat\ExFatLib\ExFatFile.cpp.o
                0x0000000010004f84                _ZN9ExFatFile13parsePathNameEPKcP8ExName_tPS1_
 .text._ZN9ExFatFile4readEPvj
                0x0000000010005004      0x1a8 C:\Users\tomas\AppData\Local\Temp\arduino-sketch-3D6AC107FF947055EEB72537F7027E49\libraries\SdFat\ExFatLib\ExFatFile.cpp.o
                0x0000000010005004                _ZN9ExFatFile4readEPvj
 .text._ZN9ExFatFile4peekEv
                0x00000000100051ac       0x32 C:\Users\tomas\AppData\Local\Temp\arduino-sketch-3D6AC107FF947055EEB72537F7027E49\libraries\SdFat\ExFatLib\ExFatFile.cpp.o
                0x00000000100051ac                _ZN9ExFatFile4peekEv
 *fill*         0x00000000100051de        0x2 
 .text._ZN9ExFatFile7seekSetEy
                0x00000000100051e0       0xe4 C:\Users\tomas\AppData\Local\Temp\arduino-sketch-3D6AC107FF947055EEB72537F7027E49\libraries\SdFat\ExFatLib\ExFatFile.cpp.o
                0x00000000100051e0                _ZN9ExFatFile7seekSetEy
 .text._ZN9ExFatFile11openPrivateEPS_P8ExName_ti
                0x00000000100052c4      0x388 C:\Users\tomas\AppData\Local\Temp\arduino-sketch-3D6AC107FF947055EEB72537F7027E49\libraries\SdFat\ExFatLib\ExFatFile.cpp.o
                0x00000000100052c4                _ZN9ExFatFile11openPrivateEPS_P8ExName_ti
 .text._ZN9ExFatFile4openEPS_PKci
                0x000000001000564c       0xb8 C:\Users\tomas\AppData\Local\Temp\arduino-sketch-3D6AC107FF947055EEB72537F7027E49\libraries\SdFat\ExFatLib\ExFatFile.cpp.o
                0x000000001000564c                _ZN9ExFatFile4openEPS_PKci
 .text._ZN9ExFatFile4openEP11ExFatVolumePKci
                0x0000000010005704       0x18 C:\Users\tomas\AppData\Local\Temp\arduino-sketch-3D6AC107FF947055EEB72537F7027E49\libraries\SdFat\ExFatLib\ExFatFile.cpp.o
                0x0000000010005704                _ZN9ExFatFile4openEP11ExFatVolumePKci
 .text._ZL16exFatDirChecksumPKht
                0x000000001000571c       0x2e C:\Users\tomas\AppData\Local\Temp\arduino-sketch-3D6AC107FF947055EEB72537F7027E49\libraries\SdFat\ExFatLib\ExFatFileWrite.cpp.o
 .text._ZN14ExFatPartition9cacheSyncEv
                0x000000001000574a       0x2a C:\Users\tomas\AppData\Local\Temp\arduino-sketch-3D6AC107FF947055EEB72537F7027E49\libraries\SdFat\ExFatLib\ExFatFileWrite.cpp.o
                0x000000001000574a                _ZN14ExFatPartition9cacheSyncEv
 .text._ZN9ExFatFile10addClusterEv
                0x0000000010005774       0x94 C:\Users\tomas\AppData\Local\Temp\arduino-sketch-3D6AC107FF947055EEB72537F7027E49\libraries\SdFat\ExFatLib\ExFatFileWrite.cpp.o
                0x0000000010005774                _ZN9ExFatFile10addClusterEv
 .text._ZN9ExFatFile7syncDirEv
                0x0000000010005808      0x130 C:\Users\tomas\AppData\Local\Temp\arduino-sketch-3D6AC107FF947055EEB72537F7027E49\libraries\SdFat\ExFatLib\ExFatFileWrite.cpp.o
                0x0000000010005808                _ZN9ExFatFile7syncDirEv
 .text._ZN9ExFatFile4syncEv
                0x0000000010005938       0x42 C:\Users\tomas\AppData\Local\Temp\arduino-sketch-3D6AC107FF947055EEB72537F7027E49\libraries\SdFat\ExFatLib\ExFatFileWrite.cpp.o
                0x0000000010005938                _ZN9ExFatFile4syncEv
 *fill*         0x000000001000597a        0x2 
 .text._ZN9ExFatFile13addDirClusterEv
                0x000000001000597c       0xc4 C:\Users\tomas\AppData\Local\Temp\arduino-sketch-3D6AC107FF947055EEB72537F7027E49\libraries\SdFat\ExFatLib\ExFatFileWrite.cpp.o
                0x000000001000597c                _ZN9ExFatFile13addDirClusterEv
 .text._ZN9ExFatFile5mkdirEPS_P8ExName_t
                0x0000000010005a40       0x54 C:\Users\tomas\AppData\Local\Temp\arduino-sketch-3D6AC107FF947055EEB72537F7027E49\libraries\SdFat\ExFatLib\ExFatFileWrite.cpp.o
                0x0000000010005a40                _ZN9ExFatFile5mkdirEPS_P8ExName_t
 .text._ZN9ExFatFile5mkdirEPS_PKcb
                0x0000000010005a94       0xaa C:\Users\tomas\AppData\Local\Temp\arduino-sketch-3D6AC107FF947055EEB72537F7027E49\libraries\SdFat\ExFatLib\ExFatFileWrite.cpp.o
                0x0000000010005a94                _ZN9ExFatFile5mkdirEPS_PKcb
 *fill*         0x0000000010005b3e        0x2 
 .text._ZN9ExFatFile8truncateEv
                0x0000000010005b40       0xd0 C:\Users\tomas\AppData\Local\Temp\arduino-sketch-3D6AC107FF947055EEB72537F7027E49\libraries\SdFat\ExFatLib\ExFatFileWrite.cpp.o
                0x0000000010005b40                _ZN9ExFatFile8truncateEv
 .text._ZN9ExFatFile5writeEPKvj
                0x0000000010005c10      0x244 C:\Users\tomas\AppData\Local\Temp\arduino-sketch-3D6AC107FF947055EEB72537F7027E49\libraries\SdFat\ExFatLib\ExFatFileWrite.cpp.o
                0x0000000010005c10                _ZN9ExFatFile5writeEPKvj
 .text._ZN9ExFatFile7cmpNameEPK9DirName_tP8ExName_t
                0x0000000010005e54       0x54 C:\Users\tomas\AppData\Local\Temp\arduino-sketch-3D6AC107FF947055EEB72537F7027E49\libraries\SdFat\ExFatLib\ExFatName.cpp.o
                0x0000000010005e54                _ZN9ExFatFile7cmpNameEPK9DirName_tP8ExName_t
 .text._ZN9ExFatFile8hashNameEP8ExName_t
                0x0000000010005ea8       0x4a C:\Users\tomas\AppData\Local\Temp\arduino-sketch-3D6AC107FF947055EEB72537F7027E49\libraries\SdFat\ExFatLib\ExFatName.cpp.o
                0x0000000010005ea8                _ZN9ExFatFile8hashNameEP8ExName_t
 *fill*         0x0000000010005ef2        0x2 
 .text._ZN14ExFatPartition10bitmapFindEmm
                0x0000000010005ef4       0xc4 C:\Users\tomas\AppData\Local\Temp\arduino-sketch-3D6AC107FF947055EEB72537F7027E49\libraries\SdFat\ExFatLib\ExFatPartition.cpp.o
                0x0000000010005ef4                _ZN14ExFatPartition10bitmapFindEmm
 .text._ZN14ExFatPartition12bitmapModifyEmmb
                0x0000000010005fb8       0xa8 C:\Users\tomas\AppData\Local\Temp\arduino-sketch-3D6AC107FF947055EEB72537F7027E49\libraries\SdFat\ExFatLib\ExFatPartition.cpp.o
                0x0000000010005fb8                _ZN14ExFatPartition12bitmapModifyEmmb
 .text._ZN14ExFatPartition8dirCacheEP8DirPos_th
                0x0000000010006060       0x44 C:\Users\tomas\AppData\Local\Temp\arduino-sketch-3D6AC107FF947055EEB72537F7027E49\libraries\SdFat\ExFatLib\ExFatPartition.cpp.o
                0x0000000010006060                _ZN14ExFatPartition8dirCacheEP8DirPos_th
 .text._ZN14ExFatPartition6fatGetEmPm
                0x00000000100060a4       0x4c C:\Users\tomas\AppData\Local\Temp\arduino-sketch-3D6AC107FF947055EEB72537F7027E49\libraries\SdFat\ExFatLib\ExFatPartition.cpp.o
                0x00000000100060a4                _ZN14ExFatPartition6fatGetEmPm
 .text._ZN14ExFatPartition9chainSizeEm
                0x00000000100060f0       0x24 C:\Users\tomas\AppData\Local\Temp\arduino-sketch-3D6AC107FF947055EEB72537F7027E49\libraries\SdFat\ExFatLib\ExFatPartition.cpp.o
                0x00000000100060f0                _ZN14ExFatPartition9chainSizeEm
 .text._ZN14ExFatPartition7dirSeekEP8DirPos_tm
                0x0000000010006114       0x4c C:\Users\tomas\AppData\Local\Temp\arduino-sketch-3D6AC107FF947055EEB72537F7027E49\libraries\SdFat\ExFatLib\ExFatPartition.cpp.o
                0x0000000010006114                _ZN14ExFatPartition7dirSeekEP8DirPos_tm
 .text._ZN14ExFatPartition6fatPutEmm
                0x0000000010006160       0x50 C:\Users\tomas\AppData\Local\Temp\arduino-sketch-3D6AC107FF947055EEB72537F7027E49\libraries\SdFat\ExFatLib\ExFatPartition.cpp.o
                0x0000000010006160                _ZN14ExFatPartition6fatPutEmm
 .text._ZN14ExFatPartition9freeChainEm
                0x00000000100061b0       0x5a C:\Users\tomas\AppData\Local\Temp\arduino-sketch-3D6AC107FF947055EEB72537F7027E49\libraries\SdFat\ExFatLib\ExFatPartition.cpp.o
                0x00000000100061b0                _ZN14ExFatPartition9freeChainEm
 *fill*         0x000000001000620a        0x2 
 .text._ZN14ExFatPartition4initEP16DedicatedSpiCardhm
                0x000000001000620c      0x124 C:\Users\tomas\AppData\Local\Temp\arduino-sketch-3D6AC107FF947055EEB72537F7027E49\libraries\SdFat\ExFatLib\ExFatPartition.cpp.o
                0x000000001000620c                _ZN14ExFatPartition4initEP16DedicatedSpiCardhm
 .text._ZN14ExFatPartition10rootLengthEv
                0x0000000010006330       0x20 C:\Users\tomas\AppData\Local\Temp\arduino-sketch-3D6AC107FF947055EEB72537F7027E49\libraries\SdFat\ExFatLib\ExFatPartition.cpp.o
                0x0000000010006330                _ZN14ExFatPartition10rootLengthEv
 .text._ZN7FatFile8openRootEP9FatVolume.part.0
                0x0000000010006350       0x2a C:\Users\tomas\AppData\Local\Temp\arduino-sketch-3D6AC107FF947055EEB72537F7027E49\libraries\SdFat\FatLib\FatFile.cpp.o
 .text._ZN12FatPartition9cacheSyncEv
                0x000000001000637a       0x28 C:\Users\tomas\AppData\Local\Temp\arduino-sketch-3D6AC107FF947055EEB72537F7027E49\libraries\SdFat\FatLib\FatFile.cpp.o
                0x000000001000637a                _ZN12FatPartition9cacheSyncEv
 .text._ZN7FatFile10addClusterEv
                0x00000000100063a2       0x3c C:\Users\tomas\AppData\Local\Temp\arduino-sketch-3D6AC107FF947055EEB72537F7027E49\libraries\SdFat\FatLib\FatFile.cpp.o
                0x00000000100063a2                _ZN7FatFile10addClusterEv
 *fill*         0x00000000100063de        0x2 
 .text._ZN7FatFile13addDirClusterEv
                0x00000000100063e0       0x78 C:\Users\tomas\AppData\Local\Temp\arduino-sketch-3D6AC107FF947055EEB72537F7027E49\libraries\SdFat\FatLib\FatFile.cpp.o
                0x00000000100063e0                _ZN7FatFile13addDirClusterEv
 .text._ZN7FatFile13cacheDirEntryEh
                0x0000000010006458       0x20 C:\Users\tomas\AppData\Local\Temp\arduino-sketch-3D6AC107FF947055EEB72537F7027E49\libraries\SdFat\FatLib\FatFile.cpp.o
                0x0000000010006458                _ZN7FatFile13cacheDirEntryEh
 .text._ZN7FatFile8openRootEP9FatVolume
                0x0000000010006478       0x14 C:\Users\tomas\AppData\Local\Temp\arduino-sketch-3D6AC107FF947055EEB72537F7027E49\libraries\SdFat\FatLib\FatFile.cpp.o
                0x0000000010006478                _ZN7FatFile8openRootEP9FatVolume
 .text._ZN7FatFile4readEPvj
                0x000000001000648c      0x184 C:\Users\tomas\AppData\Local\Temp\arduino-sketch-3D6AC107FF947055EEB72537F7027E49\libraries\SdFat\FatLib\FatFile.cpp.o
                0x000000001000648c                _ZN7FatFile4readEPvj
 .text._ZN7FatFile4peekEv
                0x0000000010006610       0x26 C:\Users\tomas\AppData\Local\Temp\arduino-sketch-3D6AC107FF947055EEB72537F7027E49\libraries\SdFat\FatLib\FatFile.cpp.o
                0x0000000010006610                _ZN7FatFile4peekEv
 .text._ZN7FatFile12readDirCacheEb
                0x0000000010006636       0x3a C:\Users\tomas\AppData\Local\Temp\arduino-sketch-3D6AC107FF947055EEB72537F7027E49\libraries\SdFat\FatLib\FatFile.cpp.o
                0x0000000010006636                _ZN7FatFile12readDirCacheEb
 .text._ZN7FatFile7seekSetEm
                0x0000000010006670       0xa0 C:\Users\tomas\AppData\Local\Temp\arduino-sketch-3D6AC107FF947055EEB72537F7027E49\libraries\SdFat\FatLib\FatFile.cpp.o
                0x0000000010006670                _ZN7FatFile7seekSetEm
 .text._ZN7FatFile15openCachedEntryEPS_tih
                0x0000000010006710       0xf6 C:\Users\tomas\AppData\Local\Temp\arduino-sketch-3D6AC107FF947055EEB72537F7027E49\libraries\SdFat\FatLib\FatFile.cpp.o
                0x0000000010006710                _ZN7FatFile15openCachedEntryEPS_tih
 *fill*         0x0000000010006806        0x2 
 .text._ZN7FatFile4syncEv
                0x0000000010006808       0xa8 C:\Users\tomas\AppData\Local\Temp\arduino-sketch-3D6AC107FF947055EEB72537F7027E49\libraries\SdFat\FatLib\FatFile.cpp.o
                0x0000000010006808                _ZN7FatFile4syncEv
 .text._ZN7FatFile5closeEv
                0x00000000100068b0       0x10 C:\Users\tomas\AppData\Local\Temp\arduino-sketch-3D6AC107FF947055EEB72537F7027E49\libraries\SdFat\FatLib\FatFile.cpp.o
                0x00000000100068b0                _ZN7FatFile5closeEv
 .text._ZN7FatFile4openEPS_PKci
                0x00000000100068c0       0xa4 C:\Users\tomas\AppData\Local\Temp\arduino-sketch-3D6AC107FF947055EEB72537F7027E49\libraries\SdFat\FatLib\FatFile.cpp.o
                0x00000000100068c0                _ZN7FatFile4openEPS_PKci
 .text._ZN7FatFile4openEP9FatVolumePKci
                0x0000000010006964       0x1c C:\Users\tomas\AppData\Local\Temp\arduino-sketch-3D6AC107FF947055EEB72537F7027E49\libraries\SdFat\FatLib\FatFile.cpp.o
                0x0000000010006964                _ZN7FatFile4openEP9FatVolumePKci
 .text._ZN7FatFile5mkdirEPS_P8FatLfn_t
                0x0000000010006980       0xc4 C:\Users\tomas\AppData\Local\Temp\arduino-sketch-3D6AC107FF947055EEB72537F7027E49\libraries\SdFat\FatLib\FatFile.cpp.o
                0x0000000010006980                _ZN7FatFile5mkdirEPS_P8FatLfn_t
 .text._ZN7FatFile5mkdirEPS_PKcb
                0x0000000010006a44       0xaa C:\Users\tomas\AppData\Local\Temp\arduino-sketch-3D6AC107FF947055EEB72537F7027E49\libraries\SdFat\FatLib\FatFile.cpp.o
                0x0000000010006a44                _ZN7FatFile5mkdirEPS_PKcb
 *fill*         0x0000000010006aee        0x2 
 .text._ZN7FatFile5writeEPKvj
                0x0000000010006af0      0x1a4 C:\Users\tomas\AppData\Local\Temp\arduino-sketch-3D6AC107FF947055EEB72537F7027E49\libraries\SdFat\FatLib\FatFile.cpp.o
                0x0000000010006af0                _ZN7FatFile5writeEPKvj
 .text._ZN7FatFile11lfnChecksumEPKh.isra.0
                0x0000000010006c94       0x1c C:\Users\tomas\AppData\Local\Temp\arduino-sketch-3D6AC107FF947055EEB72537F7027E49\libraries\SdFat\FatLib\FatFileLFN.cpp.o
 .text._ZN7FatFile8cacheDirEt
                0x0000000010006cb0       0x1c C:\Users\tomas\AppData\Local\Temp\arduino-sketch-3D6AC107FF947055EEB72537F7027E49\libraries\SdFat\FatLib\FatFileLFN.cpp.o
                0x0000000010006cb0                _ZN7FatFile8cacheDirEt
 .text._ZN7FatFile7cmpNameEtP8FatLfn_th
                0x0000000010006ccc       0x96 C:\Users\tomas\AppData\Local\Temp\arduino-sketch-3D6AC107FF947055EEB72537F7027E49\libraries\SdFat\FatLib\FatFileLFN.cpp.o
                0x0000000010006ccc                _ZN7FatFile7cmpNameEtP8FatLfn_th
 *fill*         0x0000000010006d62        0x2 
 .text._ZN7FatFile9createLFNEtP8FatLfn_th
                0x0000000010006d64       0xc8 C:\Users\tomas\AppData\Local\Temp\arduino-sketch-3D6AC107FF947055EEB72537F7027E49\libraries\SdFat\FatLib\FatFileLFN.cpp.o
                0x0000000010006d64                _ZN7FatFile9createLFNEtP8FatLfn_th
 .text._ZN7FatFile7makeSFNEP8FatLfn_t
                0x0000000010006e2c      0x126 C:\Users\tomas\AppData\Local\Temp\arduino-sketch-3D6AC107FF947055EEB72537F7027E49\libraries\SdFat\FatLib\FatFileLFN.cpp.o
                0x0000000010006e2c                _ZN7FatFile7makeSFNEP8FatLfn_t
 .text._ZN7FatFile13makeUniqueSfnEP8FatLfn_t
                0x0000000010006f52       0x96 C:\Users\tomas\AppData\Local\Temp\arduino-sketch-3D6AC107FF947055EEB72537F7027E49\libraries\SdFat\FatLib\FatFileLFN.cpp.o
                0x0000000010006f52                _ZN7FatFile13makeUniqueSfnEP8FatLfn_t
 .text._ZN7FatFile4openEPS_P8FatLfn_ti
                0x0000000010006fe8      0x274 C:\Users\tomas\AppData\Local\Temp\arduino-sketch-3D6AC107FF947055EEB72537F7027E49\libraries\SdFat\FatLib\FatFileLFN.cpp.o
                0x0000000010006fe8                _ZN7FatFile4openEPS_P8FatLfn_ti
 .text._ZN7FatFile13parsePathNameEPKcP8FatLfn_tPS1_
                0x000000001000725c       0x8c C:\Users\tomas\AppData\Local\Temp\arduino-sketch-3D6AC107FF947055EEB72537F7027E49\libraries\SdFat\FatLib\FatFileLFN.cpp.o
                0x000000001000725c                _ZN7FatFile13parsePathNameEPKcP8FatLfn_tPS1_
 .text._ZN7FatFile10getLfnCharEP8DirLfn_th
                0x00000000100072e8       0x34 C:\Users\tomas\AppData\Local\Temp\arduino-sketch-3D6AC107FF947055EEB72537F7027E49\libraries\SdFat\FatLib\FatName.cpp.o
                0x00000000100072e8                _ZN7FatFile10getLfnCharEP8DirLfn_th
 .text._ZN12FatPartition6fatGetEmPm
                0x000000001000731c       0x7a C:\Users\tomas\AppData\Local\Temp\arduino-sketch-3D6AC107FF947055EEB72537F7027E49\libraries\SdFat\FatLib\FatPartition.cpp.o
                0x000000001000731c                _ZN12FatPartition6fatGetEmPm
 .text._ZN12FatPartition6fatPutEmm
                0x0000000010007396       0x74 C:\Users\tomas\AppData\Local\Temp\arduino-sketch-3D6AC107FF947055EEB72537F7027E49\libraries\SdFat\FatLib\FatPartition.cpp.o
                0x0000000010007396                _ZN12FatPartition6fatPutEmm
 *fill*         0x000000001000740a        0x2 
 .text._ZN12FatPartition15allocateClusterEmPm
                0x000000001000740c       0x7c C:\Users\tomas\AppData\Local\Temp\arduino-sketch-3D6AC107FF947055EEB72537F7027E49\libraries\SdFat\FatLib\FatPartition.cpp.o
                0x000000001000740c                _ZN12FatPartition15allocateClusterEmPm
 .text._ZN12FatPartition9freeChainEm
                0x0000000010007488       0x38 C:\Users\tomas\AppData\Local\Temp\arduino-sketch-3D6AC107FF947055EEB72537F7027E49\libraries\SdFat\FatLib\FatPartition.cpp.o
                0x0000000010007488                _ZN12FatPartition9freeChainEm
 .text._ZN12FatPartition4initEP16DedicatedSpiCardhm
                0x00000000100074c0      0x160 C:\Users\tomas\AppData\Local\Temp\arduino-sketch-3D6AC107FF947055EEB72537F7027E49\libraries\SdFat\FatLib\FatPartition.cpp.o
                0x00000000100074c0                _ZN12FatPartition4initEP16DedicatedSpiCardhm
 .text._ZN10FsBaseFile5closeEv
                0x0000000010007620       0x26 C:\Users\tomas\AppData\Local\Temp\arduino-sketch-3D6AC107FF947055EEB72537F7027E49\libraries\SdFat\FsLib\FsFile.cpp.o
                0x0000000010007620                _ZN10FsBaseFile5closeEv
 .text._ZN10FsBaseFileaSERKS_
                0x0000000010007646       0x5a C:\Users\tomas\AppData\Local\Temp\arduino-sketch-3D6AC107FF947055EEB72537F7027E49\libraries\SdFat\FsLib\FsFile.cpp.o
                0x0000000010007646                _ZN10FsBaseFileaSERKS_
 .text._ZN10FsBaseFile4openEP8FsVolumePKci
                0x00000000100076a0       0x84 C:\Users\tomas\AppData\Local\Temp\arduino-sketch-3D6AC107FF947055EEB72537F7027E49\libraries\SdFat\FsLib\FsFile.cpp.o
                0x00000000100076a0                _ZN10FsBaseFile4openEP8FsVolumePKci
 .text._ZnwjPm  0x0000000010007724        0x4 C:\Users\tomas\AppData\Local\Temp\arduino-sketch-3D6AC107FF947055EEB72537F7027E49\libraries\SdFat\FsLib\FsNew.cpp.o
                0x0000000010007724                _ZnwjPm
 .text._ZN8FsVolume5beginEP16DedicatedSpiCardbhm
                0x0000000010007728      0x11c C:\Users\tomas\AppData\Local\Temp\arduino-sketch-3D6AC107FF947055EEB72537F7027E49\libraries\SdFat\FsLib\FsVolume.cpp.o
                0x0000000010007728                _ZN8FsVolume5beginEP16DedicatedSpiCardbhm
 .text._ZN8FsVolume4openEPKci
                0x0000000010007844       0x28 C:\Users\tomas\AppData\Local\Temp\arduino-sketch-3D6AC107FF947055EEB72537F7027E49\libraries\SdFat\FsLib\FsVolume.cpp.o
                0x0000000010007844                _ZN8FsVolume4openEPKci
 .text._ZN8FsVolume4openERKN7arduino6StringEi
                0x000000001000786c       0x28 C:\Users\tomas\AppData\Local\Temp\arduino-sketch-3D6AC107FF947055EEB72537F7027E49\libraries\SdFat\FsLib\FsVolume.cpp.o
                0x000000001000786c                _ZN8FsVolume4openERKN7arduino6StringEi
 .text._ZN7Timeout8timedOutEv.isra.0
                0x0000000010007894       0x10 C:\Users\tomas\AppData\Local\Temp\arduino-sketch-3D6AC107FF947055EEB72537F7027E49\libraries\SdFat\SdCard\SdSpiCard.cpp.o
 .text._ZN13SharedSpiCard7spiSendEh.isra.0
                0x00000000100078a4        0xa C:\Users\tomas\AppData\Local\Temp\arduino-sketch-3D6AC107FF947055EEB72537F7027E49\libraries\SdFat\SdCard\SdSpiCard.cpp.o
 .text._ZN13SharedSpiCard10spiReceiveEv.isra.0
                0x00000000100078ae        0xa C:\Users\tomas\AppData\Local\Temp\arduino-sketch-3D6AC107FF947055EEB72537F7027E49\libraries\SdFat\SdCard\SdSpiCard.cpp.o
 .text._ZN13SharedSpiCard8spiStartEv
                0x00000000100078b8       0x28 C:\Users\tomas\AppData\Local\Temp\arduino-sketch-3D6AC107FF947055EEB72537F7027E49\libraries\SdFat\SdCard\SdSpiCard.cpp.o
                0x00000000100078b8                _ZN13SharedSpiCard8spiStartEv
 .text._ZN13SharedSpiCard7spiStopEv
                0x00000000100078e0       0x28 C:\Users\tomas\AppData\Local\Temp\arduino-sketch-3D6AC107FF947055EEB72537F7027E49\libraries\SdFat\SdCard\SdSpiCard.cpp.o
                0x00000000100078e0                _ZN13SharedSpiCard7spiStopEv
 .text._ZN13SharedSpiCard8readDataEPhj
                0x0000000010007908       0x62 C:\Users\tomas\AppData\Local\Temp\arduino-sketch-3D6AC107FF947055EEB72537F7027E49\libraries\SdFat\SdCard\SdSpiCard.cpp.o
                0x0000000010007908                _ZN13SharedSpiCard8readDataEPhj
 .text._ZN13SharedSpiCard8readDataEPh
                0x000000001000796a        0xc C:\Users\tomas\AppData\Local\Temp\arduino-sketch-3D6AC107FF947055EEB72537F7027E49\libraries\SdFat\SdCard\SdSpiCard.cpp.o
                0x000000001000796a                _ZN13SharedSpiCard8readDataEPh
 .text._ZN13SharedSpiCard9waitReadyEt
                0x0000000010007976       0x2a C:\Users\tomas\AppData\Local\Temp\arduino-sketch-3D6AC107FF947055EEB72537F7027E49\libraries\SdFat\SdCard\SdSpiCard.cpp.o
                0x0000000010007976                _ZN13SharedSpiCard9waitReadyEt
 .text._ZN13SharedSpiCard9writeDataEhPKh
                0x00000000100079a0       0x4a C:\Users\tomas\AppData\Local\Temp\arduino-sketch-3D6AC107FF947055EEB72537F7027E49\libraries\SdFat\SdCard\SdSpiCard.cpp.o
                0x00000000100079a0                _ZN13SharedSpiCard9writeDataEhPKh
 .text._ZN13SharedSpiCard9writeDataEPKh
                0x00000000100079ea       0x30 C:\Users\tomas\AppData\Local\Temp\arduino-sketch-3D6AC107FF947055EEB72537F7027E49\libraries\SdFat\SdCard\SdSpiCard.cpp.o
                0x00000000100079ea                _ZN13SharedSpiCard9writeDataEPKh
 .text._ZN13SharedSpiCard9writeStopEv
                0x0000000010007a1a       0x32 C:\Users\tomas\AppData\Local\Temp\arduino-sketch-3D6AC107FF947055EEB72537F7027E49\libraries\SdFat\SdCard\SdSpiCard.cpp.o
                0x0000000010007a1a                _ZN13SharedSpiCard9writeStopEv
 .text._ZN13SharedSpiCard10syncDeviceEv
                0x0000000010007a4c       0x1e C:\Users\tomas\AppData\Local\Temp\arduino-sketch-3D6AC107FF947055EEB72537F7027E49\libraries\SdFat\SdCard\SdSpiCard.cpp.o
                0x0000000010007a4c                _ZN13SharedSpiCard10syncDeviceEv
 .text._ZN13SharedSpiCard11cardCommandEhm
                0x0000000010007a6a       0x7c C:\Users\tomas\AppData\Local\Temp\arduino-sketch-3D6AC107FF947055EEB72537F7027E49\libraries\SdFat\SdCard\SdSpiCard.cpp.o
                0x0000000010007a6a                _ZN13SharedSpiCard11cardCommandEhm
 .text._ZN13SharedSpiCard8cardAcmdEhm
                0x0000000010007ae6       0x1c C:\Users\tomas\AppData\Local\Temp\arduino-sketch-3D6AC107FF947055EEB72537F7027E49\libraries\SdFat\SdCard\SdSpiCard.cpp.o
                0x0000000010007ae6                _ZN13SharedSpiCard8cardAcmdEhm
 *fill*         0x0000000010007b02        0x2 
 .text._ZN13SharedSpiCard5beginE11SdSpiConfig
                0x0000000010007b04      0x168 C:\Users\tomas\AppData\Local\Temp\arduino-sketch-3D6AC107FF947055EEB72537F7027E49\libraries\SdFat\SdCard\SdSpiCard.cpp.o
                0x0000000010007b04                _ZN13SharedSpiCard5beginE11SdSpiConfig
 .text._ZN13SharedSpiCard9readStartEm
                0x0000000010007c6c       0x2e C:\Users\tomas\AppData\Local\Temp\arduino-sketch-3D6AC107FF947055EEB72537F7027E49\libraries\SdFat\SdCard\SdSpiCard.cpp.o
                0x0000000010007c6c                _ZN13SharedSpiCard9readStartEm
 .text._ZN13SharedSpiCard8readStopEv
                0x0000000010007c9a       0x2c C:\Users\tomas\AppData\Local\Temp\arduino-sketch-3D6AC107FF947055EEB72537F7027E49\libraries\SdFat\SdCard\SdSpiCard.cpp.o
                0x0000000010007c9a                _ZN13SharedSpiCard8readStopEv
 .text._ZN13SharedSpiCard11writeSectorEmPKh
                0x0000000010007cc6       0x6c C:\Users\tomas\AppData\Local\Temp\arduino-sketch-3D6AC107FF947055EEB72537F7027E49\libraries\SdFat\SdCard\SdSpiCard.cpp.o
                0x0000000010007cc6                _ZN13SharedSpiCard11writeSectorEmPKh
 .text._ZN13SharedSpiCard10writeStartEm
                0x0000000010007d32       0x30 C:\Users\tomas\AppData\Local\Temp\arduino-sketch-3D6AC107FF947055EEB72537F7027E49\libraries\SdFat\SdCard\SdSpiCard.cpp.o
                0x0000000010007d32                _ZN13SharedSpiCard10writeStartEm
 .text._ZN16DedicatedSpiCard5beginE11SdSpiConfig
                0x0000000010007d62       0x1e C:\Users\tomas\AppData\Local\Temp\arduino-sketch-3D6AC107FF947055EEB72537F7027E49\libraries\SdFat\SdCard\SdSpiCard.cpp.o
                0x0000000010007d62                _ZN16DedicatedSpiCard5beginE11SdSpiConfig
 .text._ZN16DedicatedSpiCard11readSectorsEmPhj
                0x0000000010007d80       0x54 C:\Users\tomas\AppData\Local\Temp\arduino-sketch-3D6AC107FF947055EEB72537F7027E49\libraries\SdFat\SdCard\SdSpiCard.cpp.o
                0x0000000010007d80                _ZN16DedicatedSpiCard11readSectorsEmPhj
 .text._ZN16DedicatedSpiCard10readSectorEmPh
                0x0000000010007dd4        0xa C:\Users\tomas\AppData\Local\Temp\arduino-sketch-3D6AC107FF947055EEB72537F7027E49\libraries\SdFat\SdCard\SdSpiCard.cpp.o
                0x0000000010007dd4                _ZN16DedicatedSpiCard10readSectorEmPh
 .text._ZN16DedicatedSpiCard12writeSectorsEmPKhj
                0x0000000010007dde       0x54 C:\Users\tomas\AppData\Local\Temp\arduino-sketch-3D6AC107FF947055EEB72537F7027E49\libraries\SdFat\SdCard\SdSpiCard.cpp.o
                0x0000000010007dde                _ZN16DedicatedSpiCard12writeSectorsEmPKhj
 .text._ZN16DedicatedSpiCard11writeSectorEmPKh
                0x0000000010007e32       0x16 C:\Users\tomas\AppData\Local\Temp\arduino-sketch-3D6AC107FF947055EEB72537F7027E49\libraries\SdFat\SdCard\SdSpiCard.cpp.o
                0x0000000010007e32                _ZN16DedicatedSpiCard11writeSectorEmPKh
 .text._Z8sdCsInith
                0x0000000010007e48        0xa C:\Users\tomas\AppData\Local\Temp\arduino-sketch-3D6AC107FF947055EEB72537F7027E49\libraries\SdFat\SpiDriver\SdSpiChipSelect.cpp.o
                0x0000000010007e48                _Z8sdCsInith
 .text._Z9sdCsWritehb
                0x0000000010007e52        0x8 C:\Users\tomas\AppData\Local\Temp\arduino-sketch-3D6AC107FF947055EEB72537F7027E49\libraries\SdFat\SpiDriver\SdSpiChipSelect.cpp.o
                0x0000000010007e52                _Z9sdCsWritehb
 .text._ZN7FsCache4syncEv
                0x0000000010007e5a       0x48 C:\Users\tomas\AppData\Local\Temp\arduino-sketch-3D6AC107FF947055EEB72537F7027E49\libraries\SdFat\common\FsCache.cpp.o
                0x0000000010007e5a                _ZN7FsCache4syncEv
 .text._ZN7FsCache7prepareEmh
                0x0000000010007ea2       0x4c C:\Users\tomas\AppData\Local\Temp\arduino-sketch-3D6AC107FF947055EEB72537F7027E49\libraries\SdFat\common\FsCache.cpp.o
                0x0000000010007ea2                _ZN7FsCache7prepareEmh
 *fill*         0x0000000010007eee        0x2 
 .text._Z11int64Stringyhbb
                0x0000000010007ef0      0x144 C:\Users\tomas\AppData\Local\Temp\arduino-sketch-3D6AC107FF947055EEB72537F7027E49\libraries\Int64String\Int64String.cpp.o
                0x0000000010007ef0                _Z11int64Stringyhbb
 .text._ZN9SerialUSB5beginEmt
                0x0000000010008034        0xa C:\Users\tomas\AppData\Local\Temp\arduino-sketch-3D6AC107FF947055EEB72537F7027E49/..\arduino-core-cache\core_47e1560ce04abac12f346abb2f6d40c8.a(SerialUSB.cpp.o)
                0x0000000010008034                _ZN9SerialUSB5beginEmt
 .text._ZN9SerialUSB5beginEm
                0x000000001000803e        0xc C:\Users\tomas\AppData\Local\Temp\arduino-sketch-3D6AC107FF947055EEB72537F7027E49/..\arduino-core-cache\core_47e1560ce04abac12f346abb2f6d40c8.a(SerialUSB.cpp.o)
                0x000000001000803e                _ZN9SerialUSB5beginEm
 .text._ZN9SerialUSB3endEv
                0x000000001000804a        0x2 C:\Users\tomas\AppData\Local\Temp\arduino-sketch-3D6AC107FF947055EEB72537F7027E49/..\arduino-core-cache\core_47e1560ce04abac12f346abb2f6d40c8.a(SerialUSB.cpp.o)
                0x000000001000804a                _ZN9SerialUSB3endEv
 .text._ZN9SerialUSB5writeEh
                0x000000001000804c       0x14 C:\Users\tomas\AppData\Local\Temp\arduino-sketch-3D6AC107FF947055EEB72537F7027E49/..\arduino-core-cache\core_47e1560ce04abac12f346abb2f6d40c8.a(SerialUSB.cpp.o)
                0x000000001000804c                _ZN9SerialUSB5writeEh
 .text._ZN9SerialUSB4peekEv
                0x0000000010008060       0x4c C:\Users\tomas\AppData\Local\Temp\arduino-sketch-3D6AC107FF947055EEB72537F7027E49/..\arduino-core-cache\core_47e1560ce04abac12f346abb2f6d40c8.a(SerialUSB.cpp.o)
                0x0000000010008060                _ZN9SerialUSB4peekEv
 .text._ZN9SerialUSB9availableEv
                0x00000000100080ac       0x38 C:\Users\tomas\AppData\Local\Temp\arduino-sketch-3D6AC107FF947055EEB72537F7027E49/..\arduino-core-cache\core_47e1560ce04abac12f346abb2f6d40c8.a(SerialUSB.cpp.o)
                0x00000000100080ac                _ZN9SerialUSB9availableEv
 .text._ZN9SerialUSB17availableForWriteEv
                0x00000000100080e4       0x38 C:\Users\tomas\AppData\Local\Temp\arduino-sketch-3D6AC107FF947055EEB72537F7027E49/..\arduino-core-cache\core_47e1560ce04abac12f346abb2f6d40c8.a(SerialUSB.cpp.o)
                0x00000000100080e4                _ZN9SerialUSB17availableForWriteEv
 .text._ZN9SerialUSB5flushEv
                0x000000001000811c       0x34 C:\Users\tomas\AppData\Local\Temp\arduino-sketch-3D6AC107FF947055EEB72537F7027E49/..\arduino-core-cache\core_47e1560ce04abac12f346abb2f6d40c8.a(SerialUSB.cpp.o)
                0x000000001000811c                _ZN9SerialUSB5flushEv
 .text._ZL16CheckSerialResetv
                0x0000000010008150       0x34 C:\Users\tomas\AppData\Local\Temp\arduino-sketch-3D6AC107FF947055EEB72537F7027E49/..\arduino-core-cache\core_47e1560ce04abac12f346abb2f6d40c8.a(SerialUSB.cpp.o)
 .text._ZN9SerialUSB4readEv
                0x0000000010008184       0x58 C:\Users\tomas\AppData\Local\Temp\arduino-sketch-3D6AC107FF947055EEB72537F7027E49/..\arduino-core-cache\core_47e1560ce04abac12f346abb2f6d40c8.a(SerialUSB.cpp.o)
                0x0000000010008184                _ZN9SerialUSB4readEv
 .text._ZN9SerialUSBcvbEv
                0x00000000100081dc       0x38 C:\Users\tomas\AppData\Local\Temp\arduino-sketch-3D6AC107FF947055EEB72537F7027E49/..\arduino-core-cache\core_47e1560ce04abac12f346abb2f6d40c8.a(SerialUSB.cpp.o)
                0x00000000100081dc                _ZN9SerialUSBcvbEv
 .text._ZN9SerialUSB5writeEPKhj
                0x0000000010008214       0xe0 C:\Users\tomas\AppData\Local\Temp\arduino-sketch-3D6AC107FF947055EEB72537F7027E49/..\arduino-core-cache\core_47e1560ce04abac12f346abb2f6d40c8.a(SerialUSB.cpp.o)
                0x0000000010008214                _ZN9SerialUSB5writeEPKhj
 .text._Z18__USBInstallSerialv
                0x00000000100082f4        0x2 C:\Users\tomas\AppData\Local\Temp\arduino-sketch-3D6AC107FF947055EEB72537F7027E49/..\arduino-core-cache\core_47e1560ce04abac12f346abb2f6d40c8.a(SerialUSB.cpp.o)
                0x00000000100082f4                _Z18__USBInstallSerialv
 *fill*         0x00000000100082f6        0x2 
 .text.tud_cdc_line_state_cb
                0x00000000100082f8       0x10 C:\Users\tomas\AppData\Local\Temp\arduino-sketch-3D6AC107FF947055EEB72537F7027E49/..\arduino-core-cache\core_47e1560ce04abac12f346abb2f6d40c8.a(SerialUSB.cpp.o)
                0x00000000100082f8                tud_cdc_line_state_cb
 .text.tud_cdc_line_coding_cb
                0x0000000010008308       0x24 C:\Users\tomas\AppData\Local\Temp\arduino-sketch-3D6AC107FF947055EEB72537F7027E49/..\arduino-core-cache\core_47e1560ce04abac12f346abb2f6d40c8.a(SerialUSB.cpp.o)
                0x0000000010008308                tud_cdc_line_coding_cb
 .text._ZN7arduino14serialEventRunEv
                0x000000001000832c       0x20 C:\Users\tomas\AppData\Local\Temp\arduino-sketch-3D6AC107FF947055EEB72537F7027E49/..\arduino-core-cache\core_47e1560ce04abac12f346abb2f6d40c8.a(SerialUSB.cpp.o)
                0x000000001000832c                _ZN7arduino14serialEventRunEv
 .text.startup._GLOBAL__sub_I__Z18__USBInstallSerialv
                0x000000001000834c       0x20 C:\Users\tomas\AppData\Local\Temp\arduino-sketch-3D6AC107FF947055EEB72537F7027E49/..\arduino-core-cache\core_47e1560ce04abac12f346abb2f6d40c8.a(SerialUSB.cpp.o)
 .text._ZN7arduino5Print5writeEPKc
                0x000000001000836c       0x1c C:\Users\tomas\AppData\Local\Temp\arduino-sketch-3D6AC107FF947055EEB72537F7027E49/..\arduino-core-cache\core_47e1560ce04abac12f346abb2f6d40c8.a(Print.cpp.o)
                0x000000001000836c                _ZN7arduino5Print5writeEPKc
 .text._ZN7arduino5Print5printEPKc
                0x0000000010008388        0x8 C:\Users\tomas\AppData\Local\Temp\arduino-sketch-3D6AC107FF947055EEB72537F7027E49/..\arduino-core-cache\core_47e1560ce04abac12f346abb2f6d40c8.a(Print.cpp.o)
                0x0000000010008388                _ZN7arduino5Print5printEPKc
 .text._ZN7arduino5Print5printEc
                0x0000000010008390        0xa C:\Users\tomas\AppData\Local\Temp\arduino-sketch-3D6AC107FF947055EEB72537F7027E49/..\arduino-core-cache\core_47e1560ce04abac12f346abb2f6d40c8.a(Print.cpp.o)
                0x0000000010008390                _ZN7arduino5Print5printEc
 *fill*         0x000000001000839a        0x2 
 .text._ZN7arduino5Print7printlnEv
                0x000000001000839c       0x10 C:\Users\tomas\AppData\Local\Temp\arduino-sketch-3D6AC107FF947055EEB72537F7027E49/..\arduino-core-cache\core_47e1560ce04abac12f346abb2f6d40c8.a(Print.cpp.o)
                0x000000001000839c                _ZN7arduino5Print7printlnEv
 .text._ZN7arduino5Print7printlnEPKNS_19__FlashStringHelperE
                0x00000000100083ac       0x14 C:\Users\tomas\AppData\Local\Temp\arduino-sketch-3D6AC107FF947055EEB72537F7027E49/..\arduino-core-cache\core_47e1560ce04abac12f346abb2f6d40c8.a(Print.cpp.o)
                0x00000000100083ac                _ZN7arduino5Print7printlnEPKNS_19__FlashStringHelperE
 .text._ZN7arduino5Print7printlnEPKc
                0x00000000100083c0        0x8 C:\Users\tomas\AppData\Local\Temp\arduino-sketch-3D6AC107FF947055EEB72537F7027E49/..\arduino-core-cache\core_47e1560ce04abac12f346abb2f6d40c8.a(Print.cpp.o)
                0x00000000100083c0                _ZN7arduino5Print7printlnEPKc
 .text._ZN7arduino5Print11printNumberEmh
                0x00000000100083c8       0x50 C:\Users\tomas\AppData\Local\Temp\arduino-sketch-3D6AC107FF947055EEB72537F7027E49/..\arduino-core-cache\core_47e1560ce04abac12f346abb2f6d40c8.a(Print.cpp.o)
                0x00000000100083c8                _ZN7arduino5Print11printNumberEmh
 .text._ZN7arduino5Print5printEli
                0x0000000010008418       0x3e C:\Users\tomas\AppData\Local\Temp\arduino-sketch-3D6AC107FF947055EEB72537F7027E49/..\arduino-core-cache\core_47e1560ce04abac12f346abb2f6d40c8.a(Print.cpp.o)
                0x0000000010008418                _ZN7arduino5Print5printEli
 .text._ZN7arduino5Print5printEii
                0x0000000010008456        0x8 C:\Users\tomas\AppData\Local\Temp\arduino-sketch-3D6AC107FF947055EEB72537F7027E49/..\arduino-core-cache\core_47e1560ce04abac12f346abb2f6d40c8.a(Print.cpp.o)
                0x0000000010008456                _ZN7arduino5Print5printEii
 .text._ZN7arduino5Print7printlnEii
                0x000000001000845e       0x14 C:\Users\tomas\AppData\Local\Temp\arduino-sketch-3D6AC107FF947055EEB72537F7027E49/..\arduino-core-cache\core_47e1560ce04abac12f346abb2f6d40c8.a(Print.cpp.o)
                0x000000001000845e                _ZN7arduino5Print7printlnEii
 .text._ZN7arduino5Print7printlnEli
                0x0000000010008472       0x14 C:\Users\tomas\AppData\Local\Temp\arduino-sketch-3D6AC107FF947055EEB72537F7027E49/..\arduino-core-cache\core_47e1560ce04abac12f346abb2f6d40c8.a(Print.cpp.o)
                0x0000000010008472                _ZN7arduino5Print7printlnEli
 *fill*         0x0000000010008486        0x2 
 .text._ZN7arduino5Print14printULLNumberEyh
                0x0000000010008488       0xdc C:\Users\tomas\AppData\Local\Temp\arduino-sketch-3D6AC107FF947055EEB72537F7027E49/..\arduino-core-cache\core_47e1560ce04abac12f346abb2f6d40c8.a(Print.cpp.o)
                0x0000000010008488                _ZN7arduino5Print14printULLNumberEyh
 .text._ZN7arduino5Print5printEyi
                0x0000000010008564       0x1e C:\Users\tomas\AppData\Local\Temp\arduino-sketch-3D6AC107FF947055EEB72537F7027E49/..\arduino-core-cache\core_47e1560ce04abac12f346abb2f6d40c8.a(Print.cpp.o)
                0x0000000010008564                _ZN7arduino5Print5printEyi
 .text._ZN7arduino5Print7printlnEyi
                0x0000000010008582       0x18 C:\Users\tomas\AppData\Local\Temp\arduino-sketch-3D6AC107FF947055EEB72537F7027E49/..\arduino-core-cache\core_47e1560ce04abac12f346abb2f6d40c8.a(Print.cpp.o)
                0x0000000010008582                _ZN7arduino5Print7printlnEyi
 *fill*         0x000000001000859a        0x2 
 .text._ZN7arduino5Print10printFloatEdi
                0x000000001000859c      0x16c C:\Users\tomas\AppData\Local\Temp\arduino-sketch-3D6AC107FF947055EEB72537F7027E49/..\arduino-core-cache\core_47e1560ce04abac12f346abb2f6d40c8.a(Print.cpp.o)
                0x000000001000859c                _ZN7arduino5Print10printFloatEdi
 .text._ZN7arduino5Print7printlnEdi
                0x0000000010008708       0x18 C:\Users\tomas\AppData\Local\Temp\arduino-sketch-3D6AC107FF947055EEB72537F7027E49/..\arduino-core-cache\core_47e1560ce04abac12f346abb2f6d40c8.a(Print.cpp.o)
                0x0000000010008708                _ZN7arduino5Print7printlnEdi
 .text._ZN7arduino6StringD2Ev
                0x0000000010008720       0x12 C:\Users\tomas\AppData\Local\Temp\arduino-sketch-3D6AC107FF947055EEB72537F7027E49/..\arduino-core-cache\core_47e1560ce04abac12f346abb2f6d40c8.a(String.cpp.o)
                0x0000000010008720                _ZN7arduino6StringD1Ev
                0x0000000010008720                _ZN7arduino6StringD2Ev
 .text._ZN7arduino6String10invalidateEv
                0x0000000010008732       0x18 C:\Users\tomas\AppData\Local\Temp\arduino-sketch-3D6AC107FF947055EEB72537F7027E49/..\arduino-core-cache\core_47e1560ce04abac12f346abb2f6d40c8.a(String.cpp.o)
                0x0000000010008732                _ZN7arduino6String10invalidateEv
 .text._ZN7arduino6String12changeBufferEj
                0x000000001000874a       0x18 C:\Users\tomas\AppData\Local\Temp\arduino-sketch-3D6AC107FF947055EEB72537F7027E49/..\arduino-core-cache\core_47e1560ce04abac12f346abb2f6d40c8.a(String.cpp.o)
                0x000000001000874a                _ZN7arduino6String12changeBufferEj
 .text._ZN7arduino6String7reserveEj
                0x0000000010008762       0x2a C:\Users\tomas\AppData\Local\Temp\arduino-sketch-3D6AC107FF947055EEB72537F7027E49/..\arduino-core-cache\core_47e1560ce04abac12f346abb2f6d40c8.a(String.cpp.o)
                0x0000000010008762                _ZN7arduino6String7reserveEj
 .text._ZN7arduino6String4copyEPKcj
                0x000000001000878c       0x32 C:\Users\tomas\AppData\Local\Temp\arduino-sketch-3D6AC107FF947055EEB72537F7027E49/..\arduino-core-cache\core_47e1560ce04abac12f346abb2f6d40c8.a(String.cpp.o)
                0x000000001000878c                _ZN7arduino6String4copyEPKcj
 .text._ZN7arduino6StringC2EPKc
                0x00000000100087be       0x26 C:\Users\tomas\AppData\Local\Temp\arduino-sketch-3D6AC107FF947055EEB72537F7027E49/..\arduino-core-cache\core_47e1560ce04abac12f346abb2f6d40c8.a(String.cpp.o)
                0x00000000100087be                _ZN7arduino6StringC2EPKc
                0x00000000100087be                _ZN7arduino6StringC1EPKc
 .text._ZN7arduino6String4moveERS0_
                0x00000000100087e4       0x44 C:\Users\tomas\AppData\Local\Temp\arduino-sketch-3D6AC107FF947055EEB72537F7027E49/..\arduino-core-cache\core_47e1560ce04abac12f346abb2f6d40c8.a(String.cpp.o)
                0x00000000100087e4                _ZN7arduino6String4moveERS0_
 .text._ZN7arduino6StringaSERKS0_
                0x0000000010008828       0x20 C:\Users\tomas\AppData\Local\Temp\arduino-sketch-3D6AC107FF947055EEB72537F7027E49/..\arduino-core-cache\core_47e1560ce04abac12f346abb2f6d40c8.a(String.cpp.o)
                0x0000000010008828                _ZN7arduino6StringaSERKS0_
 .text._ZN7arduino6StringC2ERKS0_
                0x0000000010008848       0x14 C:\Users\tomas\AppData\Local\Temp\arduino-sketch-3D6AC107FF947055EEB72537F7027E49/..\arduino-core-cache\core_47e1560ce04abac12f346abb2f6d40c8.a(String.cpp.o)
                0x0000000010008848                _ZN7arduino6StringC2ERKS0_
                0x0000000010008848                _ZN7arduino6StringC1ERKS0_
 .text._ZN7arduino6StringaSEOS0_
                0x000000001000885c       0x10 C:\Users\tomas\AppData\Local\Temp\arduino-sketch-3D6AC107FF947055EEB72537F7027E49/..\arduino-core-cache\core_47e1560ce04abac12f346abb2f6d40c8.a(String.cpp.o)
                0x000000001000885c                _ZN7arduino6StringaSEOS0_
 .text._ZN7arduino6StringaSEPKc
                0x000000001000886c       0x22 C:\Users\tomas\AppData\Local\Temp\arduino-sketch-3D6AC107FF947055EEB72537F7027E49/..\arduino-core-cache\core_47e1560ce04abac12f346abb2f6d40c8.a(String.cpp.o)
                0x000000001000886c                _ZN7arduino6StringaSEPKc
 .text._ZN7arduino6StringC2Ehh
                0x000000001000888e       0x22 C:\Users\tomas\AppData\Local\Temp\arduino-sketch-3D6AC107FF947055EEB72537F7027E49/..\arduino-core-cache\core_47e1560ce04abac12f346abb2f6d40c8.a(String.cpp.o)
                0x000000001000888e                _ZN7arduino6StringC1Ehh
                0x000000001000888e                _ZN7arduino6StringC2Ehh
 .text._ZN7arduino6StringC2Eih
                0x00000000100088b0       0x24 C:\Users\tomas\AppData\Local\Temp\arduino-sketch-3D6AC107FF947055EEB72537F7027E49/..\arduino-core-cache\core_47e1560ce04abac12f346abb2f6d40c8.a(String.cpp.o)
                0x00000000100088b0                _ZN7arduino6StringC1Eih
                0x00000000100088b0                _ZN7arduino6StringC2Eih
 .text._ZN7arduino6String6concatEPKcj
                0x00000000100088d4       0x42 C:\Users\tomas\AppData\Local\Temp\arduino-sketch-3D6AC107FF947055EEB72537F7027E49/..\arduino-core-cache\core_47e1560ce04abac12f346abb2f6d40c8.a(String.cpp.o)
                0x00000000100088d4                _ZN7arduino6String6concatEPKcj
 .text._ZN7arduino6String6concatEPKc.part.0
                0x0000000010008916       0x18 C:\Users\tomas\AppData\Local\Temp\arduino-sketch-3D6AC107FF947055EEB72537F7027E49/..\arduino-core-cache\core_47e1560ce04abac12f346abb2f6d40c8.a(String.cpp.o)
 .text._ZN7arduino6String6concatEPKc
                0x000000001000892e       0x10 C:\Users\tomas\AppData\Local\Temp\arduino-sketch-3D6AC107FF947055EEB72537F7027E49/..\arduino-core-cache\core_47e1560ce04abac12f346abb2f6d40c8.a(String.cpp.o)
                0x000000001000892e                _ZN7arduino6String6concatEPKc
 .text._ZN7arduinoplERKNS_15StringSumHelperERKNS_6StringE
                0x000000001000893e       0x1a C:\Users\tomas\AppData\Local\Temp\arduino-sketch-3D6AC107FF947055EEB72537F7027E49/..\arduino-core-cache\core_47e1560ce04abac12f346abb2f6d40c8.a(String.cpp.o)
                0x000000001000893e                _ZN7arduinoplERKNS_15StringSumHelperERKNS_6StringE
 .text._ZN7arduinoplERKNS_15StringSumHelperEPKc
                0x0000000010008958       0x1c C:\Users\tomas\AppData\Local\Temp\arduino-sketch-3D6AC107FF947055EEB72537F7027E49/..\arduino-core-cache\core_47e1560ce04abac12f346abb2f6d40c8.a(String.cpp.o)
                0x0000000010008958                _ZN7arduinoplERKNS_15StringSumHelperEPKc
 .text.get_absolute_time
                0x0000000010008974       0x2c C:\Users\tomas\AppData\Local\Temp\arduino-sketch-3D6AC107FF947055EEB72537F7027E49/..\arduino-core-cache\core_47e1560ce04abac12f346abb2f6d40c8.a(delay.cpp.o)
 .text.delay    0x00000000100089a0        0xc C:\Users\tomas\AppData\Local\Temp\arduino-sketch-3D6AC107FF947055EEB72537F7027E49/..\arduino-core-cache\core_47e1560ce04abac12f346abb2f6d40c8.a(delay.cpp.o)
                0x00000000100089a0                delay
 .text.delayMicroseconds
                0x00000000100089ac        0xe C:\Users\tomas\AppData\Local\Temp\arduino-sketch-3D6AC107FF947055EEB72537F7027E49/..\arduino-core-cache\core_47e1560ce04abac12f346abb2f6d40c8.a(delay.cpp.o)
                0x00000000100089ac                delayMicroseconds
 .text.millis   0x00000000100089ba       0x26 C:\Users\tomas\AppData\Local\Temp\arduino-sketch-3D6AC107FF947055EEB72537F7027E49/..\arduino-core-cache\core_47e1560ce04abac12f346abb2f6d40c8.a(delay.cpp.o)
                0x00000000100089ba                millis
 .text._ZN6RP204015_SystickHandlerEv
                0x00000000100089e0       0x1c C:\Users\tomas\AppData\Local\Temp\arduino-sketch-3D6AC107FF947055EEB72537F7027E49/..\arduino-core-cache\core_47e1560ce04abac12f346abb2f6d40c8.a(main.cpp.o)
                0x00000000100089e0                _ZN6RP204015_SystickHandlerEv
 .text._ZN6_MFIFO12registerCoreEv.part.0
                0x00000000100089fc       0x24 C:\Users\tomas\AppData\Local\Temp\arduino-sketch-3D6AC107FF947055EEB72537F7027E49/..\arduino-core-cache\core_47e1560ce04abac12f346abb2f6d40c8.a(main.cpp.o)
 .text.main1    0x0000000010008a20       0x30 C:\Users\tomas\AppData\Local\Temp\arduino-sketch-3D6AC107FF947055EEB72537F7027E49/..\arduino-core-cache\core_47e1560ce04abac12f346abb2f6d40c8.a(main.cpp.o)
                0x0000000010008a20                main1
 .text._ZN6_MFIFO5beginEi.part.0.constprop.0
                0x0000000010008a50       0x3c C:\Users\tomas\AppData\Local\Temp\arduino-sketch-3D6AC107FF947055EEB72537F7027E49/..\arduino-core-cache\core_47e1560ce04abac12f346abb2f6d40c8.a(main.cpp.o)
 .text._ZN6RP20405beginEv
                0x0000000010008a8c      0x134 C:\Users\tomas\AppData\Local\Temp\arduino-sketch-3D6AC107FF947055EEB72537F7027E49/..\arduino-core-cache\core_47e1560ce04abac12f346abb2f6d40c8.a(main.cpp.o)
                0x0000000010008a8c                _ZN6RP20405beginEv
 .text.initVariant
                0x0000000010008bc0        0x2 C:\Users\tomas\AppData\Local\Temp\arduino-sketch-3D6AC107FF947055EEB72537F7027E49/..\arduino-core-cache\core_47e1560ce04abac12f346abb2f6d40c8.a(main.cpp.o)
                0x0000000010008bc0                initVariant
 *fill*         0x0000000010008bc2        0x2 
 .text._Z6__loopv
                0x0000000010008bc4       0x30 C:\Users\tomas\AppData\Local\Temp\arduino-sketch-3D6AC107FF947055EEB72537F7027E49/..\arduino-core-cache\core_47e1560ce04abac12f346abb2f6d40c8.a(main.cpp.o)
                0x0000000010008bc4                _Z6__loopv
 .text.__wrap___getreent
                0x0000000010008bf4       0x1c C:\Users\tomas\AppData\Local\Temp\arduino-sketch-3D6AC107FF947055EEB72537F7027E49/..\arduino-core-cache\core_47e1560ce04abac12f346abb2f6d40c8.a(main.cpp.o)
                0x0000000010008bf4                __wrap___getreent
 .text.startup._GLOBAL__sub_I_rp2040
                0x0000000010008c10       0x14 C:\Users\tomas\AppData\Local\Temp\arduino-sketch-3D6AC107FF947055EEB72537F7027E49/..\arduino-core-cache\core_47e1560ce04abac12f346abb2f6d40c8.a(main.cpp.o)
 .text.startup.main
                0x0000000010008c24      0x128 C:\Users\tomas\AppData\Local\Temp\arduino-sketch-3D6AC107FF947055EEB72537F7027E49/..\arduino-core-cache\core_47e1560ce04abac12f346abb2f6d40c8.a(main.cpp.o)
                0x0000000010008c24                main
 .text.adc_read
                0x0000000010008d4c       0x20 C:\Users\tomas\AppData\Local\Temp\arduino-sketch-3D6AC107FF947055EEB72537F7027E49/..\arduino-core-cache\core_47e1560ce04abac12f346abb2f6d40c8.a(wiring_analog.cpp.o)
 .text.analogRead
                0x0000000010008d6c       0x9c C:\Users\tomas\AppData\Local\Temp\arduino-sketch-3D6AC107FF947055EEB72537F7027E49/..\arduino-core-cache\core_47e1560ce04abac12f346abb2f6d40c8.a(wiring_analog.cpp.o)
                0x0000000010008d6c                analogRead
 .text.analogReadResolution
                0x0000000010008e08       0x34 C:\Users\tomas\AppData\Local\Temp\arduino-sketch-3D6AC107FF947055EEB72537F7027E49/..\arduino-core-cache\core_47e1560ce04abac12f346abb2f6d40c8.a(wiring_analog.cpp.o)
                0x0000000010008e08                analogReadResolution
 .text.__pinMode
                0x0000000010008e3c       0xa4 C:\Users\tomas\AppData\Local\Temp\arduino-sketch-3D6AC107FF947055EEB72537F7027E49/..\arduino-core-cache\core_47e1560ce04abac12f346abb2f6d40c8.a(wiring_digital.cpp.o)
                0x0000000010008e3c                pinMode
                0x0000000010008e3c                __pinMode
 .text.__digitalWrite
                0x0000000010008ee0       0x44 C:\Users\tomas\AppData\Local\Temp\arduino-sketch-3D6AC107FF947055EEB72537F7027E49/..\arduino-core-cache\core_47e1560ce04abac12f346abb2f6d40c8.a(wiring_digital.cpp.o)
                0x0000000010008ee0                __digitalWrite
                0x0000000010008ee0                digitalWrite
 .text.__digitalRead
                0x0000000010008f24       0x16 C:\Users\tomas\AppData\Local\Temp\arduino-sketch-3D6AC107FF947055EEB72537F7027E49/..\arduino-core-cache\core_47e1560ce04abac12f346abb2f6d40c8.a(wiring_digital.cpp.o)
                0x0000000010008f24                __digitalRead
                0x0000000010008f24                digitalRead
 .text._ZNSt5dequeImSaImEE4backEv
                0x0000000010008f3a       0x18 C:\Users\tomas\AppData\Local\Temp\arduino-sketch-3D6AC107FF947055EEB72537F7027E49/..\arduino-core-cache\core_47e1560ce04abac12f346abb2f6d40c8.a(wiring_private.cpp.o)
                0x0000000010008f3a                _ZNSt5dequeImSaImEE4backEv
 *fill*         0x0000000010008f52        0x2 
 .text.interrupts
                0x0000000010008f54       0x58 C:\Users\tomas\AppData\Local\Temp\arduino-sketch-3D6AC107FF947055EEB72537F7027E49/..\arduino-core-cache\core_47e1560ce04abac12f346abb2f6d40c8.a(wiring_private.cpp.o)
                0x0000000010008f54                interrupts
 .text.noInterrupts
                0x0000000010008fac      0x164 C:\Users\tomas\AppData\Local\Temp\arduino-sketch-3D6AC107FF947055EEB72537F7027E49/..\arduino-core-cache\core_47e1560ce04abac12f346abb2f6d40c8.a(wiring_private.cpp.o)
                0x0000000010008fac                noInterrupts
 .text.startup._GLOBAL__sub_I_interrupts
                0x0000000010009110       0x74 C:\Users\tomas\AppData\Local\Temp\arduino-sketch-3D6AC107FF947055EEB72537F7027E49/..\arduino-core-cache\core_47e1560ce04abac12f346abb2f6d40c8.a(wiring_private.cpp.o)
 .text._ZN9CoreMutexC2EP5mutexb
                0x0000000010009184       0x48 C:\Users\tomas\AppData\Local\Temp\arduino-sketch-3D6AC107FF947055EEB72537F7027E49/..\arduino-core-cache\core_47e1560ce04abac12f346abb2f6d40c8.a(CoreMutex.cpp.o)
                0x0000000010009184                _ZN9CoreMutexC1EP5mutexb
                0x0000000010009184                _ZN9CoreMutexC2EP5mutexb
 .text._ZN9CoreMutexD2Ev
                0x00000000100091cc       0x2c C:\Users\tomas\AppData\Local\Temp\arduino-sketch-3D6AC107FF947055EEB72537F7027E49/..\arduino-core-cache\core_47e1560ce04abac12f346abb2f6d40c8.a(CoreMutex.cpp.o)
                0x00000000100091cc                _ZN9CoreMutexD1Ev
                0x00000000100091cc                _ZN9CoreMutexD2Ev
 .text._ZL10timer_tasklPv
                0x00000000100091f8       0x18 C:\Users\tomas\AppData\Local\Temp\arduino-sketch-3D6AC107FF947055EEB72537F7027E49/..\arduino-core-cache\core_47e1560ce04abac12f346abb2f6d40c8.a(RP2040USB.cpp.o)
 .text._ZL7usb_irqv
                0x0000000010009210       0x20 C:\Users\tomas\AppData\Local\Temp\arduino-sketch-3D6AC107FF947055EEB72537F7027E49/..\arduino-core-cache\core_47e1560ce04abac12f346abb2f6d40c8.a(RP2040USB.cpp.o)
 .text._ZL20update_us_since_bootP15absolute_time_ty.part.0
                0x0000000010009230       0x1c C:\Users\tomas\AppData\Local\Temp\arduino-sketch-3D6AC107FF947055EEB72537F7027E49/..\arduino-core-cache\core_47e1560ce04abac12f346abb2f6d40c8.a(RP2040USB.cpp.o)
 .text.tud_descriptor_device_cb
                0x000000001000924c       0x84 C:\Users\tomas\AppData\Local\Temp\arduino-sketch-3D6AC107FF947055EEB72537F7027E49/..\arduino-core-cache\core_47e1560ce04abac12f346abb2f6d40c8.a(RP2040USB.cpp.o)
                0x000000001000924c                tud_descriptor_device_cb
 .text._Z20__SetupDescHIDReportv
                0x00000000100092d0      0x254 C:\Users\tomas\AppData\Local\Temp\arduino-sketch-3D6AC107FF947055EEB72537F7027E49/..\arduino-core-cache\core_47e1560ce04abac12f346abb2f6d40c8.a(RP2040USB.cpp.o)
                0x00000000100092d0                _Z20__SetupDescHIDReportv
 .text.tud_hid_descriptor_report_cb
                0x0000000010009524        0xc C:\Users\tomas\AppData\Local\Temp\arduino-sketch-3D6AC107FF947055EEB72537F7027E49/..\arduino-core-cache\core_47e1560ce04abac12f346abb2f6d40c8.a(RP2040USB.cpp.o)
                0x0000000010009524                tud_hid_descriptor_report_cb
 .text.tud_descriptor_configuration_cb
                0x0000000010009530        0xc C:\Users\tomas\AppData\Local\Temp\arduino-sketch-3D6AC107FF947055EEB72537F7027E49/..\arduino-core-cache\core_47e1560ce04abac12f346abb2f6d40c8.a(RP2040USB.cpp.o)
                0x0000000010009530                tud_descriptor_configuration_cb
 .text._Z20__SetupUSBDescriptorv
                0x000000001000953c      0x154 C:\Users\tomas\AppData\Local\Temp\arduino-sketch-3D6AC107FF947055EEB72537F7027E49/..\arduino-core-cache\core_47e1560ce04abac12f346abb2f6d40c8.a(RP2040USB.cpp.o)
                0x000000001000953c                _Z20__SetupUSBDescriptorv
 .text.tud_descriptor_string_cb
                0x0000000010009690       0x68 C:\Users\tomas\AppData\Local\Temp\arduino-sketch-3D6AC107FF947055EEB72537F7027E49/..\arduino-core-cache\core_47e1560ce04abac12f346abb2f6d40c8.a(RP2040USB.cpp.o)
                0x0000000010009690                tud_descriptor_string_cb
 .text._Z10__USBStartv
                0x00000000100096f8       0x7c C:\Users\tomas\AppData\Local\Temp\arduino-sketch-3D6AC107FF947055EEB72537F7027E49/..\arduino-core-cache\core_47e1560ce04abac12f346abb2f6d40c8.a(RP2040USB.cpp.o)
                0x00000000100096f8                _Z10__USBStartv
 .text.tud_hid_get_report_cb
                0x0000000010009774        0x4 C:\Users\tomas\AppData\Local\Temp\arduino-sketch-3D6AC107FF947055EEB72537F7027E49/..\arduino-core-cache\core_47e1560ce04abac12f346abb2f6d40c8.a(RP2040USB.cpp.o)
                0x0000000010009774                tud_hid_get_report_cb
 .text.tud_hid_set_report_cb
                0x0000000010009778        0x2 C:\Users\tomas\AppData\Local\Temp\arduino-sketch-3D6AC107FF947055EEB72537F7027E49/..\arduino-core-cache\core_47e1560ce04abac12f346abb2f6d40c8.a(RP2040USB.cpp.o)
                0x0000000010009778                tud_hid_set_report_cb
 *fill*         0x000000001000977a        0x2 
 .text.__get_freertos_mutex_for_ptr
                0x000000001000977c       0x50 C:\Users\tomas\AppData\Local\Temp\arduino-sketch-3D6AC107FF947055EEB72537F7027E49/..\arduino-core-cache\core_47e1560ce04abac12f346abb2f6d40c8.a(_freertos.cpp.o)
                0x000000001000977c                __get_freertos_mutex_for_ptr
 .text.adc_init
                0x00000000100097cc       0x34 C:\Users\tomas\AppData\Local\Arduino15\packages\rp2040\hardware\rp2040\2.6.0/lib/libpico.a(adc.c.obj)
                0x00000000100097cc                adc_init
 .text.spin_locks_reset
                0x0000000010009800       0x1c C:\Users\tomas\AppData\Local\Arduino15\packages\rp2040\hardware\rp2040\2.6.0/lib/libpico.a(sync.c.obj)
                0x0000000010009800                spin_locks_reset
 .text.next_striped_spin_lock_num
                0x000000001000981c       0x18 C:\Users\tomas\AppData\Local\Arduino15\packages\rp2040\hardware\rp2040\2.6.0/lib/libpico.a(sync.c.obj)
                0x000000001000981c                next_striped_spin_lock_num
 .text.spin_lock_claim_unused
                0x0000000010009834       0x1c C:\Users\tomas\AppData\Local\Arduino15\packages\rp2040\hardware\rp2040\2.6.0/lib/libpico.a(sync.c.obj)
                0x0000000010009834                spin_lock_claim_unused
 .text.clock_configure
                0x0000000010009850       0xd4 C:\Users\tomas\AppData\Local\Arduino15\packages\rp2040\hardware\rp2040\2.6.0/lib/libpico.a(clocks.c.obj)
                0x0000000010009850                clock_configure
 .text.clocks_init
                0x0000000010009924       0xf4 C:\Users\tomas\AppData\Local\Arduino15\packages\rp2040\hardware\rp2040\2.6.0/lib/libpico.a(clocks.c.obj)
                0x0000000010009924                clocks_init
 .text.clock_get_hz
                0x0000000010009a18        0xc C:\Users\tomas\AppData\Local\Arduino15\packages\rp2040\hardware\rp2040\2.6.0/lib/libpico.a(clocks.c.obj)
                0x0000000010009a18                clock_get_hz
 .text.gpio_set_function
                0x0000000010009a24       0x2c C:\Users\tomas\AppData\Local\Arduino15\packages\rp2040\hardware\rp2040\2.6.0/lib/libpico.a(gpio.c.obj)
                0x0000000010009a24                gpio_set_function
 .text.gpio_set_pulls
                0x0000000010009a50       0x2c C:\Users\tomas\AppData\Local\Arduino15\packages\rp2040\hardware\rp2040\2.6.0/lib/libpico.a(gpio.c.obj)
                0x0000000010009a50                gpio_set_pulls
 .text.gpio_set_drive_strength
                0x0000000010009a7c       0x20 C:\Users\tomas\AppData\Local\Arduino15\packages\rp2040\hardware\rp2040\2.6.0/lib/libpico.a(gpio.c.obj)
                0x0000000010009a7c                gpio_set_drive_strength
 .text.gpio_set_input_enabled
                0x0000000010009a9c       0x1c C:\Users\tomas\AppData\Local\Arduino15\packages\rp2040\hardware\rp2040\2.6.0/lib/libpico.a(gpio.c.obj)
                0x0000000010009a9c                gpio_set_input_enabled
 .text.gpio_init
                0x0000000010009ab8       0x16 C:\Users\tomas\AppData\Local\Arduino15\packages\rp2040\hardware\rp2040\2.6.0/lib/libpico.a(gpio.c.obj)
                0x0000000010009ab8                gpio_init
 *fill*         0x0000000010009ace        0x2 
 .text.set_raw_irq_handler_and_unlock
                0x0000000010009ad0       0x28 C:\Users\tomas\AppData\Local\Arduino15\packages\rp2040\hardware\rp2040\2.6.0/lib/libpico.a(irq.c.obj)
 .text.irq_is_enabled
                0x0000000010009af8       0x18 C:\Users\tomas\AppData\Local\Arduino15\packages\rp2040\hardware\rp2040\2.6.0/lib/libpico.a(irq.c.obj)
                0x0000000010009af8                irq_is_enabled
 .text.irq_set_mask_enabled
                0x0000000010009b10       0x20 C:\Users\tomas\AppData\Local\Arduino15\packages\rp2040\hardware\rp2040\2.6.0/lib/libpico.a(irq.c.obj)
                0x0000000010009b10                irq_set_mask_enabled
 .text.irq_set_enabled
                0x0000000010009b30        0xe C:\Users\tomas\AppData\Local\Arduino15\packages\rp2040\hardware\rp2040\2.6.0/lib/libpico.a(irq.c.obj)
                0x0000000010009b30                irq_set_enabled
 *fill*         0x0000000010009b3e        0x2 
 .text.irq_set_pending
                0x0000000010009b40       0x10 C:\Users\tomas\AppData\Local\Arduino15\packages\rp2040\hardware\rp2040\2.6.0/lib/libpico.a(irq.c.obj)
                0x0000000010009b40                irq_set_pending
 .text.irq_get_vtable_handler
                0x0000000010009b50       0x10 C:\Users\tomas\AppData\Local\Arduino15\packages\rp2040\hardware\rp2040\2.6.0/lib/libpico.a(irq.c.obj)
                0x0000000010009b50                irq_get_vtable_handler
 .text.irq_set_exclusive_handler
                0x0000000010009b60       0x40 C:\Users\tomas\AppData\Local\Arduino15\packages\rp2040\hardware\rp2040\2.6.0/lib/libpico.a(irq.c.obj)
                0x0000000010009b60                irq_set_exclusive_handler
 .text.irq_remove_handler
                0x0000000010009ba0      0x160 C:\Users\tomas\AppData\Local\Arduino15\packages\rp2040\hardware\rp2040\2.6.0/lib/libpico.a(irq.c.obj)
                0x0000000010009ba0                irq_remove_handler
 .text.irq_add_tail_to_free_list
                0x0000000010009d00       0xa8 C:\Users\tomas\AppData\Local\Arduino15\packages\rp2040\hardware\rp2040\2.6.0/lib/libpico.a(irq.c.obj)
                0x0000000010009d00                irq_add_tail_to_free_list
 .text.irq_init_priorities
                0x0000000010009da8       0x24 C:\Users\tomas\AppData\Local\Arduino15\packages\rp2040\hardware\rp2040\2.6.0/lib/libpico.a(irq.c.obj)
                0x0000000010009da8                irq_init_priorities
 .text.user_irq_claim_unused
                0x0000000010009dcc       0x2c C:\Users\tomas\AppData\Local\Arduino15\packages\rp2040\hardware\rp2040\2.6.0/lib/libpico.a(irq.c.obj)
                0x0000000010009dcc                user_irq_claim_unused
 .text.time_reached
                0x0000000010009df8       0x28 C:\Users\tomas\AppData\Local\Arduino15\packages\rp2040\hardware\rp2040\2.6.0/lib/libpico.a(time.c.obj)
 .text.timer_pool_entry_comparator
                0x0000000010009e20       0x30 C:\Users\tomas\AppData\Local\Arduino15\packages\rp2040\hardware\rp2040\2.6.0/lib/libpico.a(time.c.obj)
                0x0000000010009e20                timer_pool_entry_comparator
 .text.alarm_pool_post_alloc_init
                0x0000000010009e50       0x3c C:\Users\tomas\AppData\Local\Arduino15\packages\rp2040\hardware\rp2040\2.6.0/lib/libpico.a(time.c.obj)
 .text.sleep_until_callback
                0x0000000010009e8c       0x30 C:\Users\tomas\AppData\Local\Arduino15\packages\rp2040\hardware\rp2040\2.6.0/lib/libpico.a(time.c.obj)
 .text.ph_add_child_node.isra.0
                0x0000000010009ebc       0x22 C:\Users\tomas\AppData\Local\Arduino15\packages\rp2040\hardware\rp2040\2.6.0/lib/libpico.a(time.c.obj)
 *fill*         0x0000000010009ede        0x2 
 .text.add_alarm_under_lock
                0x0000000010009ee0       0xc8 C:\Users\tomas\AppData\Local\Arduino15\packages\rp2040\hardware\rp2040\2.6.0/lib/libpico.a(time.c.obj)
 .text.alarm_pool_alarm_callback
                0x0000000010009fa8      0x188 C:\Users\tomas\AppData\Local\Arduino15\packages\rp2040\hardware\rp2040\2.6.0/lib/libpico.a(time.c.obj)
 .text.alarm_pool_init_default
                0x000000001000a130       0x34 C:\Users\tomas\AppData\Local\Arduino15\packages\rp2040\hardware\rp2040\2.6.0/lib/libpico.a(time.c.obj)
                0x000000001000a130                alarm_pool_init_default
 .text.alarm_pool_get_default
                0x000000001000a164        0x8 C:\Users\tomas\AppData\Local\Arduino15\packages\rp2040\hardware\rp2040\2.6.0/lib/libpico.a(time.c.obj)
                0x000000001000a164                alarm_pool_get_default
 .text.alarm_pool_add_alarm_at
                0x000000001000a16c       0xda C:\Users\tomas\AppData\Local\Arduino15\packages\rp2040\hardware\rp2040\2.6.0/lib/libpico.a(time.c.obj)
                0x000000001000a16c                alarm_pool_add_alarm_at
 .text.alarm_pool_cancel_alarm
                0x000000001000a246       0x66 C:\Users\tomas\AppData\Local\Arduino15\packages\rp2040\hardware\rp2040\2.6.0/lib/libpico.a(time.c.obj)
                0x000000001000a246                alarm_pool_cancel_alarm
 .text.sleep_until
                0x000000001000a2ac       0x98 C:\Users\tomas\AppData\Local\Arduino15\packages\rp2040\hardware\rp2040\2.6.0/lib/libpico.a(time.c.obj)
                0x000000001000a2ac                sleep_until
 .text.sleep_us
                0x000000001000a344       0x2c C:\Users\tomas\AppData\Local\Arduino15\packages\rp2040\hardware\rp2040\2.6.0/lib/libpico.a(time.c.obj)
                0x000000001000a344                sleep_us
 .text.sleep_ms
                0x000000001000a370       0x14 C:\Users\tomas\AppData\Local\Arduino15\packages\rp2040\hardware\rp2040\2.6.0/lib/libpico.a(time.c.obj)
                0x000000001000a370                sleep_ms
 .text.best_effort_wfe_or_timeout
                0x000000001000a384       0x40 C:\Users\tomas\AppData\Local\Arduino15\packages\rp2040\hardware\rp2040\2.6.0/lib/libpico.a(time.c.obj)
                0x000000001000a384                best_effort_wfe_or_timeout
 .text.hardware_alarm_irq_handler
                0x000000001000a3c4       0x90 C:\Users\tomas\AppData\Local\Arduino15\packages\rp2040\hardware\rp2040\2.6.0/lib/libpico.a(timer.c.obj)
 .text.hardware_alarm_claim
                0x000000001000a454       0x18 C:\Users\tomas\AppData\Local\Arduino15\packages\rp2040\hardware\rp2040\2.6.0/lib/libpico.a(timer.c.obj)
                0x000000001000a454                hardware_alarm_claim
 .text.time_us_64
                0x000000001000a46c       0x14 C:\Users\tomas\AppData\Local\Arduino15\packages\rp2040\hardware\rp2040\2.6.0/lib/libpico.a(timer.c.obj)
                0x000000001000a46c                time_us_64
 .text.busy_wait_until
                0x000000001000a480       0x1c C:\Users\tomas\AppData\Local\Arduino15\packages\rp2040\hardware\rp2040\2.6.0/lib/libpico.a(timer.c.obj)
                0x000000001000a480                busy_wait_until
 .text.hardware_alarm_set_callback
                0x000000001000a49c       0x94 C:\Users\tomas\AppData\Local\Arduino15\packages\rp2040\hardware\rp2040\2.6.0/lib/libpico.a(timer.c.obj)
                0x000000001000a49c                hardware_alarm_set_callback
 .text.hardware_alarm_set_target
                0x000000001000a530       0xbc C:\Users\tomas\AppData\Local\Arduino15\packages\rp2040\hardware\rp2040\2.6.0/lib/libpico.a(timer.c.obj)
                0x000000001000a530                hardware_alarm_set_target
 .text.hardware_alarm_cancel
                0x000000001000a5ec       0x40 C:\Users\tomas\AppData\Local\Arduino15\packages\rp2040\hardware\rp2040\2.6.0/lib/libpico.a(timer.c.obj)
                0x000000001000a5ec                hardware_alarm_cancel
 .text.ph_add_child_node.isra.0
                0x000000001000a62c       0x22 C:\Users\tomas\AppData\Local\Arduino15\packages\rp2040\hardware\rp2040\2.6.0/lib/libpico.a(pheap.c.obj)
 .text.ph_merge_nodes
                0x000000001000a64e       0x36 C:\Users\tomas\AppData\Local\Arduino15\packages\rp2040\hardware\rp2040\2.6.0/lib/libpico.a(pheap.c.obj)
 .text.ph_clear
                0x000000001000a684       0x34 C:\Users\tomas\AppData\Local\Arduino15\packages\rp2040\hardware\rp2040\2.6.0/lib/libpico.a(pheap.c.obj)
                0x000000001000a684                ph_clear
 .text.ph_post_alloc_init
                0x000000001000a6b8        0xe C:\Users\tomas\AppData\Local\Arduino15\packages\rp2040\hardware\rp2040\2.6.0/lib/libpico.a(pheap.c.obj)
                0x000000001000a6b8                ph_post_alloc_init
 .text.ph_merge_two_pass
                0x000000001000a6c6       0x48 C:\Users\tomas\AppData\Local\Arduino15\packages\rp2040\hardware\rp2040\2.6.0/lib/libpico.a(pheap.c.obj)
                0x000000001000a6c6                ph_merge_two_pass
 .text.ph_remove_any_head
                0x000000001000a70e       0x4a C:\Users\tomas\AppData\Local\Arduino15\packages\rp2040\hardware\rp2040\2.6.0/lib/libpico.a(pheap.c.obj)
 .text.ph_remove_head
                0x000000001000a758       0x14 C:\Users\tomas\AppData\Local\Arduino15\packages\rp2040\hardware\rp2040\2.6.0/lib/libpico.a(pheap.c.obj)
                0x000000001000a758                ph_remove_head
 .text.ph_remove_and_free_node
                0x000000001000a76c       0x6e C:\Users\tomas\AppData\Local\Arduino15\packages\rp2040\hardware\rp2040\2.6.0/lib/libpico.a(pheap.c.obj)
                0x000000001000a76c                ph_remove_and_free_node
 .text.queue_init_with_spinlock
                0x000000001000a7da       0x22 C:\Users\tomas\AppData\Local\Arduino15\packages\rp2040\hardware\rp2040\2.6.0/lib/libpico.a(queue.c.obj)
                0x000000001000a7da                queue_init_with_spinlock
 .text.mutex_init
                0x000000001000a7fc       0x1a C:\Users\tomas\AppData\Local\Arduino15\packages\rp2040\hardware\rp2040\2.6.0/lib/libpico.a(mutex.c.obj)
                0x000000001000a7fc                mutex_init
 .text.recursive_mutex_init
                0x000000001000a816       0x1a C:\Users\tomas\AppData\Local\Arduino15\packages\rp2040\hardware\rp2040\2.6.0/lib/libpico.a(mutex.c.obj)
                0x000000001000a816                recursive_mutex_init
 .text.pll_init
                0x000000001000a830       0x9c C:\Users\tomas\AppData\Local\Arduino15\packages\rp2040\hardware\rp2040\2.6.0/lib/libpico.a(pll.c.obj)
                0x000000001000a830                pll_init
 .text.watchdog_start_tick
                0x000000001000a8cc       0x10 C:\Users\tomas\AppData\Local\Arduino15\packages\rp2040\hardware\rp2040\2.6.0/lib/libpico.a(watchdog.c.obj)
                0x000000001000a8cc                watchdog_start_tick
 .text.xosc_init
                0x000000001000a8dc       0x28 C:\Users\tomas\AppData\Local\Arduino15\packages\rp2040\hardware\rp2040\2.6.0/lib/libpico.a(xosc.c.obj)
                0x000000001000a8dc                xosc_init
 .text.exception_get_vtable_handler
                0x000000001000a904       0x10 C:\Users\tomas\AppData\Local\Arduino15\packages\rp2040\hardware\rp2040\2.6.0/lib/libpico.a(exception.c.obj)
                0x000000001000a904                exception_get_vtable_handler
 .text.exception_set_exclusive_handler
                0x000000001000a914       0x48 C:\Users\tomas\AppData\Local\Arduino15\packages\rp2040\hardware\rp2040\2.6.0/lib/libpico.a(exception.c.obj)
                0x000000001000a914                exception_set_exclusive_handler
 .text.rom_func_lookup
                0x000000001000a95c       0x10 C:\Users\tomas\AppData\Local\Arduino15\packages\rp2040\hardware\rp2040\2.6.0/lib/libpico.a(bootrom.c.obj)
                0x000000001000a95c                rom_func_lookup
 .text.rom_data_lookup
                0x000000001000a96c       0x10 C:\Users\tomas\AppData\Local\Arduino15\packages\rp2040\hardware\rp2040\2.6.0/lib/libpico.a(bootrom.c.obj)
                0x000000001000a96c                rom_data_lookup
 .text.rom_funcs_lookup
                0x000000001000a97c       0x26 C:\Users\tomas\AppData\Local\Arduino15\packages\rp2040\hardware\rp2040\2.6.0/lib/libpico.a(bootrom.c.obj)
                0x000000001000a97c                rom_funcs_lookup
 *fill*         0x000000001000a9a2        0x2 
 .text._pio_find_offset_for_program.isra.0
                0x000000001000a9a4       0x48 C:\Users\tomas\AppData\Local\Arduino15\packages\rp2040\hardware\rp2040\2.6.0/lib/libpico.a(pio.c.obj)
 .text._pio_add_program_at_offset
                0x000000001000a9ec       0x80 C:\Users\tomas\AppData\Local\Arduino15\packages\rp2040\hardware\rp2040\2.6.0/lib/libpico.a(pio.c.obj)
 .text.pio_claim_unused_sm
                0x000000001000aa6c       0x34 C:\Users\tomas\AppData\Local\Arduino15\packages\rp2040\hardware\rp2040\2.6.0/lib/libpico.a(pio.c.obj)
                0x000000001000aa6c                pio_claim_unused_sm
 .text.pio_can_add_program
                0x000000001000aaa0       0x2a C:\Users\tomas\AppData\Local\Arduino15\packages\rp2040\hardware\rp2040\2.6.0/lib/libpico.a(pio.c.obj)
                0x000000001000aaa0                pio_can_add_program
 *fill*         0x000000001000aaca        0x2 
 .text.pio_add_program
                0x000000001000aacc       0x3c C:\Users\tomas\AppData\Local\Arduino15\packages\rp2040\hardware\rp2040\2.6.0/lib/libpico.a(pio.c.obj)
                0x000000001000aacc                pio_add_program
 .text.pio_sm_init
                0x000000001000ab08       0x88 C:\Users\tomas\AppData\Local\Arduino15\packages\rp2040\hardware\rp2040\2.6.0/lib/libpico.a(pio.c.obj)
                0x000000001000ab08                pio_sm_init
 .text.spi_deinit
                0x000000001000ab90       0x38 C:\Users\tomas\AppData\Local\Arduino15\packages\rp2040\hardware\rp2040\2.6.0/lib/libpico.a(spi.c.obj)
                0x000000001000ab90                spi_deinit
 .text.spi_set_baudrate
                0x000000001000abc8       0x8c C:\Users\tomas\AppData\Local\Arduino15\packages\rp2040\hardware\rp2040\2.6.0/lib/libpico.a(spi.c.obj)
                0x000000001000abc8                spi_set_baudrate
 .text.spi_init
                0x000000001000ac54       0x6c C:\Users\tomas\AppData\Local\Arduino15\packages\rp2040\hardware\rp2040\2.6.0/lib/libpico.a(spi.c.obj)
                0x000000001000ac54                spi_init
 .text          0x000000001000acc0       0x10 C:\Users\tomas\AppData\Local\Arduino15\packages\rp2040\hardware\rp2040\2.6.0/lib/libpico.a(bit_ops_aeabi.S.obj)
 .text.startup._retrieve_unique_id_on_boot
                0x000000001000acd0       0x10 C:\Users\tomas\AppData\Local\Arduino15\packages\rp2040\hardware\rp2040\2.6.0/lib/libpico.a(unique_id.c.obj)
 .text.pico_get_unique_board_id_string
                0x000000001000ace0       0x44 C:\Users\tomas\AppData\Local\Arduino15\packages\rp2040\hardware\rp2040\2.6.0/lib/libpico.a(unique_id.c.obj)
                0x000000001000ace0                pico_get_unique_board_id_string
 .text.set_sys_clock_pll
                0x000000001000ad24       0x78 C:\Users\tomas\AppData\Local\Arduino15\packages\rp2040\hardware\rp2040\2.6.0/lib/libpico.a(stdlib.c.obj)
                0x000000001000ad24                set_sys_clock_pll
 .text.check_sys_clock_khz
                0x000000001000ad9c       0x8c C:\Users\tomas\AppData\Local\Arduino15\packages\rp2040\hardware\rp2040\2.6.0/lib/libpico.a(stdlib.c.obj)
                0x000000001000ad9c                check_sys_clock_khz
 .text.runtime_init
                0x000000001000ae28       0xcc C:\Users\tomas\AppData\Local\Arduino15\packages\rp2040\hardware\rp2040\2.6.0/lib/libpico.a(runtime.c.obj)
                0x000000001000ae28                runtime_init
 .text._exit    0x000000001000aef4        0x4 C:\Users\tomas\AppData\Local\Arduino15\packages\rp2040\hardware\rp2040\2.6.0/lib/libpico.a(runtime.c.obj)
                0x000000001000aef4                _exit
 .text._sbrk    0x000000001000aef8       0x30 C:\Users\tomas\AppData\Local\Arduino15\packages\rp2040\hardware\rp2040\2.6.0/lib/libpico.a(runtime.c.obj)
                0x000000001000aef8                _sbrk
 .text.exit     0x000000001000af28        0x4 C:\Users\tomas\AppData\Local\Arduino15\packages\rp2040\hardware\rp2040\2.6.0/lib/libpico.a(runtime.c.obj)
                0x000000001000af28                exit
 .text.__assert_func
                0x000000001000af2c       0x30 C:\Users\tomas\AppData\Local\Arduino15\packages\rp2040\hardware\rp2040\2.6.0/lib/libpico.a(runtime.c.obj)
                0x000000001000af2c                __assert_func
 .text.panic    0x000000001000af5c       0x2c C:\Users\tomas\AppData\Local\Arduino15\packages\rp2040\hardware\rp2040\2.6.0/lib/libpico.a(runtime.c.obj)
                0x000000001000af5c                panic
 .text.hard_assertion_failure
                0x000000001000af88        0xc C:\Users\tomas\AppData\Local\Arduino15\packages\rp2040\hardware\rp2040\2.6.0/lib/libpico.a(runtime.c.obj)
                0x000000001000af88                hard_assertion_failure
 .text.__wrap___aeabi_idiv
                0x000000001000af94       0x50 C:\Users\tomas\AppData\Local\Arduino15\packages\rp2040\hardware\rp2040\2.6.0/lib/libpico.a(divider.S.obj)
                0x000000001000af94                __wrap___aeabi_idivmod
                0x000000001000af94                divmod_s32s32
                0x000000001000af94                div_s32s32
                0x000000001000af94                __wrap___aeabi_idiv
                0x000000001000af9c                divmod_s32s32_unsafe
                0x000000001000afc8                divmod_s32s32_savestate
 .text.__wrap___aeabi_uidiv
                0x000000001000afe4       0x4c C:\Users\tomas\AppData\Local\Arduino15\packages\rp2040\hardware\rp2040\2.6.0/lib/libpico.a(divider.S.obj)
                0x000000001000afe4                __wrap___aeabi_uidiv
                0x000000001000afe4                __wrap___aeabi_uidivmod
                0x000000001000afe4                div_u32u32
                0x000000001000afe4                divmod_u32u32
                0x000000001000afec                divmod_u32u32_unsafe
                0x000000001000b014                divmod_u32u32_savestate
 .text.__wrap___aeabi_ldiv
                0x000000001000b030      0x434 C:\Users\tomas\AppData\Local\Arduino15\packages\rp2040\hardware\rp2040\2.6.0/lib/libpico.a(divider.S.obj)
                0x000000001000b030                div_s64s64
                0x000000001000b030                divmod_s64s64
                0x000000001000b030                __wrap___aeabi_ldivmod
                0x000000001000b068                divmod_u64u64
                0x000000001000b068                div_u64u64
                0x000000001000b068                __wrap___aeabi_uldivmod
                0x000000001000b078                divmod_u64u64_savestate
                0x000000001000b0a0                divmod_s64s64_unsafe
                0x000000001000b128                divmod_u64u64_unsafe
 .text.__wrap___aeabi_darithmetic
                0x000000001000b464       0x80 C:\Users\tomas\AppData\Local\Arduino15\packages\rp2040\hardware\rp2040\2.6.0/lib/libpico.a(double_aeabi.S.obj)
                0x000000001000b464                __wrap___aeabi_drsub
                0x000000001000b46a                __wrap___aeabi_dsub
                0x000000001000b47c                __wrap___aeabi_dadd
                0x000000001000b48e                __wrap___aeabi_ddiv
                0x000000001000b4ca                __wrap___aeabi_dmul
 .text.__wrap___aeabi_cdcmple
                0x000000001000b4e4       0x6c C:\Users\tomas\AppData\Local\Arduino15\packages\rp2040\hardware\rp2040\2.6.0/lib/libpico.a(double_aeabi.S.obj)
                0x000000001000b4e4                __wrap___aeabi_cdrcmple
                0x000000001000b4f4                __wrap___aeabi_cdcmpeq
                0x000000001000b4f4                __wrap___aeabi_cdcmple
 .text.__wrap___aeabi_dcmpeq
                0x000000001000b550       0x10 C:\Users\tomas\AppData\Local\Arduino15\packages\rp2040\hardware\rp2040\2.6.0/lib/libpico.a(double_aeabi.S.obj)
                0x000000001000b550                __wrap___aeabi_dcmpeq
 .text.__wrap___aeabi_dcmplt
                0x000000001000b560        0xc C:\Users\tomas\AppData\Local\Arduino15\packages\rp2040\hardware\rp2040\2.6.0/lib/libpico.a(double_aeabi.S.obj)
                0x000000001000b560                __wrap___aeabi_dcmplt
 .text.__wrap___aeabi_dcmple
                0x000000001000b56c       0x10 C:\Users\tomas\AppData\Local\Arduino15\packages\rp2040\hardware\rp2040\2.6.0/lib/libpico.a(double_aeabi.S.obj)
                0x000000001000b56c                __wrap___aeabi_dcmple
 .text.__wrap___aeabi_dcmpge
                0x000000001000b57c       0x10 C:\Users\tomas\AppData\Local\Arduino15\packages\rp2040\hardware\rp2040\2.6.0/lib/libpico.a(double_aeabi.S.obj)
                0x000000001000b57c                __wrap___aeabi_dcmpge
 .text.__wrap___aeabi_dcmpgt
                0x000000001000b58c        0xa C:\Users\tomas\AppData\Local\Arduino15\packages\rp2040\hardware\rp2040\2.6.0/lib/libpico.a(double_aeabi.S.obj)
                0x000000001000b58c                __wrap___aeabi_dcmpgt
 .text.__wrap___aeabi_dcmpun
                0x000000001000b596       0x1c C:\Users\tomas\AppData\Local\Arduino15\packages\rp2040\hardware\rp2040\2.6.0/lib/libpico.a(double_aeabi.S.obj)
                0x000000001000b596                __wrap___aeabi_dcmpun
 *fill*         0x000000001000b5b2        0x2 
 .text.__wrap___aeabi_i2d
                0x000000001000b5b4       0x38 C:\Users\tomas\AppData\Local\Arduino15\packages\rp2040\hardware\rp2040\2.6.0/lib/libpico.a(double_aeabi.S.obj)
                0x000000001000b5b4                __wrap___aeabi_ui2d
                0x000000001000b5bc                __wrap___aeabi_i2d
 .text.__wrap___aeabi_d2iz
                0x000000001000b5ec       0x48 C:\Users\tomas\AppData\Local\Arduino15\packages\rp2040\hardware\rp2040\2.6.0/lib/libpico.a(double_aeabi.S.obj)
                0x000000001000b5ec                double2int_z
                0x000000001000b5ec                __wrap___aeabi_d2iz
 .text.__wrap___aeabi_d2uiz
                0x000000001000b634       0x18 C:\Users\tomas\AppData\Local\Arduino15\packages\rp2040\hardware\rp2040\2.6.0/lib/libpico.a(double_aeabi.S.obj)
                0x000000001000b634                __wrap___aeabi_d2uiz
                0x000000001000b634                double2uint
 .text.__wrap___aeabi_l2d
                0x000000001000b64c       0x18 C:\Users\tomas\AppData\Local\Arduino15\packages\rp2040\hardware\rp2040\2.6.0/lib/libpico.a(double_aeabi.S.obj)
                0x000000001000b64c                __wrap___aeabi_l2d
 .text.__wrap___aeabi_ul2d
                0x000000001000b664       0x18 C:\Users\tomas\AppData\Local\Arduino15\packages\rp2040\hardware\rp2040\2.6.0/lib/libpico.a(double_aeabi.S.obj)
                0x000000001000b664                __wrap___aeabi_ul2d
 .text.__wrap___aeabi_d2lz
                0x000000001000b67c       0x26 C:\Users\tomas\AppData\Local\Arduino15\packages\rp2040\hardware\rp2040\2.6.0/lib/libpico.a(double_aeabi.S.obj)
                0x000000001000b67c                double2int64_z
                0x000000001000b67c                __wrap___aeabi_d2lz
 *fill*         0x000000001000b6a2        0x2 
 .text.double2int64
                0x000000001000b6a4       0x18 C:\Users\tomas\AppData\Local\Arduino15\packages\rp2040\hardware\rp2040\2.6.0/lib/libpico.a(double_aeabi.S.obj)
                0x000000001000b6a4                double2int64
 .text.__wrap___aeabi_d2ulz
                0x000000001000b6bc       0x18 C:\Users\tomas\AppData\Local\Arduino15\packages\rp2040\hardware\rp2040\2.6.0/lib/libpico.a(double_aeabi.S.obj)
                0x000000001000b6bc                __wrap___aeabi_d2ulz
 .text.double2ufix64
                0x000000001000b6d4       0x18 C:\Users\tomas\AppData\Local\Arduino15\packages\rp2040\hardware\rp2040\2.6.0/lib/libpico.a(double_aeabi.S.obj)
                0x000000001000b6d4                double2ufix64
 .text.__wrap___aeabi_d2f
                0x000000001000b6ec       0x18 C:\Users\tomas\AppData\Local\Arduino15\packages\rp2040\hardware\rp2040\2.6.0/lib/libpico.a(double_aeabi.S.obj)
                0x000000001000b6ec                __wrap___aeabi_d2f
 .text.__aeabi_double_init
                0x000000001000b704       0x58 C:\Users\tomas\AppData\Local\Arduino15\packages\rp2040\hardware\rp2040\2.6.0/lib/libpico.a(double_init_rom.c.obj)
                0x000000001000b704                __aeabi_double_init
 .text.double_table_shim_on_use_helper
                0x000000001000b75c       0x2c C:\Users\tomas\AppData\Local\Arduino15\packages\rp2040\hardware\rp2040\2.6.0/lib/libpico.a(double_v1_rom_shim.S.obj)
                0x000000001000b75c                double_table_shim_on_use_helper
 .text.__wrap___aeabi_dsub
                0x000000001000b788       0x10 C:\Users\tomas\AppData\Local\Arduino15\packages\rp2040\hardware\rp2040\2.6.0/lib/libpico.a(double_v1_rom_shim.S.obj)
                0x000000001000b788                drsub_shim
                0x000000001000b78e                dsub_shim
 .text.dadd_shim
                0x000000001000b798      0x15c C:\Users\tomas\AppData\Local\Arduino15\packages\rp2040\hardware\rp2040\2.6.0/lib/libpico.a(double_v1_rom_shim.S.obj)
                0x000000001000b798                dadd_shim
 .text.dmul_shim
                0x000000001000b8f4      0x15c C:\Users\tomas\AppData\Local\Arduino15\packages\rp2040\hardware\rp2040\2.6.0/lib/libpico.a(double_v1_rom_shim.S.obj)
                0x000000001000b8f4                dmul_shim
 .text.ddiv_shim
                0x000000001000ba50      0x1b0 C:\Users\tomas\AppData\Local\Arduino15\packages\rp2040\hardware\rp2040\2.6.0/lib/libpico.a(double_v1_rom_shim.S.obj)
                0x000000001000ba50                ddiv_shim
 .text.double2uint_shim
                0x000000001000bc00        0xe C:\Users\tomas\AppData\Local\Arduino15\packages\rp2040\hardware\rp2040\2.6.0/lib/libpico.a(double_v1_rom_shim.S.obj)
                0x000000001000bc00                double2uint_shim
                0x000000001000bc02                double2ufix_shim
 .text.double2int64_shim
                0x000000001000bc0e       0x1a C:\Users\tomas\AppData\Local\Arduino15\packages\rp2040\hardware\rp2040\2.6.0/lib/libpico.a(double_v1_rom_shim.S.obj)
                0x000000001000bc0e                double2int64_shim
                0x000000001000bc10                double2fix64_shim
 .text.double2uint64_shim
                0x000000001000bc28       0x70 C:\Users\tomas\AppData\Local\Arduino15\packages\rp2040\hardware\rp2040\2.6.0/lib/libpico.a(double_v1_rom_shim.S.obj)
                0x000000001000bc28                double2uint64_shim
                0x000000001000bc2a                double2ufix64_shim
                0x000000001000bc4a                d2fix_a
 .text.double2float_shim
                0x000000001000bc98       0x5c C:\Users\tomas\AppData\Local\Arduino15\packages\rp2040\hardware\rp2040\2.6.0/lib/libpico.a(double_v1_rom_shim.S.obj)
                0x000000001000bc98                double2float_shim
 .text.x2double_shims
                0x000000001000bcf4       0x90 C:\Users\tomas\AppData\Local\Arduino15\packages\rp2040\hardware\rp2040\2.6.0/lib/libpico.a(double_v1_rom_shim.S.obj)
                0x000000001000bcf4                uint2double_shim
                0x000000001000bcf6                ufix2double_shim
                0x000000001000bcfc                int2double_shim
                0x000000001000bcfe                fix2double_shim
                0x000000001000bd04                uint642double_shim
                0x000000001000bd06                ufix642double_shim
                0x000000001000bd0c                int642double_shim
                0x000000001000bd0e                fix642double_shim
 .text.dunpacks
                0x000000001000bd84       0x3c C:\Users\tomas\AppData\Local\Arduino15\packages\rp2040\hardware\rp2040\2.6.0/lib/libpico.a(double_v1_rom_shim.S.obj)
                0x000000001000bd84                dunpacks
 .text.__aeabi_lmul
                0x000000001000bdc0       0x32 C:\Users\tomas\AppData\Local\Arduino15\packages\rp2040\hardware\rp2040\2.6.0/lib/libpico.a(pico_int64_ops_aeabi.S.obj)
                0x000000001000bdc0                __wrap___aeabi_lmul
 *fill*         0x000000001000bdf2        0x2 
 .text.__wrap___aeabi_farithmetic
                0x000000001000bdf4       0x48 C:\Users\tomas\AppData\Local\Arduino15\packages\rp2040\hardware\rp2040\2.6.0/lib/libpico.a(float_aeabi.S.obj)
                0x000000001000bdf4                __wrap___aeabi_frsub
                0x000000001000bdfa                __wrap___aeabi_fsub
                0x000000001000be00                __wrap___aeabi_fadd
                0x000000001000be06                __wrap___aeabi_fdiv
                0x000000001000be2e                __wrap___aeabi_fmul
 .text.__wrap___aeabi_cfcmple
                0x000000001000be3c       0x50 C:\Users\tomas\AppData\Local\Arduino15\packages\rp2040\hardware\rp2040\2.6.0/lib/libpico.a(float_aeabi.S.obj)
                0x000000001000be3c                __wrap___aeabi_cfrcmple
                0x000000001000be48                __wrap___aeabi_cfcmple
                0x000000001000be48                __wrap___aeabi_cfcmpeq
 .text.__wrap___aeabi_fcmple
                0x000000001000be8c       0x10 C:\Users\tomas\AppData\Local\Arduino15\packages\rp2040\hardware\rp2040\2.6.0/lib/libpico.a(float_aeabi.S.obj)
                0x000000001000be8c                __wrap___aeabi_fcmple
 .text.__wrap___aeabi_fcmpun
                0x000000001000be9c       0x18 C:\Users\tomas\AppData\Local\Arduino15\packages\rp2040\hardware\rp2040\2.6.0/lib/libpico.a(float_aeabi.S.obj)
                0x000000001000be9c                __wrap___aeabi_fcmpun
 .text.__wrap___aeabi_ui2f
                0x000000001000beb4        0xa C:\Users\tomas\AppData\Local\Arduino15\packages\rp2040\hardware\rp2040\2.6.0/lib/libpico.a(float_aeabi.S.obj)
                0x000000001000beb4                __wrap___aeabi_ui2f
 *fill*         0x000000001000bebe        0x2 
 .text.__wrap___aeabi_i2f
                0x000000001000bec0       0x44 C:\Users\tomas\AppData\Local\Arduino15\packages\rp2040\hardware\rp2040\2.6.0/lib/libpico.a(float_aeabi.S.obj)
                0x000000001000bec0                __wrap___aeabi_i2f
 .text.__wrap___aeabi_l2f
                0x000000001000bf04       0x20 C:\Users\tomas\AppData\Local\Arduino15\packages\rp2040\hardware\rp2040\2.6.0/lib/libpico.a(float_aeabi.S.obj)
                0x000000001000bf08                __wrap___aeabi_l2f
 .text.__wrap___aeabi_ul2f
                0x000000001000bf24       0x20 C:\Users\tomas\AppData\Local\Arduino15\packages\rp2040\hardware\rp2040\2.6.0/lib/libpico.a(float_aeabi.S.obj)
                0x000000001000bf28                __wrap___aeabi_ul2f
 .text.__wrap___aeabi_f2ulz
                0x000000001000bf44       0x14 C:\Users\tomas\AppData\Local\Arduino15\packages\rp2040\hardware\rp2040\2.6.0/lib/libpico.a(float_aeabi.S.obj)
                0x000000001000bf44                __wrap___aeabi_f2ulz
 .text.__wrap___aeabi_f2d
                0x000000001000bf58       0x14 C:\Users\tomas\AppData\Local\Arduino15\packages\rp2040\hardware\rp2040\2.6.0/lib/libpico.a(float_aeabi.S.obj)
                0x000000001000bf58                __wrap___aeabi_f2d
 .text.__aeabi_float_init
                0x000000001000bf6c       0x5c C:\Users\tomas\AppData\Local\Arduino15\packages\rp2040\hardware\rp2040\2.6.0/lib/libpico.a(float_init_rom.c.obj)
                0x000000001000bf6c                __aeabi_float_init
 .text.float_table_shim_on_use_helper
                0x000000001000bfc8       0x2c C:\Users\tomas\AppData\Local\Arduino15\packages\rp2040\hardware\rp2040\2.6.0/lib/libpico.a(float_v1_rom_shim.S.obj)
                0x000000001000bfc8                float_table_shim_on_use_helper
 .text.642float_shims
                0x000000001000bff4       0x44 C:\Users\tomas\AppData\Local\Arduino15\packages\rp2040\hardware\rp2040\2.6.0/lib/libpico.a(float_v1_rom_shim.S.obj)
                0x000000001000bff4                uint642float_shim
                0x000000001000bff6                ufix642float_shim
                0x000000001000c006                int642float_shim
                0x000000001000c008                fix642float_shim
 .text.float264_shims
                0x000000001000c038       0x4c C:\Users\tomas\AppData\Local\Arduino15\packages\rp2040\hardware\rp2040\2.6.0/lib/libpico.a(float_v1_rom_shim.S.obj)
                0x000000001000c038                float2int64_shim
                0x000000001000c03a                float2fix64_shim
                0x000000001000c042                float2uint64_shim
                0x000000001000c044                float2ufix64_shim
 .text.d2fix_a_float
                0x000000001000c084       0x5c C:\Users\tomas\AppData\Local\Arduino15\packages\rp2040\hardware\rp2040\2.6.0/lib/libpico.a(float_v1_rom_shim.S.obj)
 .text.float2double_shim
                0x000000001000c0e0       0x30 C:\Users\tomas\AppData\Local\Arduino15\packages\rp2040\hardware\rp2040\2.6.0/lib/libpico.a(float_v1_rom_shim.S.obj)
                0x000000001000c0e0                float2double_shim
 .text          0x000000001000c110       0x10 C:\Users\tomas\AppData\Local\Arduino15\packages\rp2040\hardware\rp2040\2.6.0/lib/libpico.a(mem_ops_aeabi.S.obj)
                0x000000001000c110                __aeabi_mem_init
 .text.memset   0x000000001000c120        0xc C:\Users\tomas\AppData\Local\Arduino15\packages\rp2040\hardware\rp2040\2.6.0/lib/libpico.a(mem_ops_aeabi.S.obj)
                0x000000001000c120                __wrap_memset
 .text.memcpy   0x000000001000c12c        0xc C:\Users\tomas\AppData\Local\Arduino15\packages\rp2040\hardware\rp2040\2.6.0/lib/libpico.a(mem_ops_aeabi.S.obj)
                0x000000001000c12c                __wrap_memcpy
                0x000000001000c12c                __wrap___aeabi_memcpy
 .text._Znwj    0x000000001000c138        0x8 C:\Users\tomas\AppData\Local\Arduino15\packages\rp2040\hardware\rp2040\2.6.0/lib/libpico.a(new_delete.cpp.obj)
                0x000000001000c138                _Znwj
 .text._ZdlPvj  0x000000001000c140        0x8 C:\Users\tomas\AppData\Local\Arduino15\packages\rp2040\hardware\rp2040\2.6.0/lib/libpico.a(new_delete.cpp.obj)
                0x000000001000c140                _ZdlPvj
 .text.multicore_fifo_pop_blocking_inline
                0x000000001000c148       0x14 C:\Users\tomas\AppData\Local\Arduino15\packages\rp2040\hardware\rp2040\2.6.0/lib/libpico.a(multicore.c.obj)
 .text.core1_trampoline
                0x000000001000c15c        0x2 C:\Users\tomas\AppData\Local\Arduino15\packages\rp2040\hardware\rp2040\2.6.0/lib/libpico.a(multicore.c.obj)
 .text.core1_wrapper
                0x000000001000c15e        0xc C:\Users\tomas\AppData\Local\Arduino15\packages\rp2040\hardware\rp2040\2.6.0/lib/libpico.a(multicore.c.obj)
                0x000000001000c15e                core1_wrapper
 .text.multicore_fifo_push_blocking_inline
                0x000000001000c16a       0x12 C:\Users\tomas\AppData\Local\Arduino15\packages\rp2040\hardware\rp2040\2.6.0/lib/libpico.a(multicore.c.obj)
 .text.multicore_fifo_pop_blocking
                0x000000001000c17c        0x8 C:\Users\tomas\AppData\Local\Arduino15\packages\rp2040\hardware\rp2040\2.6.0/lib/libpico.a(multicore.c.obj)
                0x000000001000c17c                multicore_fifo_pop_blocking
 .text.multicore_launch_core1_raw
                0x000000001000c184       0x6a C:\Users\tomas\AppData\Local\Arduino15\packages\rp2040\hardware\rp2040\2.6.0/lib/libpico.a(multicore.c.obj)
                0x000000001000c184                multicore_launch_core1_raw
 *fill*         0x000000001000c1ee        0x2 
 .text.multicore_launch_core1_with_stack
                0x000000001000c1f0       0x34 C:\Users\tomas\AppData\Local\Arduino15\packages\rp2040\hardware\rp2040\2.6.0/lib/libpico.a(multicore.c.obj)
                0x000000001000c1f0                multicore_launch_core1_with_stack
 .text.multicore_launch_core1
                0x000000001000c224       0x20 C:\Users\tomas\AppData\Local\Arduino15\packages\rp2040\hardware\rp2040\2.6.0/lib/libpico.a(multicore.c.obj)
                0x000000001000c224                multicore_launch_core1
 .text.get_driver
                0x000000001000c244       0x40 C:\Users\tomas\AppData\Local\Arduino15\packages\rp2040\hardware\rp2040\2.6.0/lib/libpico.a(usbd.c.obj)
 .text.configuration_reset
                0x000000001000c284       0x4c C:\Users\tomas\AppData\Local\Arduino15\packages\rp2040\hardware\rp2040\2.6.0/lib/libpico.a(usbd.c.obj)
 .text.invoke_class_control
                0x000000001000c2d0       0x1a C:\Users\tomas\AppData\Local\Arduino15\packages\rp2040\hardware\rp2040\2.6.0/lib/libpico.a(usbd.c.obj)
 .text.osal_queue_send.constprop.0.isra.0
                0x000000001000c2ea       0x30 C:\Users\tomas\AppData\Local\Arduino15\packages\rp2040\hardware\rp2040\2.6.0/lib/libpico.a(usbd.c.obj)
 *fill*         0x000000001000c31a        0x2 
 .text.tud_mounted
                0x000000001000c31c       0x10 C:\Users\tomas\AppData\Local\Arduino15\packages\rp2040\hardware\rp2040\2.6.0/lib/libpico.a(usbd.c.obj)
                0x000000001000c31c                tud_mounted
 .text.tud_suspended
                0x000000001000c32c       0x10 C:\Users\tomas\AppData\Local\Arduino15\packages\rp2040\hardware\rp2040\2.6.0/lib/libpico.a(usbd.c.obj)
                0x000000001000c32c                tud_suspended
 .text.tud_inited
                0x000000001000c33c        0xc C:\Users\tomas\AppData\Local\Arduino15\packages\rp2040\hardware\rp2040\2.6.0/lib/libpico.a(usbd.c.obj)
                0x000000001000c33c                tud_inited
 .text.tud_init
                0x000000001000c348       0x98 C:\Users\tomas\AppData\Local\Arduino15\packages\rp2040\hardware\rp2040\2.6.0/lib/libpico.a(usbd.c.obj)
                0x000000001000c348                tud_init
 .text.dcd_event_handler
                0x000000001000c3e0       0x7c C:\Users\tomas\AppData\Local\Arduino15\packages\rp2040\hardware\rp2040\2.6.0/lib/libpico.a(usbd.c.obj)
                0x000000001000c3e0                dcd_event_handler
 .text.dcd_event_bus_signal
                0x000000001000c45c       0x22 C:\Users\tomas\AppData\Local\Arduino15\packages\rp2040\hardware\rp2040\2.6.0/lib/libpico.a(usbd.c.obj)
                0x000000001000c45c                dcd_event_bus_signal
 .text.dcd_event_bus_reset
                0x000000001000c47e       0x2a C:\Users\tomas\AppData\Local\Arduino15\packages\rp2040\hardware\rp2040\2.6.0/lib/libpico.a(usbd.c.obj)
                0x000000001000c47e                dcd_event_bus_reset
 .text.dcd_event_setup_received
                0x000000001000c4a8       0x26 C:\Users\tomas\AppData\Local\Arduino15\packages\rp2040\hardware\rp2040\2.6.0/lib/libpico.a(usbd.c.obj)
                0x000000001000c4a8                dcd_event_setup_received
 .text.dcd_event_xfer_complete
                0x000000001000c4ce       0x38 C:\Users\tomas\AppData\Local\Arduino15\packages\rp2040\hardware\rp2040\2.6.0/lib/libpico.a(usbd.c.obj)
                0x000000001000c4ce                dcd_event_xfer_complete
 *fill*         0x000000001000c506        0x2 
 .text.usbd_edpt_open
                0x000000001000c508       0x30 C:\Users\tomas\AppData\Local\Arduino15\packages\rp2040\hardware\rp2040\2.6.0/lib/libpico.a(usbd.c.obj)
                0x000000001000c508                usbd_edpt_open
 .text.usbd_open_edpt_pair
                0x000000001000c538       0x4e C:\Users\tomas\AppData\Local\Arduino15\packages\rp2040\hardware\rp2040\2.6.0/lib/libpico.a(usbd.c.obj)
                0x000000001000c538                usbd_open_edpt_pair
 *fill*         0x000000001000c586        0x2 
 .text.usbd_edpt_claim
                0x000000001000c588       0x68 C:\Users\tomas\AppData\Local\Arduino15\packages\rp2040\hardware\rp2040\2.6.0/lib/libpico.a(usbd.c.obj)
                0x000000001000c588                usbd_edpt_claim
 .text.usbd_edpt_release
                0x000000001000c5f0       0x4c C:\Users\tomas\AppData\Local\Arduino15\packages\rp2040\hardware\rp2040\2.6.0/lib/libpico.a(usbd.c.obj)
                0x000000001000c5f0                usbd_edpt_release
 .text.usbd_edpt_xfer
                0x000000001000c63c       0x44 C:\Users\tomas\AppData\Local\Arduino15\packages\rp2040\hardware\rp2040\2.6.0/lib/libpico.a(usbd.c.obj)
                0x000000001000c63c                usbd_edpt_xfer
 .text.usbd_edpt_stall
                0x000000001000c680       0x34 C:\Users\tomas\AppData\Local\Arduino15\packages\rp2040\hardware\rp2040\2.6.0/lib/libpico.a(usbd.c.obj)
                0x000000001000c680                usbd_edpt_stall
 .text.usbd_edpt_clear_stall
                0x000000001000c6b4       0x34 C:\Users\tomas\AppData\Local\Arduino15\packages\rp2040\hardware\rp2040\2.6.0/lib/libpico.a(usbd.c.obj)
                0x000000001000c6b4                usbd_edpt_clear_stall
 .text.usbd_edpt_stalled
                0x000000001000c6e8       0x1c C:\Users\tomas\AppData\Local\Arduino15\packages\rp2040\hardware\rp2040\2.6.0/lib/libpico.a(usbd.c.obj)
                0x000000001000c6e8                usbd_edpt_stalled
 .text.tud_task
                0x000000001000c704      0x558 C:\Users\tomas\AppData\Local\Arduino15\packages\rp2040\hardware\rp2040\2.6.0/lib/libpico.a(usbd.c.obj)
                0x000000001000c704                tud_task
 .text._data_stage_xact
                0x000000001000cc5c       0x58 C:\Users\tomas\AppData\Local\Arduino15\packages\rp2040\hardware\rp2040\2.6.0/lib/libpico.a(usbd_control.c.obj)
 .text._status_stage_xact.isra.0
                0x000000001000ccb4       0x14 C:\Users\tomas\AppData\Local\Arduino15\packages\rp2040\hardware\rp2040\2.6.0/lib/libpico.a(usbd_control.c.obj)
 .text.tud_control_status
                0x000000001000ccc8       0x24 C:\Users\tomas\AppData\Local\Arduino15\packages\rp2040\hardware\rp2040\2.6.0/lib/libpico.a(usbd_control.c.obj)
                0x000000001000ccc8                tud_control_status
 .text.tud_control_xfer
                0x000000001000ccec       0x54 C:\Users\tomas\AppData\Local\Arduino15\packages\rp2040\hardware\rp2040\2.6.0/lib/libpico.a(usbd_control.c.obj)
                0x000000001000ccec                tud_control_xfer
 .text.usbd_control_reset
                0x000000001000cd40       0x14 C:\Users\tomas\AppData\Local\Arduino15\packages\rp2040\hardware\rp2040\2.6.0/lib/libpico.a(usbd_control.c.obj)
                0x000000001000cd40                usbd_control_reset
 .text.usbd_control_set_complete_callback
                0x000000001000cd54        0xc C:\Users\tomas\AppData\Local\Arduino15\packages\rp2040\hardware\rp2040\2.6.0/lib/libpico.a(usbd_control.c.obj)
                0x000000001000cd54                usbd_control_set_complete_callback
 .text.usbd_control_set_request
                0x000000001000cd60       0x1c C:\Users\tomas\AppData\Local\Arduino15\packages\rp2040\hardware\rp2040\2.6.0/lib/libpico.a(usbd_control.c.obj)
                0x000000001000cd60                usbd_control_set_request
 .text.usbd_control_xfer_cb
                0x000000001000cd7c       0xa4 C:\Users\tomas\AppData\Local\Arduino15\packages\rp2040\hardware\rp2040\2.6.0/lib/libpico.a(usbd_control.c.obj)
                0x000000001000cd7c                usbd_control_xfer_cb
 .text._prep_out_transaction
                0x000000001000ce20       0x42 C:\Users\tomas\AppData\Local\Arduino15\packages\rp2040\hardware\rp2040\2.6.0/lib/libpico.a(cdc_device.c.obj)
 *fill*         0x000000001000ce62        0x2 
 .text.tud_cdc_n_connected
                0x000000001000ce64       0x30 C:\Users\tomas\AppData\Local\Arduino15\packages\rp2040\hardware\rp2040\2.6.0/lib/libpico.a(cdc_device.c.obj)
                0x000000001000ce64                tud_cdc_n_connected
 .text.tud_cdc_n_available
                0x000000001000ce94       0x18 C:\Users\tomas\AppData\Local\Arduino15\packages\rp2040\hardware\rp2040\2.6.0/lib/libpico.a(cdc_device.c.obj)
                0x000000001000ce94                tud_cdc_n_available
 .text.tud_cdc_n_read
                0x000000001000ceac       0x28 C:\Users\tomas\AppData\Local\Arduino15\packages\rp2040\hardware\rp2040\2.6.0/lib/libpico.a(cdc_device.c.obj)
                0x000000001000ceac                tud_cdc_n_read
 .text.tud_cdc_n_peek
                0x000000001000ced4       0x18 C:\Users\tomas\AppData\Local\Arduino15\packages\rp2040\hardware\rp2040\2.6.0/lib/libpico.a(cdc_device.c.obj)
                0x000000001000ced4                tud_cdc_n_peek
 .text.tud_cdc_n_write_flush
                0x000000001000ceec       0x78 C:\Users\tomas\AppData\Local\Arduino15\packages\rp2040\hardware\rp2040\2.6.0/lib/libpico.a(cdc_device.c.obj)
                0x000000001000ceec                tud_cdc_n_write_flush
 .text.tud_cdc_n_write
                0x000000001000cf64       0x34 C:\Users\tomas\AppData\Local\Arduino15\packages\rp2040\hardware\rp2040\2.6.0/lib/libpico.a(cdc_device.c.obj)
                0x000000001000cf64                tud_cdc_n_write
 .text.tud_cdc_n_write_available
                0x000000001000cf98       0x18 C:\Users\tomas\AppData\Local\Arduino15\packages\rp2040\hardware\rp2040\2.6.0/lib/libpico.a(cdc_device.c.obj)
                0x000000001000cf98                tud_cdc_n_write_available
 .text.cdcd_init
                0x000000001000cfb0       0x7c C:\Users\tomas\AppData\Local\Arduino15\packages\rp2040\hardware\rp2040\2.6.0/lib/libpico.a(cdc_device.c.obj)
                0x000000001000cfb0                cdcd_init
 .text.cdcd_reset
                0x000000001000d02c       0x30 C:\Users\tomas\AppData\Local\Arduino15\packages\rp2040\hardware\rp2040\2.6.0/lib/libpico.a(cdc_device.c.obj)
                0x000000001000d02c                cdcd_reset
 .text.cdcd_open
                0x000000001000d05c       0xa4 C:\Users\tomas\AppData\Local\Arduino15\packages\rp2040\hardware\rp2040\2.6.0/lib/libpico.a(cdc_device.c.obj)
                0x000000001000d05c                cdcd_open
 .text.cdcd_control_xfer_cb
                0x000000001000d100       0xd8 C:\Users\tomas\AppData\Local\Arduino15\packages\rp2040\hardware\rp2040\2.6.0/lib/libpico.a(cdc_device.c.obj)
                0x000000001000d100                cdcd_control_xfer_cb
 .text.cdcd_xfer_cb
                0x000000001000d1d8       0xe4 C:\Users\tomas\AppData\Local\Arduino15\packages\rp2040\hardware\rp2040\2.6.0/lib/libpico.a(cdc_device.c.obj)
                0x000000001000d1d8                cdcd_xfer_cb
 .text.hidd_reset
                0x000000001000d2bc       0x14 C:\Users\tomas\AppData\Local\Arduino15\packages\rp2040\hardware\rp2040\2.6.0/lib/libpico.a(hid_device.c.obj)
                0x000000001000d2bc                hidd_reset
 .text.hidd_init
                0x000000001000d2d0        0xa C:\Users\tomas\AppData\Local\Arduino15\packages\rp2040\hardware\rp2040\2.6.0/lib/libpico.a(hid_device.c.obj)
                0x000000001000d2d0                hidd_init
 *fill*         0x000000001000d2da        0x2 
 .text.hidd_open
                0x000000001000d2dc       0xb4 C:\Users\tomas\AppData\Local\Arduino15\packages\rp2040\hardware\rp2040\2.6.0/lib/libpico.a(hid_device.c.obj)
                0x000000001000d2dc                hidd_open
 .text.hidd_control_xfer_cb
                0x000000001000d390      0x1e4 C:\Users\tomas\AppData\Local\Arduino15\packages\rp2040\hardware\rp2040\2.6.0/lib/libpico.a(hid_device.c.obj)
                0x000000001000d390                hidd_control_xfer_cb
 .text.hidd_xfer_cb
                0x000000001000d574       0x80 C:\Users\tomas\AppData\Local\Arduino15\packages\rp2040\hardware\rp2040\2.6.0/lib/libpico.a(hid_device.c.obj)
                0x000000001000d574                hidd_xfer_cb
 .text.tusb_init
                0x000000001000d5f4        0xa C:\Users\tomas\AppData\Local\Arduino15\packages\rp2040\hardware\rp2040\2.6.0/lib/libpico.a(tusb.c.obj)
                0x000000001000d5f4                tusb_init
 .text.tusb_inited
                0x000000001000d5fe        0x8 C:\Users\tomas\AppData\Local\Arduino15\packages\rp2040\hardware\rp2040\2.6.0/lib/libpico.a(tusb.c.obj)
                0x000000001000d5fe                tusb_inited
 *fill*         0x000000001000d606        0x2 
 .text.tu_edpt_validate
                0x000000001000d608       0x60 C:\Users\tomas\AppData\Local\Arduino15\packages\rp2040\hardware\rp2040\2.6.0/lib/libpico.a(tusb.c.obj)
                0x000000001000d608                tu_edpt_validate
 .text.tu_edpt_bind_driver
                0x000000001000d668       0x2a C:\Users\tomas\AppData\Local\Arduino15\packages\rp2040\hardware\rp2040\2.6.0/lib/libpico.a(tusb.c.obj)
                0x000000001000d668                tu_edpt_bind_driver
 .text.advance_pointer
                0x000000001000d692       0x18 C:\Users\tomas\AppData\Local\Arduino15\packages\rp2040\hardware\rp2040\2.6.0/lib/libpico.a(tusb_fifo.c.obj)
 .text._tu_fifo_correct_read_pointer
                0x000000001000d6aa       0x1e C:\Users\tomas\AppData\Local\Arduino15\packages\rp2040\hardware\rp2040\2.6.0/lib/libpico.a(tusb_fifo.c.obj)
 .text._ff_unlock
                0x000000001000d6c8        0xc C:\Users\tomas\AppData\Local\Arduino15\packages\rp2040\hardware\rp2040\2.6.0/lib/libpico.a(tusb_fifo.c.obj)
 .text._ff_pull_const_addr
                0x000000001000d6d4       0x58 C:\Users\tomas\AppData\Local\Arduino15\packages\rp2040\hardware\rp2040\2.6.0/lib/libpico.a(tusb_fifo.c.obj)
 .text._tu_fifo_peek_n
                0x000000001000d72c      0x12a C:\Users\tomas\AppData\Local\Arduino15\packages\rp2040\hardware\rp2040\2.6.0/lib/libpico.a(tusb_fifo.c.obj)
 *fill*         0x000000001000d856        0x2 
 .text._ff_push_const_addr
                0x000000001000d858       0x48 C:\Users\tomas\AppData\Local\Arduino15\packages\rp2040\hardware\rp2040\2.6.0/lib/libpico.a(tusb_fifo.c.obj)
 .text._tu_fifo_peek
                0x000000001000d8a0       0x48 C:\Users\tomas\AppData\Local\Arduino15\packages\rp2040\hardware\rp2040\2.6.0/lib/libpico.a(tusb_fifo.c.obj)
 .text._ff_lock
                0x000000001000d8e8       0x10 C:\Users\tomas\AppData\Local\Arduino15\packages\rp2040\hardware\rp2040\2.6.0/lib/libpico.a(tusb_fifo.c.obj)
 .text._tu_fifo_read_n
                0x000000001000d8f8       0x3e C:\Users\tomas\AppData\Local\Arduino15\packages\rp2040\hardware\rp2040\2.6.0/lib/libpico.a(tusb_fifo.c.obj)
 .text._tu_fifo_write_n.part.0
                0x000000001000d936      0x14a C:\Users\tomas\AppData\Local\Arduino15\packages\rp2040\hardware\rp2040\2.6.0/lib/libpico.a(tusb_fifo.c.obj)
 .text.tu_fifo_config
                0x000000001000da80       0x52 C:\Users\tomas\AppData\Local\Arduino15\packages\rp2040\hardware\rp2040\2.6.0/lib/libpico.a(tusb_fifo.c.obj)
                0x000000001000da80                tu_fifo_config
 .text.tu_fifo_count
                0x000000001000dad2       0x20 C:\Users\tomas\AppData\Local\Arduino15\packages\rp2040\hardware\rp2040\2.6.0/lib/libpico.a(tusb_fifo.c.obj)
                0x000000001000dad2                tu_fifo_count
 .text.tu_fifo_empty
                0x000000001000daf2       0x10 C:\Users\tomas\AppData\Local\Arduino15\packages\rp2040\hardware\rp2040\2.6.0/lib/libpico.a(tusb_fifo.c.obj)
                0x000000001000daf2                tu_fifo_empty
 .text.tu_fifo_remaining
                0x000000001000db02       0x1c C:\Users\tomas\AppData\Local\Arduino15\packages\rp2040\hardware\rp2040\2.6.0/lib/libpico.a(tusb_fifo.c.obj)
                0x000000001000db02                tu_fifo_remaining
 .text.tu_fifo_read
                0x000000001000db1e       0x36 C:\Users\tomas\AppData\Local\Arduino15\packages\rp2040\hardware\rp2040\2.6.0/lib/libpico.a(tusb_fifo.c.obj)
                0x000000001000db1e                tu_fifo_read
 .text.tu_fifo_read_n
                0x000000001000db54        0xa C:\Users\tomas\AppData\Local\Arduino15\packages\rp2040\hardware\rp2040\2.6.0/lib/libpico.a(tusb_fifo.c.obj)
                0x000000001000db54                tu_fifo_read_n
 .text.tu_fifo_peek
                0x000000001000db5e       0x28 C:\Users\tomas\AppData\Local\Arduino15\packages\rp2040\hardware\rp2040\2.6.0/lib/libpico.a(tusb_fifo.c.obj)
                0x000000001000db5e                tu_fifo_peek
 .text.tu_fifo_write
                0x000000001000db86       0x60 C:\Users\tomas\AppData\Local\Arduino15\packages\rp2040\hardware\rp2040\2.6.0/lib/libpico.a(tusb_fifo.c.obj)
                0x000000001000db86                tu_fifo_write
 .text.tu_fifo_write_n
                0x000000001000dbe6       0x12 C:\Users\tomas\AppData\Local\Arduino15\packages\rp2040\hardware\rp2040\2.6.0/lib/libpico.a(tusb_fifo.c.obj)
                0x000000001000dbe6                tu_fifo_write_n
 .text.tu_fifo_clear
                0x000000001000dbf8       0x34 C:\Users\tomas\AppData\Local\Arduino15\packages\rp2040\hardware\rp2040\2.6.0/lib/libpico.a(tusb_fifo.c.obj)
                0x000000001000dbf8                tu_fifo_clear
 .text.tu_fifo_set_overwritable
                0x000000001000dc2c       0x24 C:\Users\tomas\AppData\Local\Arduino15\packages\rp2040\hardware\rp2040\2.6.0/lib/libpico.a(tusb_fifo.c.obj)
                0x000000001000dc2c                tu_fifo_set_overwritable
 .text.hw_claim_lock
                0x000000001000dc50       0x18 C:\Users\tomas\AppData\Local\Arduino15\packages\rp2040\hardware\rp2040\2.6.0/lib/libpico.a(claim.c.obj)
                0x000000001000dc50                hw_claim_lock
 .text.hw_claim_unlock
                0x000000001000dc68       0x14 C:\Users\tomas\AppData\Local\Arduino15\packages\rp2040\hardware\rp2040\2.6.0/lib/libpico.a(claim.c.obj)
                0x000000001000dc68                hw_claim_unlock
 .text.hw_is_claimed
                0x000000001000dc7c       0x16 C:\Users\tomas\AppData\Local\Arduino15\packages\rp2040\hardware\rp2040\2.6.0/lib/libpico.a(claim.c.obj)
                0x000000001000dc7c                hw_is_claimed
 .text.hw_claim_or_assert
                0x000000001000dc92       0x3a C:\Users\tomas\AppData\Local\Arduino15\packages\rp2040\hardware\rp2040\2.6.0/lib/libpico.a(claim.c.obj)
                0x000000001000dc92                hw_claim_or_assert
 .text.hw_claim_unused_from_range
                0x000000001000dccc       0x54 C:\Users\tomas\AppData\Local\Arduino15\packages\rp2040\hardware\rp2040\2.6.0/lib/libpico.a(claim.c.obj)
                0x000000001000dccc                hw_claim_unused_from_range
 .text.running_on_fpga
                0x000000001000dd20       0x10 C:\Users\tomas\AppData\Local\Arduino15\packages\rp2040\hardware\rp2040\2.6.0/lib/libpico.a(platform.c.obj)
                0x000000001000dd20                running_on_fpga
 .text.lock_init
                0x000000001000dd30       0x10 C:\Users\tomas\AppData\Local\Arduino15\packages\rp2040\hardware\rp2040\2.6.0/lib/libpico.a(lock_core.c.obj)
                0x000000001000dd30                lock_init
 .text.critical_section_init_with_lock_num
                0x000000001000dd40       0x14 C:\Users\tomas\AppData\Local\Arduino15\packages\rp2040\hardware\rp2040\2.6.0/lib/libpico.a(critical_section.c.obj)
                0x000000001000dd40                critical_section_init_with_lock_num
 .text.critical_section_init
                0x000000001000dd54       0x14 C:\Users\tomas\AppData\Local\Arduino15\packages\rp2040\hardware\rp2040\2.6.0/lib/libpico.a(critical_section.c.obj)
                0x000000001000dd54                critical_section_init
 .text.flash_get_unique_id
                0x000000001000dd68       0x42 C:\Users\tomas\AppData\Local\Arduino15\packages\rp2040\hardware\rp2040\2.6.0/lib/libpico.a(flash.c.obj)
                0x000000001000dd68                flash_get_unique_id
 *fill*         0x000000001000ddaa        0x2 
 .text.hw_endpoint_init
                0x000000001000ddac       0xc8 C:\Users\tomas\AppData\Local\Arduino15\packages\rp2040\hardware\rp2040\2.6.0/lib/libpico.a(dcd_rp2040.c.obj)
 .text.reset_non_control_endpoints
                0x000000001000de74       0x3c C:\Users\tomas\AppData\Local\Arduino15\packages\rp2040\hardware\rp2040\2.6.0/lib/libpico.a(dcd_rp2040.c.obj)
 .text.dcd_rp2040_irq
                0x000000001000deb0      0x128 C:\Users\tomas\AppData\Local\Arduino15\packages\rp2040\hardware\rp2040\2.6.0/lib/libpico.a(dcd_rp2040.c.obj)
 .text.dcd_int_enable
                0x000000001000dfd8        0xc C:\Users\tomas\AppData\Local\Arduino15\packages\rp2040\hardware\rp2040\2.6.0/lib/libpico.a(dcd_rp2040.c.obj)
                0x000000001000dfd8                dcd_int_enable
 .text.dcd_set_address
                0x000000001000dfe4       0x14 C:\Users\tomas\AppData\Local\Arduino15\packages\rp2040\hardware\rp2040\2.6.0/lib/libpico.a(dcd_rp2040.c.obj)
                0x000000001000dfe4                dcd_set_address
 .text.dcd_connect
                0x000000001000dff8       0x10 C:\Users\tomas\AppData\Local\Arduino15\packages\rp2040\hardware\rp2040\2.6.0/lib/libpico.a(dcd_rp2040.c.obj)
                0x000000001000dff8                dcd_connect
 .text.dcd_init
                0x000000001000e008       0x64 C:\Users\tomas\AppData\Local\Arduino15\packages\rp2040\hardware\rp2040\2.6.0/lib/libpico.a(dcd_rp2040.c.obj)
                0x000000001000e008                dcd_init
 .text.dcd_edpt0_status_complete
                0x000000001000e06c       0x18 C:\Users\tomas\AppData\Local\Arduino15\packages\rp2040\hardware\rp2040\2.6.0/lib/libpico.a(dcd_rp2040.c.obj)
                0x000000001000e06c                dcd_edpt0_status_complete
 .text.dcd_edpt_open
                0x000000001000e084       0x20 C:\Users\tomas\AppData\Local\Arduino15\packages\rp2040\hardware\rp2040\2.6.0/lib/libpico.a(dcd_rp2040.c.obj)
                0x000000001000e084                dcd_edpt_open
 .text.dcd_edpt_close_all
                0x000000001000e0a4        0x8 C:\Users\tomas\AppData\Local\Arduino15\packages\rp2040\hardware\rp2040\2.6.0/lib/libpico.a(dcd_rp2040.c.obj)
                0x000000001000e0a4                dcd_edpt_close_all
 .text.dcd_edpt_xfer
                0x000000001000e0ac       0x24 C:\Users\tomas\AppData\Local\Arduino15\packages\rp2040\hardware\rp2040\2.6.0/lib/libpico.a(dcd_rp2040.c.obj)
                0x000000001000e0ac                dcd_edpt_xfer
 .text.dcd_edpt_stall
